:020000024000BC
:100000006FD0F267000000000018011800280128D6
:100010000228032800290129022903290429052986
:10002000062907290829002A012A022A032A042A64
:10003000052AA62AA0E60600A833040042040020F0
:10004000BC040020CA0300209C03002032030020CF
:100050004A3504008A35040028370400A839040012
:100060008C3A040008320400BA3104008C020020EB
:1000700036020020463F0400D0070020203504004F
:100080004E3C04003C8306001E8506008A8506005F
:1000900090380600C8380600D4680500485C0500A2
:1000A0009A7D06007E3C0400D8400600E2EF040082
:1000B00072F00400CCF0040066470400A44704007A
:1000C000244604000AB2040026AD0400480A0020B9
:1000D0005EBE0400C4C1040046A00400E89F040002
:1000E000AAA3040092A00400C69F04003EA004003E
:1000F0007C9F04000CA1040064A1040014A104006E
:1001000018A10400AEA104006CA104009CA104008D
:100110005CA6040060A6040008A1040010A104006D
:10012000ACA104005EA604005AA20400BAA7040011
:1001300022CF040096CF0400D0CF040056B40400B0
:100140006CB40400A4B40400EE94040014970400FA
:10015000F0970400066504009C5F0400028B040015
:10016000186004004A860400D6C306002EBC0600B0
:100170001AC1060034D8060000D706005EDB060070
:100180001ADB060056DB0600A6DC06000AAB0600FA
:1001900036DC060090CE0600B6CE0600D6CE0600AF
:1001A00016DD060006D50600A4D4060086DD06008E
:1001B0008EAD060022AE060042AE0600F4AD06008B
:1001C00056600600AE4B0600044F0600EC4C0600DD
:1001D000C6560600F27D0600347D06003EAB0600E2
:1001E000C2400400D8380600B8400600B0410600FE
:1001F000FC730600887406000A76060030B8040016
:10020000945F06005A5706008A490600185A0600ED
:100210005E4B0600BA0900204439060084DB060064
:100220001EDB060052DB06004EDB060032390400FE
:100230009AB504008CDB060042620600A663060045
:100240001264060078C1060088DB0600D2DB0600D7
:10025000D45B0500D6DB06001C250020342E0020D0
:1002600058C10600F6C20600DADB06002EDC0600E6
:1002700032DC060090DB0600CADB0600CEDB06009F
:100280006373B60082801C419105110523AEF5FE13
:10029000C5BFB737002037370020938787EF130794
:1002A00047616373F700828023A007009107D5BFE1
:1002B000411122C4B747024006C603A4C72023A6A3
:1002C00007200F10000011C199E5B747024023A68F
:1002D0008720014545A093073500C207C183F19BE4
:1002E000C207C183130740036366F7023737002054
:1002F00003254719373700208326C7186391A602C4
:10030000373700200327072269D3C207DD8D054553
:10031000029765BF3737002003250719E1BF7A210F
:1003200031EF5A21636CF704B73600203306F740EB
:1003300021489386C6196375C8028328050003D82F
:100340006600138687001D8F2A9661175AA2232004
:1003500016012313060010C15EA1130788FFFAA23D
:100360006EA1EE222105B387F540FEA2B7470240F9
:1003700023A68720B2402244410182800841BDBFAC
:10038000B747024003A8C72023A607200F1000008C
:1003900001E523A607218280B737002003AE471965
:1003A000B737002003A3C7188146F28763FE6708AA
:1003B00083A80700636DF50863EBA808138787001F
:1003C0006364E508F223216705076319E600373601
:1003D0000020034746FA05072302E6FA37360020D5
:1003E0001305C619CE237A21239307001306C619D5
:1003F0002E97420741837AA16383C70337350020D4
:1004000003250519630DF500EA2211E9DE2223A078
:1004100016012107BE95A105CEA27AA2B687984300
:1004200063046702B736002083A60619630ED7005F
:10043000762399EAD6234E231843A106AE96D6A377
:1004400098C37E22A1077EA2B747024099B7BE8615
:10045000C687A9BFB7370020B736002083A7471942
:1004600003A6C6182A87B305B5406314F6003A857B
:1004700029A8938687009C43E369D7FEE377F7FEBC
:100480002E85E3E4D5FEE3F2F5FE828023AC05FE83
:100490001C4181E70CC18280BA8703A787FF6DFFEB
:1004A00023ACB7FE8280411126C24AC0B744024045
:1004B00006C622C403A9C42023A604200F100000EE
:1004C00009E923A62421B240224492440249410171
:1004D00082802A842105BD654205C18D4181C93BC9
:1004E00011C9FD572320050042A17CA123A6242188
:1004F0002105D1BF23A624210145F1B701114AC826
:100500004EC6B747024006CE22CC26CA83A9C720D2
:100510002A8923A607200F10000037350020032466
:1005200085198144014609E889ECA1654A8597301F
:1005300004E0E780A06E25A08347E4FF639D2703C6
:10054000A1C0A68513058519973004E0E78040EC2B
:1005500069DCA1654A85973004E0E7804026F240D7
:100560006244B747024023A6372126854249D24438
:10057000B2490561828091E02286032484FF65B739
:10058000A284E5BFB737002083A7871E99E33E8585
:100590008280BA236315B7009823E30AA7FEDC47DD
:1005A000F5B7B747024003A7C72023A607200F10BF
:1005B000000001C599C1814711E6B747024023A653
:1005C000E7208280B386F50003C80600B306F50075
:1005D000850723800601E317F6FEC5B737470240BB
:1005E0008327C720232607200F10000019C191C1BF
:1005F00011E6374702402326F7208280910503A7A2
:10060000C5FF11057D16232EE5FEDDB737470240F5
:100610008327C720232607200F10000001C53307BA
:10062000C50011E6374702402326F72082800505E2
:10063000A30FB5FEE31DE5FEF5B7B747024083A65D
:10064000C72023A607200F10000081473307F500BD
:100650000307070019E7374702402326D7203E85C6
:1006600082808507E5B7011126CA4AC8B74702400C
:1006700006CE22CC83A4C7202A892E8623A6072053
:100680000F100000131506019305F004418132C6D6
:1006900005312A8401C53246CA8521372285F240B8
:1006A0006244B747024023A697204249D2440561DD
:1006B0008280B747024003A7C72023A607200F1058
:1006C000000001C599C1814711EAB747024023A63E
:1006D000E720054582808507E309F6FE3308F5002B
:1006E000B386F500034808009422E306D8FEB74716
:1006F000024023A6E72001458280B747024003A7B6
:10070000C72023A607200F1000009307F6FFBE9511
:100710002A966317C500B747024023A6E7208280C8
:10072000FD159C310505A30FF5FEE5B737470240DF
:100730008327C720232607200F10000001C5330799
:10074000C50019E6374702402326F720014582807D
:1007500005058346F5FFE397B6FEE31BE5FE374745
:1007600002402326F72005458280797126D2B734CE
:10077000002022D403A4841E06D64AD04ECE52CCEA
:1007800056CA5AC85EC662C455C4373A00203739C3
:100790000020B7390020814BB73A002037CBC90180
:1007A000130ACA1E1309C919938949233E2099EFD8
:1007B0005C44639A0B0023A4F41E032CC40022851E
:1007C000C1366284A9A823A6FB00C5BF83A70A1E61
:1007D00082971C443307F5406376F50003A7490070
:1007E0001D8F2A979306FB3763EAE6062328090044
:1007F0002E200820973004E0E78060FC5C405844DD
:10080000B1C70C4403A64900AE97BE8663E4B700A7
:1008100063E4C700B386C74014C4A28B3A8459F47A
:10082000B73700209387C719984B854663FCE604C9
:100830007D1798CBB250225492540259F249624A21
:10084000D24A424BB24B224C4561828063950B00E9
:1008500023A4E41E9DB723A6EB0085B703278A02D5
:1008600019CB63EDA7003385A74083270901637483
:10087000F5002328A900A28B404455B703A74900DF
:10088000BA97D5B723A8070075B701114EC6B74769
:10089000024006CE22CC26CA4AC852C483A9C72029
:1008A00023A607200F1000003734002093074423AD
:1008B000C843DC2713044423B9CFB73700209387FC
:1008C000873B03D7470B21CB83A4070B6385A40485
:1008D000B73700201387C719184B138AC719630F3E
:1008E000A70E373900208327091E829763E5A40EDF
:1008F0008327091E898C829703270A0163F3E4008A
:100900002687B307A7003E85544063E4E70063E40D
:10091000D7003385D740B747024023A637215C4034
:10092000639DA702B73400209384C4199848B73751
:10093000002083A7071E6315A70A82975440B74774
:1009400036FE938707C8B6973387A7003A85636456
:10095000F7006364D7003305D740B734002093878E
:100960004451DC539384445199CBB737002083A67C
:1009700007593707CDFF7D179C46F98F9CC611E1BB
:1009800048408547DCC4B737002083A747218297BA
:1009900005E1DC5089CFDC4499CB974006E0E78045
:1009A00040BE973006E0E780801B23A60400753B1D
:1009B000DC5091CBB737002003A70759B7063300A7
:1009C0001C47D58F1CC7F2406244D2444249B24909
:1009D000224A056182805C40BE9419BF268525BFEE
:1009E000829794485840B387A6003E8563E4D700B9
:1009F000E3E5E7F63385E7408DB7B737002023AC52
:100A0000A7EE11C5B73700200547238EE7EE828099
:100A1000B737002003A787EF411122C406C613840D
:100A200087EF11C30297B737002083C7C7EF93F74B
:100A3000F70F99E323200400B24022444101828051
:100A4000011126CAB734002022CC4AC89387442318
:100A500006CE4EC652C456C2DC27373900209384D6
:100A600044231304891C95E3B7370020938747512B
:100A7000D833058B19CBF8339946639BE60AA382DA
:100A80000700EF10F05F5C4482971C4491C382978B
:100A900037340020B73900209307C41903A7491E33
:100AA0009033130AC4198347C41993961700BA9652
:100AB0009622C9CA8347C41963EEC708230E0418D7
:100AC00037340020930744519C37130444516391F9
:100AD0000710B737002083A7071EF5C3DC40232883
:100AE000FA006131B737002083A74721E9CB7C307A
:100AF00011476366F70CB737002093870756DC274A
:100B0000918BD5EFB737002083C7C7EF93F7F70F67
:100B1000DDE783461A0003A6491E63C7D70C62446B
:100B2000F240D2444249B249224A924A0561B1BBDD
:100B3000F8339D46E39BE6F4A3820700EF10505480
:100B40001C4899B7850793F7F70F230EF418E3ECC9
:100B5000C7F48DB786073E970E2323100700034581
:100B6000C419B737002083A7471C13172500B73ACD
:100B70000020BA979C43239E0A1C829783D7CA1DE4
:100B80000347C41993C7F7FF7D8D9317170003A779
:100B9000491E3E971E235D8D0AA38347C41981C752
:100BA0008507230EF4188327891C81C78297232485
:100BB000091C0347C41983471A00E371F7F0F24098
:100BC0006244D2444249B249224A924A0561828033
:100BD0007C3093F7F70FE39E07EEA30404009730F1
:100BE00006E0E7802046F5B51397170032971A23E1
:100BF00079F785071DB7374702408326C720F1776D
:100C0000FD17F58F2326F72001000100B7370020DC
:100C10009387C719C84F832787262326D7206A05BD
:100C200093C7F7FF99835D8D8280B737002083C714
:100C3000F71989CFB737002083C7072491CBB7377F
:100C4000002003A347246307030002830545828035
:100C5000094582801305F00F8280B737002003C654
:100C6000473BB737002003A747F781476315F600D6
:100C7000814636858280BA8613078702835587FDB1
:100C8000E389A5FE850793F7F70FCDB7B7370020A7
:100C900003C7573BB737002083A707F92A86050704
:100CA00081463E859E236388C700850693076500BD
:100CB000E3E9E6FE01458280B737002003A787F805
:100CC00019E3014615A81C4703D8A700636B05016B
:100CD00083584700B38608016355D5008146639465
:100CE00016011843F1BF3E86C10703D3A7FF631760
:100CF000A30099C123900501328582808506C20632
:100D0000C182F1BFB737002003C6473BB737002089
:100D100003A7473581476315F600814636858280F3
:100D2000BA861307C703835567FCE389A5FE8507C9
:100D300093F7F70FCDB7032785116DCB411122C46F
:100D400006C65C258345E5042A8493F7C70F5CA596
:100D50001437522713958601618563F7C5066351E1
:100D60000506082793F6F60714B7054693E627000D
:100D70006314C50093E6170054A45C4389075CC361
:100D80004CB8032504112E864C430905EFF07F81F2
:100D9000832784115038D443DA27B296118FD4C3F5
:100DA000DAA789473CBCB73700200347640383C7F1
:100DB000E71F6371F7045C2493E707015CA41DA897
:100DC00093E717005CA46DBF9376F60F6359050295
:100DD0000827854513E627006314B50013E61700BE
:100DE00050A454B8A304070085473CBC8327841152
:100DF0009C43D5FBB240224401454101828093E7E8
:100E000017005CA454B8A3040700032504114C4345
:100E10000905EFF00FF9832784115038D443DA27FE
:100E2000B296118FD4C3DAA78D47C1B7054582802A
:100E3000B737002083A7474E411122C406C6858BD1
:100E40002A84D5E34165130525F5977005E0E78011
:100E500080C851C93C253EA583270412ADE3232059
:100E6000A4122322A41285472311F4042320050091
:100E70007C2854415EA5583418A5054718B5373766
:100E80000020032787531385170215811C437D1506
:100E90001375F50F9CC25C43DCC21C479CC65C47C3
:100EA000DCC61C4B9CCA5C4BDCCA1C4F9CCE5C4F06
:100EB000DCCE19CD9386060213070702C1BF832734
:100EC000441288C3835724042322A412850769BFD0
:100ED000B73700209387873B9A2705079AA7B24028
:100EE0002244410182805C2423090400054593C704
:100EF00047005CA4EDB71C2D93F7E70FC5EB1C3D35
:100F0000D5E73029542509CA3737002083456503C2
:100F10000347F71F63E7E50013F7060149CB0147D5
:100F200009C6C18A0357251E81C68356651E36979A
:100F30003DCFB737002003D5C7231307C712374665
:100F40000F00B335A702411113060624814622C4BF
:100F500026C206C67D543305A70297D006E0E78077
:100F60000023B737002083C73720B384A700B737E3
:100F7000002003A747458327070963F387003E84C2
:100F8000184375FBB737002083A7071E8297814758
:100F90006364A400B307A440B2402244B3B79700EF
:100FA00093C7170092443E854101828081473E8568
:100FB0008280B737002003A7C7537C53FDFF828090
:100FC00001114EC6B73900209387893B22CC03A478
:100FD000470A26CAB7340020938744239E274AC86D
:100FE000035964080325040906CE3309F902B747FB
:100FF0000F001387F7239387072452C456C25AC0A1
:101000009389893B938444233A993359F902636D58
:101010002503373A002083270A1E3309254182978A
:101020006367A9023309A940634609028357040490
:10103000A30F040085072310F4048347041463946A
:1010400007102285CD2D11A2DC403E95D9B7DC409A
:101050003E99C9BF83270A1E829703278408636FBE
:10106000E508198D7E3C9A248E07B387E7021307A3
:10107000003293870719B3D7E70263E5A708B74A99
:101080000F00138BFA23938A0A24835704048507DD
:101090002310F4048347041499E32285692D2285E3
:1010A000976005E0E78020B4631D052483260409CA
:1010B0008327C408D840B6973E8563E4D70063E42D
:1010C000E7003385E7407C3C035964082328A408E3
:1010D00085077CBC9E243309F9025A993359590378
:1010E000636C25053309254183270A1E82976369AE
:1010F000A9043305A940E34A05F80DBFDC40998FE8
:101100003E958DB7A1452285976005E0E780E0A573
:10111000A305A402B737002003A307226303031E1D
:101120006244F240D2444249B249224A924A024BB6
:101130008945154505610283330927412A996DB711
:10114000DC403E997DB72285512D2285976005E0D0
:10115000E78060A96317051A8A2483576408B74695
:101160000F001386F623B387A7029386062403276E
:101170000409230B040283AA4400B297B3D7D70211
:10118000636BF718B307F7408326C4082324F408D9
:10119000014BB387E6003E8963E4D70063E457015F
:1011A000338957411E3023282409A1CB83560404D8
:1011B0005A3037460F0056B03387E640B387E70210
:1011C0003A301306062481468145BA97C207C18387
:1011D0003385A7023EB097D006E0E78040FB11CDF3
:1011E0004A95333925012E99AA8763142B0163642C
:1011F0005501B30755412328F40883270A1E829717
:101200002A8983270A1E8297E30D25FF83270A1E5A
:101210000329840882976365A9103305A9406302F6
:10122000051283DA84008357640837490F001307D7
:10123000F923B387570313090924BA97B3D72703B0
:101240003737002003473720BA9763ECA70EB33532
:101250002503035A2402568681463305250397D079
:1012600006E0E780C0F2330BAA0033055A03374685
:101270000F00130606248146814597D006E0E780DB
:1012800000F10DC1B337250356868146B305B90277
:101290003305A902BE9597D006E0E78040EF3305FD
:1012A000AA402AB03545973006E0E78040EA23A2FD
:1012B000890A383485476318F706930700FD7CA434
:1012C000B737002003A5C74FDC24B5C7EFF0EFF216
:1012D000B736002003A6C653B7370020938747517F
:1012E0001547F8B35846F977FD17F98F5CC60F100C
:1012F000000083A7C6538966060B94C723A267071D
:10130000D8C7F2406244D2444249B249224A924A82
:10131000024B05618280B3065701B387F640ADB535
:10132000DC403E99DDBD930710FC7CA4B73700205C
:1013300003A5474F51BF8145973004E0E78000A6E1
:1013400041BFDC2423A2090A85C3B737002003A5C7
:10135000C74E973004E0E78000DFB7E700E03707CB
:10136000000223A2E72071BF8347940285456244AF
:10137000F240D2444249B249224A924A024BB395C2
:10138000F500C205C18101450561172304E067002E
:101390000343011122CC4AC84EC606CE26CA52C407
:1013A00056C25AC0383585472A842E8983290509B3
:1013B0006315F71E83570508035BC503373A002002
:1013C00093064A2383DA8600130A4A2363FF6719C8
:1013D0001429639CE618032785116318071803274F
:1013E000450A6314071874351D476390E6182A3DB3
:1013F000330BFB409307204E3305650383244409D8
:1014000037460F001306062481463305F502B73729
:10141000002083C72720B3549502B3B5AA02BE9417
:10142000C204C180231394083385AA0297D006E032
:10143000E780E0D5AA9933B5A9002E954E8783277A
:101440004A0019E163E4F9003387F940B384540397
:10145000B7460F009387F623938606242320E900DE
:10146000BE94B3D4D40293171B00A6976369F70EFA
:101470001D8F2320E900B739002083A7091E83248C
:101480000900829763EEA4103385A440635D050ACA
:1014900083A7091E373B0020130B4B23829703279A
:1014A00009006365E510198D7E3C03578B008E079C
:1014B000B387E7021307003293870719B3D7E70210
:1014C00063EBA70E374A0F00930AFA23130A0A2484
:1014D0008357040485072310F4048347041499E315
:1014E0002285912C2285975005E0E780C06F6DE141
:1014F000832604098327C40803274B00B6973E853B
:1015000063E4D70063E4E7003385E7407C3C835421
:1015100064082328A40885077CBC83578B00B38408
:10152000F402D694B3D444036363950CB30495409A
:1015300083A7091E23209900829763EEA40A3385AE
:10154000A440E34705F8B737002083C7372063E29C
:10155000A708B737002023AE874401459DA88326FE
:101560004A00B387F6403E9729B783576408374748
:101570000F00B38457039307F723A6979304072418
:10158000B3D4970263E79900B3849940232099006C
:10159000DDB583274A00BE99C5BF23A03501E1BD53
:1015A000B737002083A78723BE94F9BD83274B005C
:1015B000998F3E95D5BDA1452285975005E0E780DE
:1015C000C05AA305A402B737002083A7072281EFE2
:1015D0007D55F2406244D2444249B249224A924A7D
:1015E000024B05618280894515458297D5B7B304C2
:1015F0009740AA9435BF83274B00BE9489B721CD6D
:1016000001116C0022CC06CE2A84613339C1FD570A
:101610006307F502B73600209386C61EFC3A94563F
:10162000324791C285836360F702B307F7403EC635
:10163000B24503459402972004E0E780202EF24053
:10164000624405618280B736002083A686233697E0
:10165000E9BFBD32EDB78280B737002079711387BB
:10166000873B4AD00329C70906D622D426D24ECEBC
:1016700052CC56CA094763000906B7340020938A42
:10168000873B93874451FC339546938444510D47DF
:101690006383F604DC442A8A99CB973006E0E7801E
:1016A00040EE972006E0E780804B23A60400FD591A
:1016B0006C004A85F93915E937150020130505D561
:1016C000EFF0AFB3A147DCA0B737002083A7C75323
:1016D0000947F8D30D47B250225492540259F249A7
:1016E000624AD24A3A854561828063743501324448
:1016F000AA8903290900E31D09FAFD571307F00F12
:10170000E38BF9FC914763F187029307B4FF232031
:10171000FA0023A8FA0A0147DDFFB737002083A7A4
:1017200087232320FA0045BFB737002083A78723EC
:10173000ED17A297E9BF797126D206D622D44AD0F6
:101740004ECE52CC56CA5AC85EC683475503034490
:101750007513AA843E941374F40F9307400263F642
:1017600087001304B4FD1374F40F03AA841383AA2F
:10177000C413A38B841222865285D68597D006E0A7
:10178000E780609B058915E503CBD41201498149A7
:10179000337B6403930B50024A865285D68597D0DB
:1017A00006E0E7804099058915C5639169031374C4
:1017B000F90F238B8412B250225492540259F249E9
:1017C000624AD24A424BB24B456182808509E209A6
:1017D00093D989410509E31179FDE1BF8327850983
:1017E00003560504797193D60701BD8EC206C182E6
:1017F000358E1357764093575640898B058B5D8FF6
:1018000093573640918B5D8F93571640A18B5D8F18
:1018100093171600C18B5D8F9317360093F707025D
:101820005D8F931756009355860093F707041E06A5
:101830005D8F1376F60F518F93D7554013D63540F1
:10184000118A898BD18F13D67540D18F13D615404D
:10185000218AD18F13961500418AD18F13963500B6
:1018600013760602D18F13965500137606049E0553
:10187000D18F93F5F50FCD8FA20745465D8F3307C6
:10188000C70222D42A8426D252CC56CA032A8413F1
:10189000832AC4135AC806D6369742074183935702
:1018A0007740135557400989858BC98F13553740A9
:1018B0001189C98F135517402189C98F1315170036
:1018C0004189C98F1315370013750502C98F131588
:1018D000570093558700137505041E07C98F1377AA
:1018E000F70FD98F13D5354013D755401189098B80
:1018F000498F13D57540498F13D515402189498FDC
:10190000139515004189498F13953500137505020C
:10191000498F13955500137505049E05498F93F55E
:10192000F50F4D8F2207D98FB387C7024AD04ECE0D
:101930005EC662C4B697C207C18313D7774013D57A
:1019400057400989058B498F13D537401189498F35
:1019500013D517402189498F139517004189498F65
:101960001395370013750502498F1395570093D5CA
:101970008700137505049E07498F93F7F70FD98FDA
:1019800013D5354013D755401189098B498F13D58D
:101990007540498F13D515402189498F139515003E
:1019A0004189498F1395350013750502498F1395A9
:1019B0005500137505049E05498F93F5F50F4D8F5E
:1019C0002207D98FB387C702130650025285D685E6
:1019D000B697BD8E93940601C18033F6C402137B83
:1019E000F60F97C006E0E780007505890DED834787
:1019F000D41201498149B3849702130C5002C1806B
:101A00004A865285D68597C006E0E780C072058970
:101A1000937BF90F11C563863403850993F9F90F98
:101A20000509E31F89FD230B6413B250225492541D
:101A30000259F249624AD24A424BB24B224C4561AA
:101A400082805E8BCDB78327C508035685087971E0
:101A500093D60701BD8EC206C182358E13577640DC
:101A600093575640898B058B5D8F93573640918BEA
:101A70005D8F93571640A18B5D8F93171600C18B16
:101A80005D8F9317360093F707025D8F931756000B
:101A90009355860093F707041E065D8F1376F60FA5
:101AA000518F93D7554013D63540118A898BD18FEA
:101AB00013D67540D18F13D61540218AD18F139636
:101AC0001500418AD18F1396350013760602D18F07
:101AD00013965500137606049E05D18F93F5F50FE6
:101AE000CD8FA20745465D8F3307C70222D42A84D3
:101AF00026D252CC56CA032A040A832A440A5AC858
:101B000006D636974207418393577740135557407F
:101B10000989858BC98F135537401189C98F135592
:101B200017402189C98F131517004189C98F1315D3
:101B3000370013750502C98F131557009355870099
:101B4000137505041E07C98F1377F70FD98F13D5A7
:101B5000354013D755401189098B498F13D57540EE
:101B6000498F13D515402189498F13951500418957
:101B7000498F1395350013750502498F139555004C
:101B8000137505049E05498F93F5F50F4D8F2207B8
:101B9000D98FB387C7024AD04ECE5EC662C4B6970D
:101BA000C207C18313D7774013D557400989058BE6
:101BB000498F13D537401189498F13D51740218993
:101BC000498F139517004189498F13953700137575
:101BD0000502498F1395570093D5870013750504A7
:101BE0009E07498F93F7F70FD98F13D5354013D739
:101BF00055401189098B498F13D57540498F13D5ED
:101C000015402189498F139515004189498F1395F6
:101C1000350013750502498F13955500137505049A
:101C20009E05498F93F5F50F4D8F2207D98FB38706
:101C3000C702130650025285D685B697BD8E93947F
:101C40000601C18033F6C402137BF60F97C006E08D
:101C5000E780604E05890DED8347140801498149ED
:101C6000B3849702130C5002C1804A865285D685F0
:101C700097C006E0E780204C0589937BF90F11C5DA
:101C800063863403850993F9F90F0509E31F89FD7C
:101C9000230F6407B250225492540259F249624A07
:101CA000D24A424BB24B224C456182805E8BCDB70B
:101CB0008327450903568508797193D60701BD8EA0
:101CC000C206C182358E1357764093575640898B92
:101CD000058B5D8F93573640918B5D8F93571640E0
:101CE000A18B5D8F93171600C18B5D8F9317360004
:101CF00093F707025D8F931756009355860093F76D
:101D000007041E065D8F1376F60F518F93D755404B
:101D100013D63540118A898BD18F13D67540D18F58
:101D200013D61540218AD18F13961500418AD18F81
:101D30001396350013760602D18F1396550013764D
:101D400006049E05D18F93F5F50FCD8FA20745466A
:101D50005D8F3307C70222D42A8426D252CC56CABA
:101D6000032A040B832A440B5AC806D63697420727
:101D7000418393577740135557400989858BC98F05
:101D8000135537401189C98F135517402189C98FC1
:101D9000131517004189C98F1315370013750502F4
:101DA000C98F1315570093558700137505041E0737
:101DB000C98F1377F70FD98F13D5354013D75540F7
:101DC0001189098B498F13D57540498F13D515405B
:101DD0002189498F139515004189498F1395350045
:101DE00013750502498F13955500137505049E055B
:101DF000498F93F5F50F4D8F2207D98FB387C7020F
:101E00004AD04ECE5EC662C4B697C207C18313D70E
:101E1000774013D557400989058B498F13D5374033
:101E20001189498F13D517402189498F13951700C0
:101E30004189498F1395370013750502498F139512
:101E4000570093D58700137505049E07498F93F7B4
:101E5000F70FD98F13D5354013D755401189098B0A
:101E6000498F13D57540498F13D515402189498F66
:101E7000139515004189498F139535001375050297
:101E8000498F13955500137505049E05498F93F5E9
:101E9000F50F4D8F2207D98FB387C7021306500263
:101EA0005285D685B697BD8E93940601C18033F6D0
:101EB000C402137BF60F97C006E0E780C0270589B0
:101EC0000DED8347F40801498149B3849702130C4F
:101ED0005002C1804A865285D68597C006E0E780C9
:101EE00080250589937BF90F11C563863403850925
:101EF00093F9F90F0509E31F89FD230F6407B25019
:101F0000225492540259F249624AD24A424BB24B8D
:101F1000224C456182805E8BCDB74111B7370020DE
:101F200026C283A4074106C622C44AC08547C1C44D
:101F300003A4C40A854741C03C241307700A639375
:101F4000E70858301C34B736002013864623B38781
:101F5000E7021A265042B387E7021307003293873D
:101F60000719B3D7E70203A74409938446233E9792
:101F70003A896364F7006364C7003309C740B73721
:101F8000002083A7071E232025018297B307A940BD
:101F90006374A900D840BA9781E79307F00F21A88E
:101FA00058309306204E3307D702E3F8E7FE930735
:101FB00080FA3CA48147B2402244924402493E85C3
:101FC000410182801307800AE399E7FCB7370020BC
:101FD00083A7071E82972A893545972006E0E78068
:101FE0000017B7370020938747512D47F8B3583073
:101FF0001C34B736002093864623B387E7029A261F
:10200000D442B387E7021307003293870719B3D787
:10201000E70203A744093E973A866364F7006364C6
:10202000D7003306D740E31AC9F637D505001305A4
:10203000459BEFE09F9CB737002083A7C753094714
:10204000F8D7A1BF397122DC3734002093074451FF
:102050009C4F06DE26DA4AD84ED652D456D25AD0F3
:102060005ECE62CC66CA6AC86EC613970701635D0E
:10207000071EB737002083A4074183A9C40A83C77A
:10208000990003A7C9009207330CF70003452C0001
:10209000314705053305E50203574C003A954205E3
:1020A0004181EFE04FC0AA8B630B051C130DC500E7
:1020B0002324A50103462C00B145F97A3306B60264
:1020C0001304445123130C000149373A0020373BD5
:1020D0000020B73C0020930D9005FD1A6A96232638
:1020E000CC0003C679009307D0070325CA533306F3
:1020F000F60285671CC5B7073300060630D10326F4
:102100008B500C4293F5F5E70CC20C4293F5F5E7C2
:1021100093E505100CC203A80C5983258800DD8DBA
:102120002324B80083A509002328B5050CC68355D0
:102130006C000326CC002E962324CD0003461C0001
:10214000930550024A96A301CD0003C50408014639
:10215000A3000400972006E0E78000D70326CA53B7
:102160004846B37555014CC60F1000000326CA53EC
:10217000896503288B500CC6930500F84CA0832575
:102180000800B1818D89E1E1930560196CD248C6E0
:10219000A30204008545A30004000CC2D5259720A6
:1021A00006E0E780A0F21030058A5DCAEA85268540
:1021B00097C005E0E780C0A60DED03465D004DC267
:1021C00083556C0003554C00B29563DBA508AC2821
:1021D000A848918D8905AA9503258D00EFE06FBC75
:1021E00023020D0083455D0003566C002E962313D9
:1021F000CC008325CA53310DB0517DFE03462C001F
:1022000005091379F90FE36EC9EC98245E85A38163
:10221000EB0083470C00A3820B002383CB002382B7
:10222000FB006254F250D2544259B259225A925A87
:10223000025BF24B624CD24C424DB24D21611713FE
:1022400005E0670003E1832508000948B1818D8915
:10225000639505019305E04315BF9305E01B3DB76A
:102260007D562302CD0071B7B737002083A7C7532F
:10227000FC5791C7B73700200547238EE7EEF25091
:102280006254D2544259B259225A925A025BF24BCA
:10229000624CD24C424DB24D216182800111B73760
:1022A000002022CC03A4474826CA4AC84EC606CE00
:1022B000AA8413092500854905C09C303830858BD8
:1022C0006304F700405CCDBF1946930544004A857E
:1022D000EFE02FBEE31835FF2285F2406244D2447E
:1022E0004249B249056182804111B737002022C4BA
:1022F00003A4474826C24AC006C6930425000549E0
:1023000001E82285B2402244924402494101828080
:10231000A6851305A40297C005E0E780A040E3026C
:1023200025FF405CF1BF4111B737002022C403A450
:10233000474826C24AC006C693042500054901E85D
:102340002285B24022449244024941018280A685FE
:102350001305A40197C005E0E780C03CE30225FF18
:10236000405CF1BF011122CC604126CA4AC84EC66A
:1023700052C406CEAA841D4A130965058549BC448A
:102380006364F400054591A0D8345C2063174705C9
:1023900003C784026304F7000040D5B7583083C7F1
:1023A0005405E31BF7FE1946CA8513056400EFE0E8
:1023B0004FB0E31335FF582483C79402E31EF7FCA4
:1023C0007A24BE34E31AF7FC0145F2406244D24459
:1023D0004249B249224A05618280E31FF7FA583028
:1023E00083C75405E31AF7FA1946CA851305640032
:1023F000EFE02FACE31235FBC1BF4111B73700202E
:1024000022C403A4874306C626C24AC079C88347AC
:10241000840B1307700A6393E70A0347140E83477C
:10242000A40BB736002013864623B387E7021A268B
:10243000938446235042B387E70213070032938701
:102440000719B3D7E7020327440A3E973A89636422
:10245000F7006364C7003309C740B737002083A77C
:10246000071E232025018297B307A9406374A900A2
:10247000D840BA978DC70347140E9306204E3307F2
:10248000D70263FEE700930780FA230CF40A0144A5
:102490002285B2402244924402494101828037356C
:1024A000060013054592EFE04FD5B737002083A70C
:1024B000C75309471304F00FF8D7D9BF1307800A91
:1024C0001304F00FE396E7FC373506001305459239
:1024D000EFE0AFD2B737002083A7C7530947F8D73B
:1024E00045BF054475B70111B737002022CC03A4BE
:1024F000C74726CA06CE2AC42EC6854419E401451C
:10250000F2406244D244056182809C841830858BFD
:102510006304F7000044DDB719469305A1001305D5
:102520002400EFE00F99E31795FE0545D1BFB736BC
:10253000002083A746501307001098C323A007006C
:102540001831034825002207420842970348050036
:102550004297034835006208429798D7583103489C
:102560006500220742084297034845004297034806
:10257000750062084297D8D718350348A50022078E
:10258000420842970348850042970348B500620815
:10259000429798DB58350348E500220742084297E6
:1025A0000348C5006835429762052A97D8DB983101
:1025B000A821220742052A9788212A97A831620577
:1025C0002A9798CFD831E821220742052A97C821B7
:1025D0002A97E83162052A97D8CF9835A82522078F
:1025E00042052A9788252A97A83562052A9798D305
:1025F000D835E825220742052A97C825EC352A97C1
:10260000E2052E97D8D3D843759BD8C3D843136718
:102610001700D8C398431367170098C303A7465001
:102620005C43858BBDE71C4F01451CA283A7465028
:102630009C4FA1831CB283A746509C4FC1833CA2F0
:1026400083A746509C4FE1833CB283A74650D84FA6
:1026500058A2D84F218358B2D84F418378A2D84F7F
:10266000618378B2985318A69853218318B698536B
:10267000418338A69853618338B6D85358A6D853A7
:10268000218358B6D853418378A6DC53E1837CB6C6
:102690008280010061B7B737002003A7C753160532
:1026A000136505083C4B93E707083CCBB737002080
:1026B00083A7475003A7450E88C398CB03A7850E71
:1026C0000145D8CB03A7C50B98CF03A7050CD8CFDE
:1026D00003A7450C98D303A7850CD8D303A7C50C33
:1026E00098D703A7050DD8D703A7450D98DB03A7F7
:1026F000850DD8DB03A7C50D98C703A7050ED8C75E
:1027000098431367070498C38280B737002003A754
:10271000C7531605136505083C4B93E707083CCBE8
:10272000B737002083A7475003A7C50E88C398CBAF
:1027300003A7050F0145D8CB03A7C50B98CF03A767
:10274000050CD8CF03A7450C98D303A7850CD8D385
:1027500003A7C50C98D703A7050DD8D703A7450D28
:1027600098DB03A7850DD8DB03A7C50D98C703A782
:10277000050ED8C798431367070498C3B7370020DE
:1027800093874751130700F8F8A38280B7360020DB
:1027900003A7865041114AC01C5F06C622C4998314
:1027A00026C2858B3689B5CF9307000637340020C3
:1027B0001CDF834744519304445193F7070489CFA6
:1027C000B737002083A7071E8297C8CC83474451A0
:1027D00093F7F70B230AF4508347445193F707020A
:1027E00085C383474451373700200327C75393F7E6
:1027F000F70D230AF450DC48A16614C786077CD77E
:10280000DC2093F7070491EF8547DCB0B737002051
:1028100083A7C753096798C7130700FCD8A0984837
:10282000F8D3032789501C5F9183858B89CBC147DF
:102830001CDFB7370020938747518546D4A31C5F20
:102840009D83858B91CB930700081CDFB737002051
:10285000938747510547D8A3B737002083A7475030
:10286000D8430583058B19C7D843759BD8C3D84374
:10287000799BD8C3B24022449244024941018280EC
:10288000B7370020B736002003A6C75393874651B9
:1028900003C74651058B19E79833058B01E778523A
:1028A00065FBD833A38207008280373800200327D6
:1028B00088501C5F9583858BBDE701C61C5BBD837B
:1028C0001CA29DC683278850985B460793576701D3
:1028D0006356070093E707C0C207C183039706004A
:1028E000C207C18709C7BA970947B3C7E7029EA2C3
:1028F00085C11C3191CF3E951C350547194593F68E
:10290000F7066393E602E207E187394563CE0700E5
:10291000832788503737002001459C5FED838D8BDE
:10292000A30FF750828005458280411122C406C65C
:102930003734002026C20327C4533DE5AE877453C5
:10294000FDFEB7340020938444513E85B285238137
:102950000400971006E0E780C042B737002083A745
:102960008750B70680009843558F98C3D857719BFE
:10297000D8D78327C453A3820400A3800400094747
:1029800098C38326C453B737002093874751B82391
:10299000058B11E7B833058B19E3F8526DFBB24094
:1029A00022449244410182808D47631FF500B7376E
:1029B000002083A78750B70680009843558F98C39F
:1029C000D857719BD8D775BF8547E31CF5FA544794
:1029D000F977FD17F58F5CC70F1000008327C453EC
:1029E0000967130600F898C73737002013074751C7
:1029F00050A33737002003268750184231830D8BB0
:102A000011E713076019F8D3D4C7A5BF18420946C8
:102A100031830D8B6315C7001307E043EDB7130730
:102A2000E01BD5B75D7152DC373A002003278A508E
:102A300086C6A2C4A6C2CAC04EDE1C43B739002057
:102A40003739002093F7F7E793E707081CC383A6FD
:102A500009593707CEFF7D179C46130680022A844A
:102A6000F98F9CC68327C9532800AE8423A8070486
:102A700093051008EFD09FB93545971006E0E78021
:102A8000006D83278A509376F41F3706330023A402
:102A90000700984B370FFCFF4E881367F70398CB5E
:102AA000F84FCA88130510F8137707E0558FF8CF51
:102AB0009843F576FD16758F98C337370020832627
:102AC000C95313074751A3020700A3000700054796
:102AD00098C29843D285B70204001377F7E798C3EA
:102AE00098439303802511491377F7E7136707107D
:102AF00098C303A709597D1F85491C47930F80027E
:102B0000D18F1CC793079005BCCA014734001353EB
:102B1000370026938347030013767700B3D7C74067
:102B2000858BE1C383A78550832E0859239C070416
:102B30002390070603AECE02137EDEFF23A6CE034C
:102B400083AE0700137EF70793FE0EF833EECE0137
:102B500023A0C70103AE4702336E5E0023A2C70362
:102B600083AEC853014E23A27E0603DA070663072D
:102B70004E0303AE0703038A0600135EFE00620ED7
:102B8000135E8E416358CA0103AE0703135EFE0055
:102B90002380C60103DE0706137EFE0F03AA4E063E
:102BA00063060A0003DA8705E37F49FB03AE4702A9
:102BB000337EEE0123A2C70383870600635CF40023
:102BC000034E03003396C9001346F6FF3376C60161
:102BD0002300C3003E8663D3A7002A86131586010F
:102BE000618505071377F70F8506E312F7F3B64003
:102BF000264496440649F259625A61618280B73789
:102C0000002083A7C753D8479316170163D2060243
:102C100098479316170163DD06007D57B8D73737FD
:102C200000201307C719544F850654CF116798C762
:102C300098470D83058B11CF373700201307475175
:102C4000342393E6160034A3930600F854A32147D7
:102C500098C79847058B19CB373700201307475182
:102C6000143393E6160014B3054798C798470983B1
:102C7000058B09E798470583058B31CB3737002053
:102C800013064751A30206009447B735002083A5D9
:102C900085508982858AE5C69441B1828D8AE9EEA4
:102CA000A84B54521376050294324DC2F9E29306B2
:102CB000D005D4CF8346475193E61600230AD75058
:102CC000114798C7D855719B13671700D8D59847F7
:102CD0009316370163D40602373700209306873BEB
:102CE00003C6C6071307873B418A45C203C7C60709
:102CF00013670702238EE606056798C79847931661
:102D0000270163DF0600373700201307475154239C
:102D1000E206E18663D40600854654A3096798C796
:102D200098479316070163D206023737002013072E
:102D3000873B8346D707858AADCA8346D70793E684
:102D40002600A30ED706216798C78280ADD205461C
:102D50006395C60093061006A9BF09466395C60091
:102D600093065006B9B70D466395C60093069006C4
:102D700089B79306B00635BF9306C0061DBF38322B
:102D80001367170038B209472DBF8346C7070946A6
:102D9000BD8A6388C6008346C7070D46BD8AE39D8A
:102DA000C6F49146230ED70681BF8346D707918A82
:102DB000D9DA8346D70793E6860061B7B737002094
:102DC00083A7C753B736002013874651904710CFCB
:102DD00090470D82058A11CA30231366160030A36E
:102DE000130600F850A3214690C79047058A19C6DC
:102DF00010331366160010B3054690C7904709823A
:102E0000058A09E690470582058A31C6A3020700B4
:102E10009047B735002083A585500982058A59CA95
:102E2000904131820D8A41E6A84B5053137505023B
:102E3000103221C935EA1306D005D0CF03C646515A
:102E400013661600238AC650914694C7D455F19A4A
:102E500093E61600D4D5944713962601635B0600CB
:102E60005423E206E18663D40600854654A309672D
:102E700098C798479316070163D40600216798C73F
:102E8000828055DA05456315A6001306100675B74E
:102E900009456315A6001306500645B70D45631591
:102EA000A6001306900651BF1306B00679B71306A5
:102EB000C00661B7343393E6160034B3894671B760
:102EC00037370020B73600201386065413070756FD
:102ED0005C372C3E484AAE97FD8BB355F5001CB2CB
:102EE0005CB785898DE9183B814613080002B3F76A
:102EF000E7020147B355E50085899378F70F89C943
:102F00006395D700A30016018280850693F6F60F1D
:102F10000507E31107FF8280B737002093874751E9
:102F2000DC3393F7F70FD1EBB737002083A7071EE9
:102F3000411122C44AC006C626C2829737390020F2
:102F4000930709568047130909566302A40663686C
:102F50008504018DB734002093870454BC2F13548B
:102F60005500938404546364F40485676371F40426
:102F7000813FBC2C032789009396570036971D8C00
:102F80002324E900E376F4FE22448830B2409244E0
:102F9000024981454101171306E067004362B737D4
:102FA000002083A7872333848740229565B7B240EA
:102FB000224492440249410182808280B737002036
:102FC00083A7071E011122CC26CA52C406CE4AC8C6
:102FD0004EC68297B7340020938704568047014A33
:102FE0006300A4069384045663658506018D373714
:102FF000002093070754BC2F13545500137AF50192
:1030000013090754636BF402B739002093894923ED
:10301000453D8346A90103A8840083A54900139771
:1030200056004297158C3A86636407016364B700C3
:103030003306B74090C4E37DD4FC1604336A4401E0
:10304000F24062445285D2444249B249224A056163
:103050008280B737002083A7872333848740229557
:1030600079B7B737002003A7C753856793870777DA
:103070007CD3B737002083A7075983A60709139687
:1030800056006358060083A607091396660063443A
:1030900006007453FDF28280EFD09F97730000000A
:1030A00000000000970200009382820C038302005C
:1030B00023800200630F0300F32510342EC0970510
:1030C00000009385A5FD73901534EFF03FCF73009A
:1030D000203086DCEFF0BFB2E650828000000000B6
:1030E000B73700203737002083A747190327C718B1
:1030F00001456313F7008280F62399E2D6233695C3
:103100009C43C5BFB737002083A5C71E37370020B3
:103110009387C71E13860522232AC718DA239387AD
:1031200085FFB73600204111BA97056523A6F6182A
:1031300006C61D05935637006374E500930600200C
:103140003307D600373500202328E51823A0E522D1
:10315000E11656A2231306001CC3998FE1175EA344
:1031600023130700B53FB240B73700202391A71AB9
:1031700041018280B73700203737002083A74719E5
:103180008326C71801456393F6008280FA2309E776
:10319000DA236373E5003A859C43F5B7184183A7AA
:1031A00085FF6319B7001CC1FD5723AC05FE238FB3
:1031B000F5FE8280232CF6FEC5BF411122C426C233
:1031C0003744024006C68324C420232604200F105F
:1031D000000009E9232694201545B2402244924478
:1031E000410182800347E5FF9307F00F6306F70074
:1031F000232694201145D5B797D0FB1FE78080F197
:10320000014523269420D1BF411126C24AC0B744AC
:10321000024006C622C403A9C42023A604200F101E
:10322000000089E523A62421154515A0B737002005
:1032300083C7D7192A842E856375F400894763EE06
:103240008700A53FB747024023A627210D45B2407E
:103250002244924402494101828083A785FF99E775
:1032600003C7E5FF9307F00F6308F700B937B747C7
:10327000024023A627214DBF37350020238F85FE2E
:103280001305851997D0FB1FE78080F9A16522857A
:103290006D2C014523A624215DBFB737002023AC48
:1032A00007188280BDCD797122D406D626D24AD0A5
:1032B0004ECE01444147B3D78540858BB1CF12052F
:1032C000314722953305E502B737002003A9C7220D
:1032D0008544B3948400C204C180BE892A9903271F
:1032E000090011C7032549002EC60297B245314790
:1032F0003304E40283A7C9223E941C4489E72320B7
:10330000090023220900B2502254A58D025992547B
:10331000F2492E85456182800504E31EE4F881446C
:10332000DDB72E85828041111397050122C406C6A0
:1033300026C24AC041872E846351070297D0FB1FE3
:10334000E78000F511C1953DA1673D8C2285B24013
:1033500022449244024941018280EDD9AA87014763
:103360004146B356E440858A9DCA9207BA97B14652
:10337000B387D702B736002003A9C6228544B39489
:10338000E400C204C1803E99832709000325490057
:1033900082972320090023220900258C45BF0507B9
:1033A000E311C7FC8144D5BF411126C2B747024093
:1033B00006C622C483A4C72023A607200F1000003E
:1033C000B737002083A7072137340020130484EC8B
:1033D00091C782971C403E9508C031A0B7370020A6
:1033E00083A7071EFDF71C40374703001307D73F8D
:1033F000B387E70237A72600130737ECB240BA9726
:103400001CC0B747024023A697200840224492449C
:1034100041018280797126D2B747024006D622D474
:103420004AD04ECE52CC56CA5AC85EC662C483A495
:10343000C72023A607200F10000005E123A6972030
:103440000945B250225492540259F249624AD24A72
:10345000424BB24B224C45618280B737002083A794
:10346000071EBA8A368AB28B2E8BAA898297B73703
:10347000002003A7C7223E890144B146C147330C4F
:10348000D40233068701104259E2C165938505F0E5
:10349000414597D0FB1FE780E0BA19EDB737002010
:1034A00083A7072281C7814511458297B74702400C
:1034B00023A697202D4571B7B737002003A7871E95
:1034C00039E323A4A71E230005008327C92205474B
:1034D0003317870023260500232475013AA12322F0
:1034E0005501E29723A0370123A2670123A45701C6
:1034F00063040A0023008A00B747024023A69720EE
:10350000014581B73E875C47F5FF48C76DBF05049D
:10351000E317F4F6B747024023A69720214515B7D5
:10352000B737002083A70723411122C406C63734CA
:1035300000201304C41989C782975C483E9548C887
:103540004848B240224441018280B747024083A6E6
:10355000C72023A607200F1000003737002003479D
:10356000D7196370E50237360020131715000325BD
:10357000461E3A951A21D98D0EA123A6D7200145C2
:10358000828023A6D7200D458280B747024083A6BC
:10359000C72023A607200F1000003737002003475D
:1035A000D7196372E502373600201317150003257B
:1035B000461E93C5F5FF3A951A21F98D0EA123A653
:1035C000D7200145828023A6D7200D458280011196
:1035D0004AC83747024006CE22CC26CA4EC652C43D
:1035E0000329C720232607200F100000130705FF1B
:1035F0001377F70FFD4763E3E70AB146B306D50239
:10360000B737002003A7C72236971C43C1CB93547A
:10361000450005443D893315A4001314050141807C
:10362000AE892685A28597D0FB1FE780E0CE2A8A47
:1036300029C9A2852685913FB737002083A7071E99
:10364000B73400209384442382979E242A848146A1
:10365000B385370313060064B3B737031385053208
:10366000B335B500BE95EFA0520BB30785003E877A
:10367000D44063E4A70063E4D7003387D740232412
:10368000EA00B747024023A627210145F2406244E1
:10369000D2444249B249224A05618280B74702407A
:1036A00023A627210945DDB701114AC8B7470240C3
:1036B00006CE22CC26CA4EC603A9C72023A60720C1
:1036C0000F100000BD4763EBA70431473307E50245
:1036D000B737002083A7C722BA979C43A1C30544EC
:1036E0003314A40042044180AE840145A28597D0E2
:1036F000FB1FE78060C2AA8911C5A285014571350B
:1037000023A49900B747024023A627210145F24090
:103710006244D2444249B24905618280B7470240BF
:1037200023A627210945E5B7797126D252CCB744A3
:10373000024006D622D44AD04ECE56CA5AC85EC6D9
:1037400003AAC42023A604200F100000B7370020CE
:1037500083C7D7196378F500B737002083AB071EFE
:1037600063970B00B747024023A6472199A037393A
:10377000002013094923AE8A032B49008355890091
:10378000B74736FE938707C83E9BB387C5022A8496
:10379000B2898146B3B5C50213850732B337F50048
:1037A00013060064BE95EFA042776370AB0223A6B8
:1037B00044210145B250225492540259F249624ABE
:1037C000D24A424BB24B45618280829B835589002D
:1037D000AA8413060064B38735038146B3B5350365
:1037E00013850732B337F500BE95EFA00273B30718
:1037F0009500BE840327490063E4A70063E4E70063
:10380000B384E740D685228597D0FB1FE780C0B000
:1038100001C904C5B747024023A64721054559BF42
:10382000936504F0C205C181414597D0FB1FE78035
:10383000608111E9B737002083A7072285D7A285C9
:103840001145829705B7373700208327871E99EFE8
:103850002324A71E85472326050004C523115501EF
:1038600000A11CB12322050075B7BA87D84775FFA0
:10387000C8C7CDB779714ECEB747024006D622D41D
:1038800026D24AD052CC56CA5AC85EC662C466C254
:103890006AC083A9C72023A607200F10000025C1F6
:1038A00041443689B28A2E8AAA84B14C373B002023
:1038B000054D130C0003B30B94030327CB225E9733
:1038C0001C43B9EF9375F400B315BD001355444084
:1038D000C2055686C1811375F50FB93531C18327ED
:1038E000CB22DE9784C323A247016304090023008F
:1038F0008900B747024023A63721014521A023A60E
:1039000037210945B250225492540259F249624A71
:10391000D24A424BB24B224C924C024D45618280BE
:103920000504E31A84F9B747024023A6372121454D
:10393000D1BF011122CC26CA4AC84EC6B7470240A1
:1039400006CE03A9C7202A84AE89B28423A6072005
:103950000F100000D13B2285CE8597D0FB1FE7805A
:10396000A09B2A8405C5B737002083D5C72313063B
:1039700000648146B3879502B3B59502138507327B
:10398000B337F500BE95EFA0425948C01335140077
:10399000F2406244B747024023A62721D24442495D
:1039A000B2490E0505618280011122CC4AC84EC67B
:1039B000B747024006CE26CA83A9C7202A892E848B
:1039C00023A607200F10000097D0FB1FE780C094AC
:1039D000AA8419C123110500A2854A857D36B7370F
:1039E000002083C7C71963992701B737002003D781
:1039F000C71D598C239E871CB747024023A6372139
:103A0000014591E01945F2406244D2444249B2492D
:103A100005618280011126CA4AC8B744024006CE19
:103A200022CC4EC603A9C42023A604200F100000F8
:103A30009307F00263E6A704B1473304F502B739F0
:103A4000002083A7C922A2979C439DCB9377F500C2
:103A50008545B395F500C205C1811181B13783A7B2
:103A6000C9220145A29723A0070023A2070023A68D
:103A70002421F2406244D2444249B2490561828025
:103A8000B747024023A627210945E5B7411126C2C1
:103A900006C622C4B747024083A4C72023A6072036
:103AA0000F10000097D0FB1FE780008719E9014540
:103AB000B2402244B747024023A6972092444101D6
:103AC0008280B737002083A7071E00458297B7374B
:103AD0000020938747236367A402D843B74636FE86
:103AE000938606C83305A4403697E372E5FC1307B6
:103AF0000064B335E502922781463305E502EFA065
:103B0000C2417DB7D8433A94C9BF4111B7370020AD
:103B100006C623A8A7220295B240B737002023AAE1
:103B2000A71A014541018280914763E9B700B73781
:103B300000208A059387871CBE9588C18280B7378D
:103B4000002023A4071E37350020B737002041117D
:103B500023A807225146B737002081451305851C4D
:103B600006C623A0071E22C426C23734002097D0E1
:103B7000FB1FE780E0821305C4191306800281450C
:103B800097D0FB1FE780C081EFF0CFD7B737002079
:103B900083C717201304C419854513D527008D8BBF
:103BA0003E958D473305F5029947B7340020390516
:103BB0001375F50F28A03305F5021305052497C0EA
:103BC000FB1FE780204823A6A4222DCD3020994753
:103BD00081453306F6021306062497C0FB1FE780D3
:103BE000207C83A7C4223820B73400209387072481
:103BF0000A0723A2F41CBA97373700202322F71EA6
:103C0000EFF0AFE939291C3083A6441C3736040095
:103C10001397270036971306462A10C313871700F9
:103C20001377F70F0A073736040036971306663204
:103C300010C313873700890793F7F70F8A0718B067
:103C4000B69790C3B24022449244410182803737F4
:103C500000201307C7191C33342363FFD700B7367E
:103C6000002083A6461C1386170010B31397270065
:103C7000369708C33E8582809307F00FE5BF1C414D
:103C8000F1CF41777D8FB706002089476319D70CA4
:103C90005A2171C7411126C21946AA849305F00F13
:103CA000610506C622C497D0FB1FE78060810547E7
:103CB0008D47630FE5089C4491C7985C994749CBB1
:103CC000D85C59C73734002013060004814513051A
:103CD000C41E97C0FB1FE780A06C13060004A685D6
:103CE0001305C41E97C0FB1FE780E0649307C41E42
:103CF000DA2701E713070010DAA7F82719E30547C9
:103D0000F8A79A2B19E36D479AABF83719E31547D3
:103D1000F8B7B82B19E30547B8ABB83B19E3F83748
:103D2000B8BBD82B19E32547D8ABF82801E7130710
:103D3000C003F8ABDC5791C78297B73700202392B6
:103D4000A71AB73700207D57A38AE75ECD3B81478E
:103D5000B240224492443E854101828089473E859B
:103D6000828001114AC8373900208327492306CEB3
:103D700022CC26CA52C456C24EC68297130A006489
:103D8000B335450313094923835A89008146568672
:103D900033054503EFA06218B73700201387C71912
:103DA000004FAA840145630694029389C71933859D
:103DB0008440636E94000325490056868146B335DE
:103DC000AA023305AA02EFA04215018D269523AC65
:103DD0009900F2406244D2444249B249224A924A8E
:103DE00005618280011122CC2E84B7E506000A8588
:103DF00041469385053606CEEFA0424B18080604CF
:103E00003A94B7370020035504FF83D7E723F240E5
:103E10006244AA9737450F00130505243355F50270
:103E200005618280B737002083D7E72351471D45BE
:103E3000637CF702794719456378F702130720037B
:103E400015456373F7021307B0041145637EF7004D
:103E5000130740060D456379F7001307600909450C
:103E60006374F70013B5B70F8280011122CC06CE20
:103E70002A842EC6EFF04FD3B245F240818D33A590
:103E8000A502229562441375F50F05618280011128
:103E900022CC06CE2A842EC6EFF00FD1B245F240D6
:103EA000818D33A5A50222956244420541810561B9
:103EB0008280011122CC06CE2A842EC6EFF0CFCE0E
:103EC000B245F240818D33B5A50222956244056169
:103ED0008280B737002023A2A7248280B737002032
:103EE0001387C71E585739CF411122C426C24AC072
:103EF00006C61389C71E0297B73700201387C71954
:103F00001A272A849384C71905CBBA876373A7003D
:103F1000AA87C207C183BA866373E400A286C20679
:103F2000C182958F51476359F7008327090391C3D5
:103F30008297EF00E22782A4B240224492440249D1
:103F4000410182808280011122CC37340020930706
:103F5000C41E9C5B06CEAA851304C41E81C72AC654
:103F60008297B245C9C19C410545B5CBDC41A5CB83
:103F70009E25B5C7BE25A5C7DC2589CB5C3813F7C0
:103F800037008983BA970947634BF7043735002018
:103F900041461305452397C0FB1FE780C039B7375B
:103FA000002083A64723373700202320D71E7838E8
:103FB0000DE3938747238A279307805737460F00DF
:103FC0003305F5021306062481468145EF90F2740D
:103FD00068B837450400130525D6053E0145F24073
:103FE000624405618280B73700209387C71937176D
:103FF000002023AE070013076798B737002023AAD5
:10400000E7223787320093874723FD56130727A1FE
:10401000D4C398C723860700B747024023A4D726F6
:10402000BDBF011122CC373400209307C41E88473E
:1040300006CE26CA4AC801E90545F2406244D24488
:104040004249056182801304C41E1C5CF5D7585C8C
:1040500065D77000854582971844B247E30EF7FC98
:104060004A249305E004B734002097C0FB1FE78083
:1040700060FD1387C41908D39384C41955DD5224F5
:104080009305F00F014997C0FB1FE78060317C2446
:104090009050634DF900328597C0FB1FE780800781
:1040A000014523A0040223A2040241BF4E24084478
:1040B000585CB3872503898105093E9508C202979C
:1040C000F9B701114EC6B73900209387C91E9C4726
:1040D00026CA4AC852C406CE22CC56C25AC02A8A20
:1040E000AE8432896388071E9389C91E03A789039A
:1040F000630207121307F01F6360A7123734002012
:104100001307C419832A07021304C41963980A0801
:1041100003D5C9009565938515E097C0FB1FE7801F
:1041200060F208D02A867DC583D5C90083A789039C
:1041300003A589008981829783A78900832A0402C5
:104140005CD089476314FA08C1476395F40C83D5A2
:10415000C9009147938505FCB3C5F5028A05D6953C
:10416000B8219307A0056313F70A9E216390470BBC
:104170004A852686910597C0FB1FE780C01B1C500F
:104180005685639157130145F2406244D244424937
:10419000B249224A924A024B056182805850E3821A
:1041A000E7FA03D5C9009565938525E097C0FB1F05
:1041B000E78040E9AA8A39CD83D5C9002A8683A73A
:1041C000890303A5890089818297A5BF8D47631B59
:1041D000FA00C1476390F40483D5C900938545FD77
:1041E000F199B5BF91476318FA006395440383D5ED
:1041F000C900A115F5B793070010631DFA00A14788
:1042000063EA970083D5C900C115D9BF1C505685F4
:10421000639D570B29458DBF9D6A637A5509930AA3
:1042200005E01947B3CAEA0203D7C900373B0020AB
:10423000B38AEA02BE9A9307CB19DC53130BCB194E
:104240006395570103240B021DE003D5C9009305B4
:10425000E00497C0FB1FE780E0DE2A8445DD83D5BC
:10426000C90083A789032A8689815685829791454B
:104270001307A005898193972500A297B423639122
:10428000E6049623639C460385058A052686A29547
:104290004A8597C0FB1FE780000A83270B02E3844F
:1042A00087EE228597C0FB1FE780C0E6E9BD216746
:1042B0007917E361A7F6B30A5541BDB7AC335DBFCB
:1042C00083270B02E38887F4228597C0FB1FE780D2
:1042D00060E489B7B737002083A5C71B85DD914708
:1042E0009306A0058983139727002E973023E313A5
:1042F000D6F21223631C460185078A072686BE95DF
:104300004A8597C0FB1FE7800003B5BD3C33D9BF8A
:10431000B73700209387C71E984721C3D85F15CFB2
:104320008546631CD502411122C437340020130492
:10433000C419105006C611CECE2748508981029765
:10434000085097C0FB1FE780E0DC232004022322F3
:104350000402B2402244410182808280011122CCB9
:10436000373400209307C41E56C283AA870026CA8A
:104370004AC84EC606CE52C42A89AE84B2891304F6
:10438000C41E638D0A1A5C5C99EB2945F2406244B5
:10439000D2444249B249224A924A056182801C5C59
:1043A000EDD79307F01F63E1A70C373A002093077E
:1043B000CA199C53130ACA19A9C7084483274A0279
:1043C000639CA70489476313F906C147E39FF4FA86
:1043D0004A249147130505FC3345F5029317250040
:1043E00003250A022686CE853E959307A0053CA1AB
:1043F00023102501110597C0FB1FE780C0F301457D
:1044000071B74A249305E00497C0FB1FE78080C37F
:104410002320AA025DF195BF4E241C5C03260A02EC
:10442000898182971C442322FA0269BF8D47631B4E
:10443000F900C147E39BF4F44A24130545FD937743
:10444000C5FF79BF91476317F900E39024F54A242B
:104450002115F5B793070010E319F9F2A147E3E638
:1044600097F24A244115E1BF9D676375F5069307EE
:1044700005E01947B3C7E7025A24373A0020B3874B
:10448000E702BE9A9307CA199C53130ACA19B1CB03
:1044900083274A026392570703250A0291461308AD
:1044A000A0059305F00F93D72600139727002A97AE
:1044B00030236312060783580700303363992805B9
:1044C000B306D64063C4960485078A072686CE8540
:1044D0003E9515B721677917E369A7EAB307F54059
:1044E00061BF4A249305E00497C0FB1FE78080B5B5
:1044F0002320AA0251FD51BD4E241C5C03260A0252
:1045000089815685829723225A0379B70EA3931681
:104510000601C18249BF5224B38596009105130656
:1045200006FCE3F4C5E613863400719A1106B296D0
:10453000230107012310270134B379B7373A00204C
:104540009307CA199C53130ACA1995CF03250A0267
:1045500091461308A0059305F00F93D726001397F3
:1045600027002A973023631006058358070030334D
:1045700063972801B306D640E3D896F40EA39316AA
:104580000601C182D9BF68245E249305E004330587
:10459000F5024205418197C0FB1FE780A0AA2320B6
:1045A000AA024DF5DDB352246C24B385C5023386CF
:1045B00096001106E3EBC5DCBDB7014582809C2166
:1045C0001CA1BE211CB1BE21A1833CA1DC213CB1B8
:1045D00011458280B737002023A207F0B7370020AB
:1045E00023A007F082800DCD411126C206C622C449
:1045F000AA8401458DC12E84B7E506002285414677
:104600009385053797C0FB1FE780E0D29C200545C6
:104610005CA49C305CB4B24022449244410182804C
:1046200001458280011122CC26CA06CE0947AA8400
:1046300032846381E50441468147639BC500638FF3
:10464000E6006397B6000DA841478147638EE600F8
:10465000F2406244D2443E85056182808A8522858B
:10466000593741468A8519A88A85B53F41468A85CA
:10467000228531A0E39AB6FC2E86A285268597C0B6
:10468000FB1FE78040DCAA87E1B7B737002023A0F3
:10469000A7F08280B737002023A2A7F08280011103
:1046A00022CC622106CE26CA4AC84EC62DCC83290A
:1046B0008500AE842A8803C9090081471317890140
:1046C000618763550702B147054563F787045114B5
:1046D000420403552800418033878900A2864E8614
:1046E0008545EFB0F027B337A00085077D1413553B
:1046F0006900420405891379F90341809CA088B0C0
:1047000023812401C2A0014719C01387190098C44E
:1047100009476383E7000145F2406244D2444249BD
:10472000B249056182800545C5BFC167F917630AB3
:10473000F502D94763F7B702011122CC2EC606CE87
:104740002A84EF906021B2456368B50022856244F7
:10475000F24005616FA01015F24062440545056105
:10476000828005458280C167F9176314F5006F9058
:10477000A01E411106C6EFA0700111E15D45B240D7
:10478000410182809147639DF5001C211CA23C21C0
:104790001831A207D98F3EA23C3101455CA282802C
:1047A000114582804111814522C426C206C6AA84D1
:1047B000BD232A8409E9B737002083A707F081C702
:1047C000F945268582972285B240224492444101D0
:1047D000828039714ED656D25AD006DE22DC26DAD5
:1047E0004AD852D4AA8A2E8BB28951EB36C6A53F3D
:1047F0009145EF900025AA844D493DC5B246054A32
:10480000238034010544630A0B00B6851385140028
:10481000029B0505131405014180E20993D98941E2
:1048200063D30902C1455685EFA0B004654915E57B
:1048300033868400A2852685EFB0A0582A8911ED21
:1048400031044204418091472C085685FC8426CED1
:10485000E085EFA0601B2A8901C963070A0026854D
:1048600097C0FB1FE780008BF25062544A85D254F8
:104870004259B259225A925A025B21618280BA840B
:10488000014ABDBF011122CC26CA4AC84EC606CE77
:104890002A893284B689353FAA840DE1B7370020D2
:1048A00083A747F081CF05476317E40003C40900DD
:1048B00005041374F40FA2854A858297F24062447E
:1048C00026854249D244B24905618280AE86B74509
:1048D0000400014705469385E55B6DB79E211CA149
:1048E0009E21A1831CB1094582809E211CA19E218D
:1048F000A1831CB1BE213CA1BE21A1833CB11145C5
:1049000082809E211CA19E21A1831CB1BE213CA1BD
:10491000BE21A1833CB1DC315CA1FC215CB18A25C4
:1049200019054205418182809E211CA19E21A183FF
:104930001CB1094582809E211CA19E21A1831CB12E
:10494000BE213CA1BE21A1833CB111458280CA2178
:1049500006054205418182809E211CA19E21A183E2
:104960001CB1AA2109054205418182809E211CA11A
:104970009E21A1831CB1BE213CA1BE21A1833CB1DB
:10498000CA2111054205418182809C211CA1054557
:1049900082809E21411122C406C61CA19E212E8424
:1049A0001105A183A30EF5FEBE219505230FF5FE8B
:1049B00083D7D5FFA183A30FF5FE03C6F5FF97C0EC
:1049C000FB1FE78040974820B24022441105410177
:1049D000828089476399F5001C3118210145A2079F
:1049E000D98F1EA28280114582809A21D94763FD0A
:1049F000E702011122CC06CE2EC62A84EF80D075A4
:104A0000B2469E22636DF50022856244F240B7559E
:104A10000400014709469385C58D05615DBBF240E1
:104A2000624409450561828009458280914785C5B8
:104A30001421FD15C2058547C1816390F60213D785
:104A400025008D89914781E9914711C7050534A259
:104A50001AA248C281473E85828009479147E39C5C
:104A6000E6FEC94733D7F502B3F5F502E1BFAE86DE
:104A7000B7550400014711469385A58E99BB93F75E
:104A8000350089EB8981914781C50EA248C28147D3
:104A90003E8582809147EDBFD8218947631CF7028C
:104AA000011122CC2A84C84506CEAE86014709C929
:104AB0002EC69D4597B0FB1FE7800073B2462A873C
:104AC00022856244F240B75504001946938525902B
:104AD000056101B30945828099E1114582801C215D
:104AE00005473EA2E37BF7FEFD1593F5F50F33D79F
:104AF000F502B387E702E392F5FE050548C21AA264
:104B000001458280DC210947AE866385E700414785
:104B10006399E700B755040001472146938525991D
:104B20004DB9094582800EA291E1014548C2014577
:104B30008280AE86B7550400014729469385859249
:104B400049B90EA291E1014548C201458280AE8675
:104B5000B755040001473146938565939DB90EA270
:104B600091E1014548C201458280DA21854763FF12
:104B7000E702011122CC2A84884106CE1DC12EC62F
:104B8000854597B0FB1FE78020662A87228562440F
:104B9000B246F240B755040039469385E594056165
:104BA0000DB9F24062440945056182800945828061
:104BB000914785C518218D46914763F0E602FD15A2
:104BC000C205C181B3C6E5023308D7026397050168
:104BD000050516A23AA248C281473E858280DC21A3
:104BE0000947AE866385E70041476399E700B755FB
:104BF00004000147414693852599E1BE094582801D
:104C0000B335B000139525008280011122CC26CA4D
:104C100006CE98258547AA842E844946631FF7004F
:104C200099363E2049151306200963C8A700F240B3
:104C30006244D24409450561828018348547631473
:104C4000F70013660604484001C98D4532C697B087
:104C5000FB1FE78060593246A2866244F2402A87F1
:104C60002685D244B755040093858595056195B690
:104C70008D4763F8B7021C311821F115A207D98FAF
:104C80001EA23C313821C205A207C181D98F3EA2A4
:104C90004EA289C5110508C601458280232406005D
:104CA000E5BF11458280011122CC2A84884506CEB9
:104CB000AE8601C92EC6954597B0FB1FE780C0524E
:104CC000B2462A8722856244F240B755040059460D
:104CD0009385C5960561F5BCB335B00013952500E5
:104CE0008280AE86B7550400014761469385A5983A
:104CF000CDB48547114563F0D7021C320C22A207C0
:104D0000CD8F1EA39387E6FF3EA389476386F600F7
:104D1000090650C30145828023220700E5BF0147F1
:104D200081467946814575B49E211CA19E21A183AF
:104D30001CB109458280BC2105471CA18A216397CB
:104D4000E7000A050505420541818280C947330510
:104D5000F502CDBF8A210A05420541818280BE212C
:104D60001CA18A21BE213305F502050542054181BA
:104D700082808A2182808A2182808A218280BE214B
:104D80001CA18A21BE213305F5020505420541819A
:104D900082809E211CA19E21A1831CB1BE213CA129
:104DA000BE21A1833CB1CA21110542054181828007
:104DB0009E211CA19E21A1831CB1AA2109054205A7
:104DC00041818280894711456398F6001C32142284
:104DD0000145A207D58F1EA382809A21D947AE86AE
:104DE00063F9E700B755040001470D46938585D266
:104DF00051BC094582801145639DA6001C321422D6
:104E00000145A207D58F1EA33C323422A207D58FBD
:104E10003EA38280BC210547FD1793F7F70F63611E
:104E2000F7049E2195CF011122CC2A84C84106CED9
:104E30001DC12EC6894597B0FB1FE780E03A2A873F
:104E400022856244B246F240B75504001546938568
:104E500065D3056105BCF240624409450561828065
:104E6000094582809547114563F1D706411122C457
:104E700026C24AC006C61C32BA841822A20732844F
:104E8000D98F9EA03C32382293054400A207D98FC7
:104E9000BEA08947DCA0094613855400368997B027
:104EA000FB1FE78040499307A9FF9EA49947631B16
:104EB000F90023A60400B24022449244024901456D
:104EC000410182801904C0C4FDB782809E2195CF24
:104ED000011122CC2A84C84106CE1DC12EC68545AB
:104EE00097B0FB1FE78040302A8722856244B24694
:104EF000F240B75504001D46938545D5056159B26A
:104F0000F2406244094505618280094582809947E3
:104F1000639DF6028947411106C65CA31C32142228
:104F2000B285A207D58F1EA33C3234225023A2079C
:104F3000D58F130557003EA3910597B0FB1FE7805F
:104F4000803FB240014541018280D14711456394C1
:104F5000F600C147C9B782809E219DCF011122CCA6
:104F60002A84C84106CE05C52EC6894597B0FB1FC9
:104F7000E78080272A8722856244B246F240B755EF
:104F8000040025469385E5D505616FF0BF8FF2409B
:104F9000624409450561828009458280894711453F
:104FA0006398F6001C3214220145A207D58F1EA378
:104FB0008280011122CC2A84C84106CEAE860147E8
:104FC00009C92EC6854597B0FB1FE780E021B24690
:104FD0002A8722856244F240B75504002D46938506
:104FE00025D705616FF01F8A1145639DA6001C320D
:104FF00014220145A207D58F1EA33C323422A207FA
:10500000D58F3EA38280011122CC2A84C84106CECE
:10501000AE8601C92EC6854597B0FB1FE780C01C30
:10502000B2462A8722856244F240B75504003546CD
:10503000938565D705616FF0FF8493F716001145DE
:1050400081EB89476386F600858256A310C301452C
:105050008280011122CC2A84C84106CE05C52EC605
:10506000854597B0FB1FE78020182A872285624478
:10507000B246F240B75504003D469385A5D7056179
:105080006FF05F80F24062440945056182809E2195
:105090009DCF011122CC2A84C84106CE05C52EC65B
:1050A000894597B0FB1FE78020142A872285624438
:1050B000B246F240B755040045469385E5D70561F1
:1050C0006FF04FFCF240624409450561828009455A
:1050D0008280854763F6D70208A70CB71C320C22E2
:1050E000A207CD8F1EA39387E6FF3EA38947638661
:1050F000F600090650C30145828023220700E5BF60
:1051000011458280014781464D4681456FF08FF7FA
:105110008D47114563F4D7021C320C22A207CD8FB4
:105120001EA33C322C22A207CD8F3EA39387C6FF3D
:105130005EA36386A600110610C701458280232462
:105140000700E5BF011122CC2A84884506CEAE8631
:1051500001C92EC6954597B0FB1FE780E008B2460F
:105160002A8722856244F240B75504005D46938544
:1051700025D905616FF00FF1854711456395F6005C
:105180001C2201451CA3828001478146654681455A
:105190006FF04FEF011122CC2A84C84106CEAE86B3
:1051A000014709C92EC68D4597B0FB1FE780C00394
:1051B000B2462A8722856244F240B75504006D4604
:1051C000938505DB05616FF0CFE0011122CC2A84C5
:1051D000C84106CEAE86014709C92EC68D4597B097
:1051E000FB1FE7806000B2462A8722856244F240B6
:1051F000B75504007546938505DB05616FF06FDDDB
:10520000011106CE2EC6EF90905419C5B245F2405A
:105210002A2105616FE06013F240494505618280F3
:10522000B7370020A38807F2B7370020238807F29A
:10523000B737002023AC07F0B737002023AE07F0C4
:10524000B737002023A007F2B737002023A207F2C8
:10525000B737002023AA07F0B737002023A807F0AC
:10526000B737002023940726930640389387872674
:10527000B6B3F1761307400B938606B8BAA3D6B33C
:1052800011679D46130600059305000A1305007D6E
:10529000DAA3F6B341478546130810F8BAA7DAA790
:1052A000BAABDAABFAAB9AAF9AB723960703EEA381
:1052B0008EA7F2A792ABAAAF239E0700239F0700F9
:1052C00023900702B6B7239707021308F007239825
:1052D00007022392E7042393E704239FE704239024
:1052E000E7062391E7062392E706239907031307AE
:1052F000C01CD6BBF6BB239C0702239D0702239E3E
:105300000702239F0702239007042391D7042394C5
:105310000704239507042396D7042397C7042398EB
:10532000C7042399A704239A0704239B0704239CFB
:105330000704239DC704239EC7042393A706239431
:10534000070623950706239607062397B706239893
:10535000B70623990706239AE7065147239DE706D8
:105360007D57239B0706239C0706239ED706239F72
:10537000070623900708239107082392E7088280F5
:10538000011126CAAA84214522CC06CE2E8432C61B
:1053900036C43AC297B0FB1FE78020EA0DC5A2468B
:1053A00012473246930700FD1CA1994704B13CA166
:1053B00074A178B152A1AA8522856244F240D244F8
:1053C00005616FD07FE4F2406244D244056182807F
:1053D000B737002023ACA7F08280B737002023AE78
:1053E000A7F08280B737002023A0A7F28280B737CA
:1053F000002023A2A7F28280011122CC4AC806CE47
:1054000026CA2A890144B30489006368B400F240C3
:105410006244D2444249056182802EC6EFD0DFF853
:1054200093170501C183A183B2459CA09307140083
:1054300093F7F70F850463F8B700CA97090488A3A8
:105440001374F40FC9B73E84C9B7411122C437346D
:105450000020130484246A20C16706C6FD17630E6A
:10546000F500B737002003C6C73AB735002093854B
:1054700085F2EF90F00FFD577EA0B240224441012B
:10548000828009C925151375F50F1335850E13454F
:10549000150082800145828023900500C1C6797184
:1054A00022D426D24ECE52CC5AC806D64AD056CA9C
:1054B0005EC63684328AAE892A8B814463F2440701
:1054C000B30794009C23138914004209939A07019F
:1054D00093DA0A011359090163840A04CA976341E4
:1054E000FA04B307240183CB07005E85593F0DC939
:1054F0009387FAFF2390F90063906B03130519005B
:105500002295B250225492540259F249624AD24A28
:10551000424BB24B45618280D694C204C18079BFB0
:105520000145C5B701458280011122CC37340020E6
:1055300026CA4AC84EC69307842406CE2E89D0CBED
:105540008CCBC8C7AA8441469305F00F4A8597B013
:10555000FB1FE780E0F685491304842463193503B3
:105560000848C145513D41469305F00F268597B047
:10557000FB1FE780E0F405496315250348446244B6
:10558000F240D2444249B249C1450561B5B54146F0
:1055900081454A8597B0FB1FE78080F2E31535FD12
:1055A000C1B741468145268597B0FB1FE78040F192
:1055B000E30625FDF2406244D2444249B249056106
:1055C0008280411122C43734002026C24AC0AE84F2
:1055D0002A891306000281451305842406C697B064
:1055E000FB1FE780E0DB93078424A3812701B73703
:1055F00000202388973AEFD09057854719C18147FB
:1056000049452304F424B240224492440249410112
:105610008280814791C909C985476319F500DC314A
:1056200093E707FCDCB185473E8582808947631696
:10563000F500DC3193F7F703F5B70D478547E31520
:10564000E5FED8311377F70313670704D8B1E9BF34
:10565000814785C119CDD8319306000C8547137752
:10566000070C6308D700930600048D476303D70037
:1056700089473E858280411122C4005D06C626C24C
:105680001DC8AA84085009C597B0FB1FE78080A8F1
:10569000485009C597B0FB1FE780C0A7085409C54B
:1056A00097B0FB1FE78000A7228597B0FB1FE7801C
:1056B00060A623AC0402B24022449244410182809D
:1056C00019E9B737002083C7A72491C737350020D1
:1056D000130585F08280373500201305052682806A
:1056E000B737002003C5A7248280B737002003A561
:1056F00047258280B737002003A587258280B737EA
:10570000002083A7C72588438280B737002093876E
:105710008724D44B9842050798C2A8339307F00F0B
:105720006305F50091656FD05FE28280011122CCA4
:1057300006CE2E8432C6EF9030129147B2456310E8
:10574000F502B737002083A747F295C303A30700EC
:10575000630F030022856244F24005610283B7377C
:10576000002083A7C7F181C703A34700D5B7F24044
:105770006244054505618280011122CC2A844A21B8
:1057800006CE26CA4AC84EC697B0FB1FE780C03077
:105790002DC52A8904218349C500F13D4A85EF9032
:1057A000F0494A20EF90900637390020130909F399
:1057B00083470900B9C763969704B737002083C5AC
:1057C00017F32685353C19E1230009004A20EF90A4
:1057D000B0089147631CF500B737002093878724F2
:1057E0005620FA236394E6007D57FAA3F240624400
:1057F000D2444249B2490561828081499304F00F45
:1058000065B79307F00FE383F4FC7420522028203F
:105810004E87A685B5365DBF79715EC6AA8B2E858B
:1058200052CC56CA5AC806D622D426D24AD04ECE18
:10583000AE8A328B368A97B0FB1FE780E0257DC1A8
:10584000045D2A89E5C09C50614599C31305400356
:105850009C5481C751054205418163050A007105C9
:1058600042054181DC5081C75D054205418197B009
:10587000FB1FE780809C2A8455C56146814597B00F
:10588000FB1FE780E0B1B737002083C98729639405
:10589000090083490900930700FD1CA0A947A30044
:1058A00074013CA0230364018C502312540113059E
:1058B000840191C908C47146930A440397B0FB1F41
:1058C000E78060A756858C5491C948C45146930A15
:1058D000450197B0FB1FE78000A65685630C0A00C0
:1058E00008C87146D285930AC50197B0FB1FE780AF
:1058F00080A45685CC5099C548C85D4697B0FB1F1B
:10590000E78060A3A2854E85EFD01F902254B2504D
:105910009254F249624AD24A424BB24B4A850259EA
:10592000456191BBB250225492540259F249624AE5
:10593000D24A424BB24B4561828001114EC6AA89C0
:105940002E854AC806CE22CC26CA2E8997B0FB1FC8
:10595000E780801439C5B737002083C4872991E0D8
:105960000421194597B0FB1FE780208D2A8415C9B3
:105970008145194697B0FB1FE78080A2930700FD81
:105980001CA0B947A30034013CA023122401A28526
:105990006244F2404249B2492685D24405616FD043
:1059A000BF86F2406244D2444249B24905618280D6
:1059B00039715ECEAA8B2E8526DA4ED652D456D2B7
:1059C0005AD006DE22DC4AD8AE84328BB68A3A8AB6
:1059D000BE8942C697B0FB1FE780000C39C92A89EF
:1059E000414597B0FB1FE78040852A8439C1414675
:1059F000814597B0FB1FE780A09AB737002003C509
:105A0000872919E103450900930700FD1CA0BD4744
:105A10003CA0B247A300740146A023046401A30480
:105A2000540123054401A30534015CC4A285EFD0D1
:105A3000AFFDF2506254D2544259B259225A925A8E
:105A4000025BF24B21618280797126D2AA843945AA
:105A50004AD04ECE06D622D42EC6B289368997A019
:105A6000FB1FE780807D0DCDB2459307000D1EA181
:105A7000B1472A844EA13CA1CE851905194697B09D
:105A8000FB1FE780408B23062401A2852254B250DD
:105A90000259F24913F5F40F925445616FD0CFF6D5
:105AA000B250225492540259F24945618280411108
:105AB00026C2B734002093848424B83006C622C49A
:105AC0004AC09307F00F6308F7042A89394597A065
:105AD000FB1FE78080762A841DCD930700FDB73534
:105AE00000201CA1A30025012301050093850526A4
:105AF0000D05194697B0FB1FE780E0839E24A28521
:105B0000A8303EA49C305CA42244B2409244024996
:105B100041016FD06FEFB2402244924402494101EB
:105B2000828001115AC02A8B314526CA4EC652C402
:105B300056C206CE22CC4AC8AE84B28A368ABA8908
:105B400097A0FB1FE780606F2DCD2A84268597B034
:105B5000FB1FE78060F409C55825A1476311F704CE
:105B6000B737002003C9B724930700FD1CA09D4749
:105B7000A30064013CA046A0231354012314440154
:105B800023153401A2856244F240D244B249224A2C
:105B9000924A024B4A85424905616FD0EFE6B7371A
:105BA000002003C9173BE3110BFCB737002083A784
:105BB00007FF9C47D5DBCE865286D6852685829701
:105BC00065B7F2406244D2444249B249224A924AFD
:105BD000024B05618280011122CC2A84214506CE28
:105BE0002EC697A0FB1FE780406515C5B2459307F9
:105BF00000FD1CA1C5473CA1BC313CB1DE215EA12A
:105C0000FC217CA1FC31AA857CB122856244F24052
:105C100005616FD06FDFF2406244056182804111FF
:105C20004AC02A89714526C206C622C4AE8497A0FE
:105C3000FB1FE78080603DC5930700FD1CA1F54771
:105C40003CA1BC302A849385C4003CB1DE203105E0
:105C50001946231CF5FEFE20231DF5FE9E24231E5F
:105C6000F5FEBC24230FF5FEBC34A30FF5FE97A070
:105C7000FB1FE780406CBC28A2854A853CA8DE2833
:105C80005EA8FC287CA8FC387CB89C2C1CAC9C3CF6
:105C90001CBCBC2C3CAC2244B240924402494101A1
:105CA0006FD08FD6B2402244924402494101828093
:105CB00001114AC82A89614526CA4EC606CE22CCA1
:105CC000AE89B28497A0FB1FE780205725C19307B8
:105CD00000FD1CA1BC302A84938584001CB195472B
:105CE0003CA1FC3011051946A30FF5FE97A0FB1F40
:105CF000E7806064DE2023063401A2853EA4BE2C2A
:105D00004A857EA4DE2C1EA8FE2C3EA883C7040272
:105D10005CA883C714025CB8BE30F240D2447EA8AF
:105D200062444249B24905616FD00FCEF2406244ED
:105D3000D2444249B24905618280411122C43734BC
:105D40000020130484243C2006C626C285CBB73429
:105D50000020AA851946138584F097A0FB1FE780D1
:105D6000805D2820938584F0EFF0BF8A2244B24002
:105D7000138584F0924441016FD02060B2402244E8
:105D80009244014541018280411126C2B73400206E
:105D90009387842406C622C44AC0B8339307F00F01
:105DA000938484246301F7042A89294597A0FB1F63
:105DB000E780A0482A8405C9930700FD1CA1A147DC
:105DC000A30025013CA1BC20B7350020938585F0B8
:105DD0003CB11946110597A0FB1FE780C055A830BC
:105DE000A285EFD06FC2B8208D476311F702B73795
:105DF000002083A707F299CB03A387006308030061
:105E00002244B2409244024941010283B2402244FA
:105E10009244024941018280797122D406D626D269
:105E20004AD04ECE52CC56CA09444DCD2A890A21B9
:105E3000AE89514497B0FB1FE78000C6AA845DC1BC
:105E4000373700209307C73ADC238546BA8AFD1707
:105E500093F7F70F494463F7F6085825A1476314F1
:105E6000F700639109089C5C4544ADEF916593850B
:105E700045711305C00297A0FB1FE780A01C88DCBA
:105E80002A8A4D4425C11306C002814597A0FB1FF5
:105E9000E78000518357090093064A003685231195
:105EA000FA0071469305490036C697A0FB1FE780AC
:105EB000804889472300FA00C824B24603560900E7
:105EC00083C5CA3A611513351500EFA0001D2A8459
:105ED00063860900CE852685EF90300401C42685AF
:105EE000EFF06FF92285B250225492540259F249D0
:105EF000624AD24A45618280B737002083C7073B98
:105F00000547FD1793F7F70F6377F708894749C6E9
:105F1000011122CC26CA4AC84EC652C406CEAA894E
:105F2000368AB2842E8997B0FB1FE780E0B62A84B8
:105F3000D14731C5485509C597A0FB1FE780801D93
:105F4000F145268597A0FB1FE780204B48D4CD471D
:105F50001DC5542421478147639DE600630B0A0059
:105F6000382D122993062501AA854E85EF90500100
:105F7000AA875820630E09001367670058A0F240F3
:105F80006244D2444249B249224A3E850561828038
:105F900013674700E5B7C9473E8582809307100421
:105FA00063EAA700B73700209387872606053E954A
:105FB0000A21828041657D158280011122CC2A84CC
:105FC0002E8526CA06CEAE8497B0FB1FE780C0ACF4
:105FD0000DCDB7470F009387F723094563E287028A
:105FE00081450A85414697A0FB1FE780603BA68557
:105FF00060800A8541804081A3010100EF90D06A52
:10600000F2406244D244056182804945D5BFB7372A
:1060100000202387A73A82806FA08002797152CC3A
:106020002A8A328522D426D24AD04ECE56CA5AC89F
:106030005EC606D662C4AE8BB28A368BBA843E89FF
:10604000C289468497B0FB1FE78000A50DC92A8C42
:1060500063130A0213774B005C2115CF93E72701E6
:106060002302FC008DEC631C0902639A090205E817
:10607000ED9B2302FC00832B8C0363910B08B25031
:10608000225492540259F249624AD24A424BB24BCC
:10609000224C45618280F59B93E70701D1B793E7D6
:1060A00047002302FC0001CC1C484146A285232462
:1060B000FC0213058C0197A0FB1FE780C0276393A8
:1060C0000B02D5D80325CC0209C597A0FB1FE7809A
:1060D0006004F145268597A0FB1FE7800032232648
:1060E000AC0251BFE30909F80325CC0209C597A00A
:1060F000FB1FE7802002F1454A85F1BF9DC483A7BD
:106100000B0299EB916593853571714597A0FB1F43
:10611000E78040F323A0AB0203A50B0219C571462B
:10612000A68597A0FB1FE78000216388090283A74B
:106130004B0299EB9165938525715D4597A0FB1FF7
:10614000E78040F023A2AB0203A54B0219C55D46D0
:10615000CE8597A0FB1FE780001E1DC483A78B027E
:1061600099EB916593851571514597A0FB1FE780C9
:1061700060ED23A4AB0203A58B0219C55146A2858D
:1061800097A0FB1FE780201B2254B2509254F24983
:10619000B24B224CCA865A860259424BD68552854A
:1061A000D24A624A45616FF02FE7011126CA52C4F4
:1061B00006CE22CC4AC84EC62A8AAE8497B0FB1FB0
:1061C000E780808D35C1AA89394597A0FB1FE780FC
:1061D000C0062A8431C9B737002003C98729631450
:1061E000090003C909009307000D1EA0AD473CA09C
:1061F0009385690013053400194697A0FB1FE780BB
:10620000801393F71400858085885CA444B423151B
:106210004401A2856244F240D244B249224A4A85EE
:10622000424905616FC05FFEF2406244D244424978
:10623000B249224A0561828001114EC652C456C23B
:1062400006CE22CC26CA4AC8AA8A2E8AB28997B01C
:10625000FB1FE78060842DCD2A891305C00297A01B
:10626000FB1FE78080FD2A8425C5B737002083C443
:10627000872999E0834409009307000D1EA0E94790
:106280003CA09305690013053400194697A0FB1F35
:10629000E780600AD285231554011305C4004146E6
:1062A00097A0FB1FE7802009CE851305C401414656
:1062B00097A0FB1FE7802008A2856244F240424974
:1062C000B249224A924A2685D24405616FC0DFF363
:1062D000F2406244D2444249B249224A924A05619C
:1062E0008280411122C437340020130404F1084095
:1062F00006C619C597A0FB1FE780C0E12320040054
:10630000B240224441018280011106CE22CC26CA2D
:106310004AC82EC697A0FB1FE780007831CDB24552
:10632000B737002003C987290CD5AA846314090054
:1063300003490500414597A0FB1FE78000F02A8430
:1063400005CD9307000D1EA1A5473CA1DC30938528
:1063500064001105A30FF5FE194697A0FB1FE78007
:1063600080FD9C54A285F2405CC46244D2444A85BC
:10637000424905616FC05FE9F2406244D24442493C
:10638000056182801D71A2CC86CE2A842EC697A07C
:10639000FB1FE780607015C954251147AA8749453E
:1063A0006391E6029C5FB24591C3EC2BB7160500E2
:1063B0002308B1009386E6F4100889452285EF9002
:1063C000E02CF6406644256182805145DDBFB73739
:1063D000002083C7073B0547FD1793F7F70F637A44
:1063E000F704894721CA411122C426C24AC006C601
:1063F000B2842E8997A0FB1FE780006A2A84D147C8
:1064000015C1630609005C2193E727005CA14146A2
:10641000A6851305840197A0FB1FE780C0F19C4867
:106420001CD48147B2402244924402493E85410136
:106430008280C9473E858280797122D406D62A841B
:106440002EC697A0FB1FE780206501CDB2452285AF
:10645000230EB1006C08EF90E028B2502254456141
:1064600082805145DDBF6F801034C1671387E7FF1D
:106470006395E502B737002083A7C7F191EB494543
:1064800082804945B24022449244024941018280BF
:1064900003A30700E30503FE0283411122C426C2C1
:1064A0004AC006C6FD172A892E84B284639AF50273
:1064B000B737002083A7C7F191CF9C4381CF829744
:1064C00011E9B7370020238827F3B7370020A388C6
:1064D00097F24DBFA6854A85EFE09FD245F5D5B727
:1064E0002E8597A0FB1FE780205B41DD1C210D4519
:1064F000E39A27F922852244B2400249A6859244B4
:1065000041016FC090649307100463E1A706411135
:10651000C16722C406C626C2FD172A8409456381C5
:10652000F502C547AE846312F4022E85EFC0706990
:10653000373500201305852606042A9406A0014558
:10654000B24022449244410182809307A003631623
:10655000F4002E85EFC03060E1BF9307B003E3196C
:10656000F4FC13F5F50FEFC0505FD9B709458280F1
:10657000011106CE2AC6EFE0BFCAEF20C06DEF10B2
:10658000F012EF700210B7370020938787241307AB
:1065900000F0BAA323820700B737002032451387E3
:1065A000C73AFD5634A3F2402386A73A95450561C4
:1065B0006F70C0437571939705014AC106C722C524
:1065C00026C3CEDED2DCD6DADAD8DED6E2D4E6D204
:1065D000EAD0EECEC1872E8963D30754B7340020AA
:1065E00003C5C43AB7390020373B002097A0FB1FF2
:1065F000E78000CA2A8426CCB73A0020B73B0020A7
:10660000373D002093848924B73C00201DE021659C
:106610003345A900BA402A449A440A49F659665AB1
:10662000D65A465BB65B265C965C065DF64D4961C4
:1066300082801C201307200A639BE70003CA3400F2
:106640002A20C1652286FD15EFF04F8EA1AA624770
:106650001307C73A034A270013071009639FE7147B
:106660001C3015476391E7022285EFF0EF902285F9
:10667000EFC0BFB4E24703C5C73A97A0FB1FE7804E
:1066800020C12A8461B739476391E7164A2085679C
:10669000A5076315F5040C4403CC0500631D0C002D
:1066A000850591C93735002019461305052697A0A1
:1066B000FB1FE78040C803C789248547631FF70E87
:1066C00063080C00238409246285EFF04FBE45B7B0
:1066D00089472384F924EFC0104A51BF8967138783
:1066E00027006318E504032C840063080C0C83471F
:1066F0000C0099EB83472C0003471C00A207D98F9D
:106700009EA483473C009CB003C789248947631635
:10671000F70A83470C0091C72384092403450C0022
:106720006DB78C308A248D472384F924EF70C02EF6
:10673000F5B795076317F5001C448823EFF0CFE405
:106740003DB7F9771387A7FF2A9742074183914600
:1067500063F1E6049387A7FCAA97C207C183714738
:106760006371F70289671387B7006310E50483A795
:106770008AF1E38E07EE9C43A285E38A07EE8297B7
:1067800015A0370700181307F770B357F700858B6C
:10679000B9C783270BF2E38C07EC9C43E38907EC32
:1067A00022858297E31505EC09A81387C700631FAC
:1067B000E5001C449C23E38C07EA9307F00FE308F1
:1067C000FAEAA2855285EFC03FA46DB5B9076318F8
:1067D000F50083A7CCF1E38C07E8DC4371BF896740
:1067E00093871704E305F5F8C9BF3D476397E704AE
:1067F0004A2089671387D700E30DE5FC13879701CB
:10680000E309E5FCCD07E31AF5FAFA20C167FD17A5
:10681000631DF70083A7CCF1E38B07E4DC43E38837
:1068200007E40965A2854D0599BFB737002083A706
:1068300047F2E38E07E29C43DDB71307E003E39ED4
:10684000E7F63C200547639BE7107C2037370020A4
:10685000930D07F16397070E83A70D00E5C303CCE3
:106860000700214A683013078400BA853ACEEFE06A
:106870003FDE68B0130640028145681097A0FB1FF9
:10688000E78000B23C3072471946A307F1027C3022
:10689000BA854818A309F10297A0FB1FE780A0A9B9
:1068A0005E207010D2852318F1027E2462852313A6
:1068B000F1041E282314F1043E282315F1045C285A
:1068C0002306F104FD57A306F104FD572317F10435
:1068D000EFF00FBE3C3072478DE3DD478358040173
:1068E0000358E40074304E203EC23E283EC00546A8
:1068F000D2876285EF80300D28B083A70D0081C755
:106900001145EFF01F9E03C50BF3138C0BF3E3004F
:1069100005D683451DF3EFE0BF8EE30A05D434307E
:10692000930710036389F600522083450C005287B9
:106930003685EFE0FFA423000C0015BB03CC340028
:106940000DB783270BF203CC3400114A81DFDC43FF
:10695000E38A07F081450145829729B71307900222
:106960006390E7087C2037370020930D07F1A9E7F3
:1069700083A70D009DCF03CC0700214A6830937791
:106980002500B9C705891307440168B02286D2855E
:1069900062853ACEEFF0CFB13C307247B9FFDD47A8
:1069A0008358C4010358A40174304E203EC27E2C8B
:1069B00035BF03CC3400D1B783270BF203CC3400AE
:1069C000114ACDDFDC43DDDB8145014582977DB790
:1069D00013078400BA853ACEEFE09FC7724775B7B8
:1069E0000947639CE70083A78AF1E38207C8DC4379
:1069F000E38F07C6228582979DB92D476398E700EC
:106A000083A78AF1E38507C69C47DDB70D476396E8
:106A1000E70022868D454A2005B91947639CE704A3
:106A20009305A10213051031EF60924D6C10130510
:106A30002031EF60F24C72208357C1024A2063E795
:106A4000C70016240357A10263F7E600930500026E
:106A5000EFC0301629B96373E6007AA063F3D7005C
:106A60001EA45A24362412246E2001488147EFC008
:106A70001014F5BE1D47E382E7D431476395E70064
:106A80002286B14549BF35476398E70083A78AF15D
:106A9000E38F07BCDC47A9BF130740026396E700FA
:106AA0002285EF00407EE1B6130750026398E700AD
:106AB00083A78AF1E38D07BA9C4B1DBF41476396BC
:106AC000E7002285EF0090065DB645476396E70034
:106AD0000145EF00701561BE4947639DE7008327BC
:106AE0000BF2E38C07CCDC43E38907CC81450545F9
:106AF0008297E1B14D47639CE70083270BF2E38E59
:106B000007CADC43E38B07CAA2850945D5B713073B
:106B10006002E394E7CA228693056002EDBD93F715
:106B2000150089CFB737002083A787F189C7DC43D9
:106B300099C30145829713451900E9BC93F72500D5
:106B400091CFB737002083A707F291C7DC4381C7F5
:106B5000814505458297134529006DBC93F7450093
:106B60000145E38907AAB737002083A747F13734E7
:106B700000201304842489CF85475CA0B737002008
:106B800083A707F291C7DC4381C7814505458297FA
:106B900048446C10EF90E01D6810EFF00F9AB73783
:106BA000002083D7A72881CF130600643386C7024D
:106BB000B737002003C5C73A9145EFC0FFB613456C
:106BC000490089BC011122CC2A84554506CE26CA2B
:106BD000EFF0CFBCAA8413054002EFF02FBC2AC609
:106BE00013055002EFF08FBBAA862285624432461D
:106BF000F240B3359000D24405616FC07003397123
:106C000022DC06DE8D472E84631AF500BA25962510
:106C1000F2212830CE21EFE0DFF001A88967138749
:106C2000D700631DE504BC2199E78547F250625403
:106C30003E852161828037340020832504F1F5D51B
:106C4000DC87BC31480819469105A309F1009790EB
:106C5000FB1FE780406E930700F03ED6832704F1C8
:106C6000231801002313010202D4882370008145F8
:106C7000EFF00F840545EFF0CFE645BF1387E7003F
:106C8000E305E5FA138737016319E500A82151DD13
:106C90000147814601468145BDBFE507E307F5F899
:106CA000B1476319F500B737002003C5B724EFE0FB
:106CB0009FF2A5BF930760026319F500B737002064
:106CC00003C5B724EFE0BFF58DB741677D17814756
:106CD000E31EE5F4D831C947E319F7F4F625D225C8
:106CE0000A24AE25EFC0607C2DC55D45EFF00FABEB
:106CF0003335A00068844C202A203000EF80A008A3
:106D00003C8485F79305A10013051031EF60521FF5
:106D10006C0013052031EF60B21E3C851A246373AA
:106D2000F7001EA43C863A2463F3E7003EA41E2429
:106D30003A246373F7003EA42A20EF3041107A24EE
:106D4000562432240E242A2001488147EFC02064B3
:106D5000E9BD85477C8445B7B73700201387C73A1C
:106D600074331307F00F638FE6062DCD411122C453
:106D700026C24AC006C6AA8468251389C73A5105A7
:106D80009790FB1FE780604B2A8439C59307000D5D
:106D90001EA1D9473CA1DE205EA1FC207CA1FC30D5
:106DA0007CB19C241CA5DC345CB5F02470A515C214
:106DB0008C48510508C89790FB1FE780C057A285F3
:106DC000224403457900B2409244024941016FC018
:106DD000AFC323280500E5B7B240224492440249DC
:106DE000410182808280C1671387E7FF639DE500D0
:106DF000B737002083A707F195C39C230D47639DF8
:106E0000A7006FC00058FD1749476397F500B737D3
:106E1000002083A707F1F5F73A8582804947EDBF47
:106E2000397122DC06DE26DA4AD84ED652D456D242
:106E30005AD05ECE62CC182185472A846309F704B4
:106E40001025930695009305E1000545EFE0CFE49A
:106E5000814711C11C21142011476382E604373792
:106E60000020032747F38D461833630AD70285CBEA
:106E70001DC70DE10145F2506254D2544259B25936
:106E8000225A925A025BF24B624C21618280814706
:106E90000145D1B78546631ED7088D8BE1DF0830E9
:106EA000130A2400D285EFE0AFFA3739002008B08A
:106EB000832789F32A8B130989F38149C1C3B73A20
:106EC00000209304F00F83C72AF3138C2AF363FA8C
:106ED000F90203250900939B49005E951C216381FB
:106EE00097061C31639E67051946D2850905979060
:106EF000FB1FE780405529C5832409001820DE9434
:106F0000B1E414209147E387F6F683270900BDD347
:106F100003460C0001479305F00FE30DE6F4BE8431
:106F2000C10703C507FF6301B50C05071377F70F0A
:106F3000EDB78946E310D7F4858B8DB7054525BF9E
:106F4000850993F9F90F41B788C4C9A8914763121D
:106F5000F706C8440DC11C241021630EF604182046
:106F600091476318F706C84419C59790FB1FE7803F
:106F7000601A23A60400082491659385E571050530
:106F80009790FB1FE780000C0DC118209147631BF1
:106F9000F704C8C41C24930594000505A30FF5FE4F
:106FA00010249790FB1FE780003908243335A00098
:106FB000D9B5884445B79305940005059790FB1F04
:106FC000E78060488547E31CF5F85545EFE01FFD75
:106FD000ADA088444DD19790FB1FE780A01323A458
:106FE000040051BF88C47DB794A01C30D28513859E
:106FF00024009CB019469790FB1FE780C0330824FB
:1070000091659385F57105059790FB1FE7808003D7
:107010000DC118209147E319F7F2C8C41C24930549
:1070200094000505A30FF5FE10249790FB1FE78041
:1070300080301C2481F708207D151335150025BDEF
:10704000397122DC26DA4ED652D406DE4AD856D220
:107050005AD05ECE2A84930925000831CE85B734F4
:107060000020EFE0EFDE08B0938444F39C400D472E
:107070002A8A9C336390E70437390020832789F3F9
:10708000814A130989F363810714B73B002003C7C2
:107090002BF393970A01C18303250900138B2BF36C
:1070A00063E0E70C83460B000327090081471306C2
:1070B000F00FBDAAF1D3144C70389305E1000545DB
:1070C000EFE08FBD15C9984085461C211833631029
:1070D000D7028D8BD5F30145F2506254D2544259F8
:1070E000B259225A925A025BF24B21618280894640
:1070F000858BE313D7F8F9BF1C2011476385E700A0
:107100002D47E39AE7FCB734002083A784F39384E8
:1071100084F3F1D3814A0149B73B002005A8884098
:10712000139B4A001C205A9518216310F7021C314A
:10713000639D47011946CE8509059790FB1FE7809F
:10714000803001C503A904005A99850A03C72BF3AF
:1071500093970A01C183E3E4E7FCE31F09F0A5BFAD
:1071600093944A00269518211C206318F70A1C31B5
:107170006395470B1946CE8509059790FB1FE7805D
:10718000802C41CD832709001147BE941C206385C4
:10719000E7002D47639CE70203AAC4007C3803463E
:1071A0000A006308F60252859790FB1FE78080F67D
:1071B000683891659385E57105059790FB1FE78019
:1071C00060E81DE5E38004EE054539B703AA8400B5
:1071D000F1B70C4C13051A009790FB1FE780A0260F
:1071E0008547E312F5FC5545EFE05FDB61DDE5B572
:1071F0001C2011476385E7002D47639EE700C8C444
:107200007C380505A30FF5FE70380C4C9790FB1FDA
:10721000E780601245BF88C4E5B7850A8DBDBA8492
:107220004107834507FF638AC5008507C207C183FD
:10723000E3E7D7FE51BF88C425A81C20CE8513855F
:1072400024009CA01C3019469CB09790FB1FE7803F
:10725000800E683891659385F57105059790FB1F41
:10726000E78040DE35D118209147E316F7FCC8C40B
:107270007C380505A30FF5FE70380C4C9790FB1F6A
:10728000E780600B91B701114AC837390020130914
:10729000C93A0347790006CE22CC26CA4EC69307C8
:1072A000F00F630EF70625CDAA8461459790FB1F6A
:1072B000E780A0F82A8425C59307000D1EA1D547B5
:1072C0003CA1BC3093898400CE853CB1DE205EA118
:1072D000FC207CA1E830EFE0AFB768B0CE851305A5
:1072E000840019469790FB1FE780E004FC24A285E8
:1072F000034579007CA49E281EA8BC283CA8BC3865
:107300003CB8DC285CA8DC385CB8FC287CA862446B
:10731000F240D2444249B24905616FB0FFEEF240FB
:107320006244D2444249B24905618280411122C47B
:10733000373400201304C43A783006C626C29307B7
:10734000F00F6309F7021DC5AA8419459790FB1F2A
:10735000E780A0EEAA8519CD9307000D1EA1DD4799
:107360003CA1DE20B24092445EA16830224441013B
:107370006FB09FE9B24022449244410182800111E2
:1073800022CC37340020832784F306CE26CA4AC88D
:107390004EC652C48DC3130484F32E8AAA840149B5
:1073A000084063129902630C0A049790FB1FE78060
:1073B00060D623200400F2406244D2444249B249DC
:1073C000224A0561828093194900B3073501884735
:1073D00009C99790FB1FE780E0D31C40CE9723A4F8
:1073E00007001C40CE97C84709C99790FB1FE7804C
:1073F00060D21C40BE9923A60900050955B745DD9A
:107400001396440081459790FB1FE78060F9144074
:1074100081477D5613F7F70FE37F97F813974700DF
:10742000369710A38507FDB779714AD03739002008
:10743000832749F306D622D426D24ECE52CC56CA42
:107440005AC85EC6C5C7B73A0020AA89130949F3CE
:10745000938A2AF3014405E1B737002083A687F316
:1074600099CA03C60A002A8481479305F00F13F7CF
:10747000F70F6368C7081315340021059790FB1FA9
:10748000E780A0DBAA8411E921459790FB1FE780E4
:10749000C0DAAA8421C10144CD49930700FD9CA014
:1074A0008547A3803401BCA0A0B045C49389840063
:1074B00023A23401014A373B0020930BF00F83C70E
:1074C0000A006373FA0029E883270900A685882348
:1074D000EFB09FD303C50A00814555350325090048
:1074E0009790FB1FE78000C323200900B25022546D
:1074F00092540259F249624AD24A424BB24B456118
:10750000828013974700369718236305B700050458
:107510001374F40F8507A1BF83278BF393154A00DB
:10752000BE959C21638377032380F9009C311385EA
:1075300029007D14A380F900194689051374F40FFE
:107540009790FB1FE78020DFA109050A137AFA0F45
:10755000BDB723A204008DBFB737002083A747F330
:10756000B1C7411122C406C62A841DE10945EFE0D6
:10757000FFA22A8601C9B737002003C5C73A85454F
:10758000EFC08F9A0545EFF0EFE32A84054519C84F
:10759000B737002003C5C73A8545EFC0EFC0228545
:1075A00061350545B2402244410182800145828017
:1075B00089679386B7006315D5009C45882369BF0A
:1075C0009386C7006317D5009C458546882319C953
:1075D000FDB793861704E302D5FE938727048146FF
:1075E000E304F5FE36858280797106D622D426D250
:1075F0004AD04ECE52CC56CA5AC85EC662C479C56D
:107600003C31AA8985C7404115C05945EFE01F9913
:10761000931A850193DA8A410149373A0020130B06
:10762000000DB54B83C73900636EF900B250225488
:1076300092540259F249624AD24A424BB24B224C0E
:10764000456182808307840263C9570783274AF311
:10765000130C4AF3BDC32285EFF08FFC39CD08240B
:1076600051059790FB1FE78040BDAA8439C52310C0
:107670006501230175011C201946930524003CB1C6
:107680008307840215057CA11C30A30FF5FE97909B
:10769000FB1FE78040CA1024D0A415C613854401FF
:1076A00088C8930594009790FB1FE780C0C8832784
:1076B0000C00A6858823EFB03FB50509130494029A
:1076C0001379F90F85B723A80400D5B7B737002081
:1076D00083A747F3A1DF893B2254B2509254025949
:1076E000F249624AD24A424BB24B224C01454561B3
:1076F0006FF04FCD797106D622D426D24AD04ECE25
:1077000052CC56CA5AC85EC662C45DCD3C31AA8905
:1077100085C7444195C05945EFE05F88931A8501BC
:1077200093DA8A410149373B0020930B00FD414C1D
:1077300083C73900636EF900B25022549254025943
:10774000F249624AD24A424BB24B224C4561828096
:107750008387F40063C55707130A4BF383270A0096
:10776000B9CF51459790FB1FE78020AD2A8421C9EE
:1077700023007501A3000500230185019C20194603
:10778000938524003CB18387F40015055CB59C30DB
:10779000A30FF5FE9790FB1FE780E0B99C2493852B
:1077A00094001305C4003CB419469790FB1FE78072
:1077B00080B883270A00A2858823EFB0FFA40509BB
:1077C000C1041379F90FADB7B737002083A747F38A
:1077D000A5D799392254B25092540259F249624ABB
:1077E000D24A424BB24B224C014545616FF08FBDEE
:1077F0005D7186C6A2C4A6C2CAC04EDE52DC56DA8D
:107800005AD85ED662D466D26AD06ECE630E052692
:107810003C31AA848DCB832A450063860A025945F0
:10782000EFE0CFF793178501E1873EC60144B739F2
:107830000020130A000D054CB54C130D00FDC14D81
:10784000B8306361E402B640264496440649F259D2
:10785000625AD25A425BB25B225C925C025DF24D8C
:10786000616182800387CA00B2476348F71603A7A5
:1078700049F3138949F36302071683CB0A0013F710
:107880000B014DCF4D47639EEB0623800A005685C2
:10789000EFF00FFB6303051403C70A00914763E38E
:1078A000E7146319870D51459790FB1FE780E09817
:1078B0002A8B630405122300A501A3000500230100
:1078C000B50183C60A00194693852A0034B1838620
:1078D000CA00150554B583C61A00A30FD5FE9790AC
:1078E000FB1FE78040A583C60A01194693851A014C
:1078F000A305DB001305CB009790FB1FE780A0A337
:10790000F9A055476398EB0005472380EA00A38B55
:107910000A00B5BF7547E389EBFE49476396EB0064
:1079200009472380EA00A5B741476394EB000D4760
:10793000CDBF6D47E39DEBF41147E5B713F78B001F
:1079400019C32D47F9BF13F61B0013F74B0011C6DF
:1079500019C315475DBF2147E9B713F62B0011C6C0
:1079600019C325475DB719476DBF19C3294755BFCF
:107970001D4745BF03C57A0151059790FB1FE7805E
:10798000C08B2A8B39C9231045012301950183C679
:107990000A00194693852A0034B18386CA0015056A
:1079A00074A183C61A00A30FD5FE9790FB1FE78032
:1079B000809803C67A012306CB0001CA13054B0148
:1079C0002328AB0083A58A0105BF23280B0083264B
:1079D0000900DA858822EFB03F830504F10A1374A9
:1079E000F40FB9BD03C57A01130505029790FB1F7B
:1079F000E780A0842A8B75D1C9473CA1231045019B
:107A000003C60A0093F60B0693852A00D18E34B183
:107A100083C61A0019461505A30FD5FE9790FB1FC4
:107A2000E780609183C68A00194693851A01A305F1
:107A3000DB0083C69A0013053B012306DB0083C6E7
:107A4000AA00A306DB0083C6BA002307DB008386F7
:107A5000CA00A307DB0083D6EA002318DB0083C635
:107A60000A012309DB009790FB1FE780C08C03C647
:107A70007A01A30CCB0011C613050B02232EAB0019
:107A800091B7232E0B00A1B7B737002083A747F388
:107A9000E38B07DAEFF05F992644B6409644064937
:107AA000F259625AD25A425BB25B225C925C025D2E
:107AB000F24D014561616FF0EF90B737002083A769
:107AC00047F39DC798238D476315A702B73700205A
:107AD00003C5C73A4111854506C6EFB0FFEC130553
:107AE0000003EFF07F94B240014541016FF08F8DAC
:107AF000C9473E85828079714AD037390020130901
:107B000049F38327090006D622D426D24ECE6398A5
:107B1000070E373400201304C43A5820C947298B74
:107B20005DC79165AA849385D57111459780FB1F28
:107B3000E78040512320A900CD4751C978309307F1
:107B4000F00F6314F7009C207CB01146A685978047
:107B5000FB1FE780407E930531001305F041EF40A5
:107B6000020DB737002093878724A02398813334F0
:107B7000800011C3090413051002EFE02FC213792E
:107B8000F50F9377190093794900B1CB1545EFE0D4
:107B9000EFC0BC20688419455C82EFE02FC0688686
:107BA000638E0900BC2013052002DC82EFE00FBFCA
:107BB000688513053002EFE06FBE6887AC307C004B
:107BC000380054004A862285EFB05006AA87B2508A
:107BD000225492540259F2493E8545618280E14720
:107BE000E38709FEBC20130520025C82EFE00FBB97
:107BF000688413053002EFE06FBA6886C1B7C547E5
:107C0000F9B7757126C3B734002022C506C74AC12B
:107C1000CEDED2DC9384C43ADC204944A18B63815C
:107C20000724B737002083A747F34144639A07220C
:107C3000AA89EFE05F839C2455446373F522B7342F
:107C4000002083A704F126894544639B07209165A2
:107C50009385C57129459780FB1FE780A03E23A827
:107C6000A4F04D44630E051E2946CE859780FB1F68
:107C7000E780606C13056002EFE04FB2137AF50FF6
:107C800093775A006144638D071C130600038145F6
:107C900088009780FB1FE780A07093771A00936994
:107CA0002A000144B9CF4145EFE04FAF2316A104AC
:107CB0003D45EFE0AFAE2319A1043545EFE00FAE2F
:107CC000231CA1043945EFE06FAD231FA10421451A
:107CD000EFE0CFAC2312A1061D45EFE02FAC83A748
:107CE00004F12315A1069C33638507182D45EFE0A9
:107CF000EFAA2310A1043145EFE04FAA2313A104FA
:107D000005441305C002EFE06FA9981893171400FB
:107D1000BA97239EA7FC1305B002EFE02FA89304A7
:107D200084009C188604BE942399A4FC1305900239
:107D3000EFE0CFA6239CA4FC1305A002EFE00FA662
:107D4000239FA4FC13058002EFE04FA593040401D8
:107D50009C188604BE94239AA4FC13057002EFE0DD
:107D6000EFA3239DA4FC137A4A0063040A081305B9
:107D70006003EFE0AFA205049C1893141400BE94B6
:107D8000239EA4FC13055003EFE04FA1130A8400C7
:107D90009C18060A3E9A2319AAFC13053003EFE04B
:107DA000EF9F231CAAFC13054003EFE02F9F231F26
:107DB000AAFC1305E002EFE06F9E41049C18060444
:107DC0003E94231AA4FC1305D002EFE02F9D8327D5
:107DD00009F1231DA4FC9C33C5C713051003EFE074
:107DE000EF9B2398A4FC13052003EFE02F9B239B1C
:107DF000A4FC832709F1A83393854700EFD07F8146
:107E00002AD69305F1031305F041EF305262B737DC
:107E1000002093878724AC230347F1033256B33500
:107E2000B00011C38905832609F1FC009308A1065F
:107E3000A8223EC8930721053EC6BC083EC493074E
:107E4000E1053EC2DC103EC0130861049C004E8771
:107E50009106EFB0205E2A8401C50D45EFE06FC8A2
:107E60002285BA402A449A440A49F659665A496119
:107E700082802545EFE08F922310A1042945ADBDF6
:107E80001305F002EFE08F912398A4FC1305000383
:107E9000A9BFB737002083C7073B0145A18B89C71E
:107EA00037350020130545306FD02FD3B73700206A
:107EB0007D57238907F2B7370020A389E73AB73700
:107EC000002023AC07F237770400B73700201307F0
:107ED000075B23AA07F2B737002023A8E72E3777DE
:107EE00004009387072F1307875ED8C337770400F2
:107EF0001307476F98C7377704001307077FD8C762
:107F000037770400130787D598CB37770400B73746
:107F10000020130767DE23A2E7303777040093873A
:107F200047301307E7BFD8C38280411122C43734DA
:107F30000020130424F326C2AA840820854506C61F
:107F4000EFF0EFC3B737002083C7073BA98BBDC74E
:107F50003735002004A01305052FB7340020EFD0DB
:107F60002FC7938484F39C4099C74D45B240224467
:107F7000924441018280082019E10145C5BF916505
:107F80009385B57112059780FB1FE780A00B88C011
:107F900069DD1020814512069780FB1FE780404075
:107FA000142090408147FD5513F7F70FE377D7FC76
:107FB0001397470032970CA38507FDB701452300AF
:107FC0000400EFD0EFC055BF411122C43734002068
:107FD000032544F106C619C59780FB1FE78080136F
:107FE000232A04F0B240224441018280011113058A
:107FF000700306CEEFD09FFA2AC613058003EFD098
:10800000FFF92AC413059003EFD05FF92246B24569
:10801000F240AA86054505616FB080405D71130589
:10802000D00386C6A2C4A6C2CAC0EFD03FF72A8436
:108030001305C003EFD09FF6AA841305E003EFD029
:10804000FFF52A891305F003EFD05FF58A871377D0
:10805000F50F9376F90F13F6F40F9375F40F0545AA
:10806000EFB0403EB64026449644064961618280A6
:10807000757122C537340020832744F106C726C313
:108080004AC1CEDED2DCD6DADAD8DED6E2D4054575
:108090006389070E9305F1051305F041EF3032397E
:1080A0009305F1051305F041EF307238B737002022
:1080B00093878724BC230347F105B337F00011C32E
:1080C0008907032744F1BEC6283393054700EFD044
:1080D0004FD4032744F1AAC40D452C23AEC2EFD0E0
:1080E000FFEBAAC01145EFD07FEB032444F12ADE59
:1080F00065453824034CB4003ADCEFD03FEAAA844B
:108100006945EFD0BFE92A897145EFD03FE9AA89D7
:108110006D45EFD0BFE82A8A7545EFD03FE8AA8ABF
:108120007945EFD0BFE72A8B13050004EFD01FE796
:10813000AA8B13051004EFD07FE6E2042648B64769
:108140006257F256064696451375F50F93FBFB0FE3
:10815000137BFB0F93FAFA0F137AFA0F93F9F90FC7
:108160001379F90FE1842AD05ECE5ACC56CA52C890
:108170004EC64AC426C262C0930844000545EFB00B
:108180000025BA402A449A440A49F659665AD65AF2
:10819000465BB65B265C49618280011122CC06CE2B
:1081A00026CA8D472E84631AF504B831B7340020EF
:1081B000E947CA21938484246315F700FE2063896C
:1081C000A7049790FB1FE780208D19C17E207EA514
:1081D0003A24162472204E202830EFD09F945A2043
:1081E000FE206309F7008547F2406244D2443E8591
:1081F00005618280FD57FEA0FDB78967CD07631C2E
:10820000F500BC2131476385E7004547E39DE7FC66
:10821000EFD0AFA3C9BFB1476319F500B73700204E
:1082200003C5173BEFD03F9B7DBF930760026319E7
:10823000F500B737002003C5173BEFD05F9E65B749
:1082400041677D178147E311E5FAD4314947E39D42
:10825000E6F8CC212A20300023140100EF60B02D75
:1082600059B7411122C4373400208347C4F326C2D2
:1082700006C64AC01307E00FAE846382E704130703
:10828000F00F1304C4F36384E70211459780FB1FCA
:10829000E780A0FA09CD930700FD1CA189473CA106
:1082A000854704B13CB1AA850820EFA0FFF5F95736
:1082B0001CA0B240224492440249410182802A8992
:1082C00011459780FB1FE78040F765D5930700FDB8
:1082D0001CA189473CA104B1A30125012244B73761
:1082E0000020B24092440249AA8503C5D7F3410158
:1082F0006FA09FF179714AD037390020832749F167
:1083000022D406D626D24ECE52CC56CA4544C5EB10
:10831000B73400209387C43ADC234944958BC5C306
:10832000B73700202E8A9165A38EA7F2AA8993857C
:10833000757131459780FB1FE780C0D0232AA9F0D3
:108340004D4435CD23003501A30005002946D285D3
:1083500009059780FB1FE78000FE832749F19146BE
:10836000B82363E9E60835E74D47B8A3B823136798
:108370000701B8A3930571001305F041EF30320BEC
:108380009C83F1E7B737002003C7A7248D4763100C
:10839000F70CEFD08FB52C00EF70B01D2800EFD098
:1083A000DF994545EFD09FBF014411C91306006412
:1083B0003306C50203C5C43A9145EFB0EFB6228536
:1083C000B250225492540259F249624AD24A45614B
:1083D000828085466314D700754741BF8946631480
:1083E000D700494759B78D466314D7004147B5BFF9
:1083F0005547A5BF9546CA8A630DD70099466315B0
:10840000D7000947B8A331A01D466312C7022381D4
:1084100007006545EFD09FB89307F007E30CF5F42C
:1084200003A74AF13C2393E707043CA3A1B72146E5
:108430006314C7000547F9B725466314C700B4A302
:10844000C9BFA9460544E31CD7F6114765BFEFF045
:108450003FC22A842DD5EFF03FB795B7011126CA48
:10846000B734002083A744F122CC06CE4AC8494441
:10847000B9C39C230D446390A704373900200345FA
:10848000C93A8945EFB04FD20345C93AB737002002
:108490009145239007F4EFB02FD183A744F1014712
:1084A000814680B31306F100854785450145DC8789
:1084B000EFA0D0762A842285F2406244D244424919
:1084C00005618280011106CE22CC26CA4AC88547A2
:1084D000631AF50637340020130404F41E20B9C7CC
:1084E000373700200347C72431E31307B003636B1A
:1084F000F702B734002003C5C43A8945EFB0CFCAAC
:1085000012209307006403C5C43A3306F602894576
:10851000EFB08FA123100400F2406244D2444249DC
:1085200005618280938747FC1EA0FDB7B737002006
:1085300083A747F1F5D36244F240D24442498823ED
:10854000056129BFB734002083A744F1F1D737373D
:1085500000201309C73A83474900918BD5DF89472B
:108560006310F5062D452EC69780FB1FE780E0CCF3
:108570002A845DD1B245930700FD1CA1E547A30005
:1085800005003CA1BC3115051946230FF5FEDC2181
:108590009505A30FF5FE9780FB1FE780C0D9034523
:1085A00059009307F00F6315F50083A744F1882362
:1085B000A2856244F240D244424905616FA0DFC403
:1085C0000345C73A8945EFB02FBE6244F240D2441A
:1085D0004249B7370020239007F405616FF0DF9E12
:1085E000B737002083C7073B958B89CFB73700206B
:1085F00083A7C7F491CBB737002005472386E73020
:108600006FF0DF9E4945828041458280B737002068
:1086100085450145238607306FA01061B7370020DC
:1086200083C7073B958B81CBB73700200547238F46
:10863000E7F26FF0BF9E49458280B7370020814541
:108640000545238F07F26FA03060B737002083C73E
:10865000073B958B638C07129307C01C63FCC70014
:1086600009458280F2406244D2444249B2490945F8
:1086700005618280B737002083A747F16388071020
:10868000B73700209387C7F303C807001307E00F2D
:10869000631EE80E011122CC4AC806CE26CA4EC679
:1086A00088A3130586004205368932844181A5C915
:1086B0009165938565719780FB1FE780A098AA89D3
:1086C00055D1B734002003A584F4938484F409C5FC
:1086D0009780FB1FE78000A41385890023A0A900D1
:1086E0002286814523A034019780FB1FE78040CB81
:1086F0009C402286CA8588439780FB1FE780A0C3E1
:108700009C40A286F240C2A36244D2444249B2498C
:10871000984305468D45054505616FA0B04F9165AD
:10872000938555719780FB1FE780C091AA891DD959
:10873000B734002003A504F5938404F509C5978098
:10874000FB1FE780209D1385890023A0A9002286B6
:10875000814523A034019780FB1FE78060C49C40C3
:108760002286CA8588439780FB1FE780C0BC9C4057
:10877000A286F240C2A36244D2444249B24998431D
:1087800005468D45054505616FA010494945828024
:108790009307C01C63FCA700094582800945F2408D
:1087A0006244D2444249B2490561828055C90111EF
:1087B00022CC2A8421054EC64205AE899165938557
:1087C000657141814AC806CE26CA9780FB1FE780A3
:1087D00060872A8961D5B734002003A584F4938487
:1087E00084F409C59780FB1FE780C09213058900B8
:1087F0002320A9002286814523A024019780FB1F06
:10880000E78000BA9C402286CE8588439780FB1F74
:10881000E78060B29C40C2A3B737002083A747F12E
:1088200085CFB737002083C7073B958B85CBB737FC
:10883000002083A787F491CF9843D6236244F24067
:10884000D2444249B24905468D45054505616FA0B0
:10885000703C01478146DDB7014591B7494581B775
:10886000B737002083A747F18DC7B737002083C7EC
:10887000073B958B8DC3B737002083A787F499C733
:108880009843D62305468D450545D1B70147814616
:10889000D5BF01458280494582809307C01C63FC97
:1088A000A700094582800945F2406244D24442490A
:1088B000B2490561828055C9011122CC2A84210563
:1088C0004EC64205AE8991659385557141814AC86E
:1088D00006CE26CA9770FB1FE780C0762A8961D52D
:1088E000B734002003A504F5938404F509C59780E7
:1088F000FB1FE7802082130589002320A900228620
:10890000814523A024019780FB1FE78060A99C403C
:108910002286CE8588439780FB1FE780C0A19C40BC
:10892000C2A3B737002083A747F185CFB737002010
:1089300083C7073B958B85CBB737002083A707F507
:1089400091CF9843D6236244F240D2444249B2497F
:1089500005468D45054505616FA0102C01478146F0
:10896000DDB7014591B7494581B7B737002083A7E7
:1089700047F18DC7B737002083C7073B958B8DC361
:10898000B737002083A707F599C79843D623054634
:108990008D450545D1B701478146D5BF0145828048
:1089A000494582809307C01C63F4A7000945828073
:1089B000797122D44ECE06D626D24AD0AE892A84E8
:1089C00025C1210591654205938575714181977097
:1089D000FB1FE78020672A89094563040908B7342B
:1089E000002003A5C4F49384C4F409C59770FB1F49
:1089F000E7804072130589002320A9002286814563
:108A000023A024019780FB1FE78080999C40228649
:108A1000CE8588439780FB1FE780E0919C40C2A3EE
:108A2000B737002083A747F1014585CFB73700202E
:108A300083C7073B4945958B8DC76C001305D03024
:108A4000EF40124CB247014593F7070F99CBB73768
:108A5000002083A7C7F48D4505459443D223EFA09A
:108A6000701CB250225492540259F24945618280DE
:108A7000B737002083A787F489CFD2238C434111D5
:108A800006C69780FB1FE780008BB240014541017D
:108A9000828009458280B737002083A787F485C785
:108AA000B737002003A707F5894719CF52230C4396
:108AB000411106C69780FB1FE780E087B2408147DF
:108AC0003E854101828089473E858280B7370020FC
:108AD00083A787F485C7B737002003A7C7F4894762
:108AE00019CF52230C43411106C69780FB1FE78024
:108AF0008084B24081473E854101828089473E851E
:108B00008280797106D622D426D24AD04ECE52CC5B
:108B10008D4763FCA7008944B25022542685025930
:108B20009254F249624A45618280373900200347F6
:108B30008924C144E312F7FE9307F5FF93098924C2
:108B400093F7F70F8546AE842A8403CA29001309D8
:108B5000892463EAF6068DE199452800EFC0DF8994
:108B6000B739002003C5C93A914523018900EFA018
:108B7000BFE335E481444DB719468145280097800D
:108B8000FB1FE780E08119462C0026859780FB1F9C
:108B9000E780608B49F119469305F00F2800977024
:108BA000FB1FE780E07F19462C0026859780FB1F7E
:108BB000E78060892DF11946A68528009770FB1F74
:108BC000E780607771BFE31DE5F803A5C9002C00BD
:108BD000EF70201AAA8449D52381490135BF2800A6
:108BE000EFD0AF95AA8405ED930571001305F04110
:108BF000EF30E2038483BDFC8D47E31DF4F6454569
:108C0000EFD0CFB925D9B7771800938707A03306DF
:108C1000F50203C5C93A9145EFA0BFD1F5BD2301C7
:108C20004901DDBDB737002083C7073B918B8DC35A
:108C3000373500204111130545F406C6EFC02FFB60
:108C4000B240B73700207D572397E7244101828047
:108C500001456FC0CFF9B73700207D57A38EE7F2EB
:108C6000B73700207957238EE7F2B73700202386E5
:108C70000730B7370020238F07F2B7370020239043
:108C800007F4B737002023A407F4B737002023A840
:108C900007F4B737002023A607F437970400B73747
:108CA0000020938787FF130767EB98C3378704007B
:108CB0001307474CD8C3378704001307070798C723
:108CC000378704001307C7FED8C737870400130788
:108CD000C70198CBB7870400373700209387A719BF
:108CE0002322F7F48280411126C2B734002083A7E3
:108CF00044F106C622C49DCB2A840D459770FB1F04
:108D0000E780A053AA8501CD930700FD1CA18D47E4
:108D100000B13CA183A744F18823EFA0EFCE19C492
:108D20002244B240924441016FF00FAAB240224463
:108D3000924441018280797152CC373A00208327D6
:108D40004AF14AD006D622D426D24ECE56CA01497E
:108D5000A1C703C91700B73400208547AA899384A7
:108D600084246305F904DC2005499DE70D459770CF
:108D7000FB1FE780804CAA8509CD930700FD1CA14D
:108D80009147A30035013CA183274AF18823EFA036
:108D9000AFC7EFF06FA30549B25022544A859254F1
:108DA0000259F249624AD24A45618280B7370020AF
:108DB00083A787F4D28A85E30145EFD02F9E2A86C8
:108DC00001CAB737002003C5C73A8945EFA0DF9530
:108DD00083A74AF1B1A09443D2239305E10005454E
:108DE000EFC08FEB71D91C21858BF9D70545EFD0EA
:108DF000EF9A9307B0032A8463FEA702B7370020D7
:108E000003C5C73A5D66130606708945EFA07FB2B9
:108E1000B7370020130444FC239087F483274AF1DA
:108E2000094798B3DC2081C723820400B5B74E857B
:108E30005D3D9DB7130600643306C50251B741116D
:108E400022C42A840D4506C69770FB1FE780E03ECA
:108E50000DC1930700FD1CA1CD473CA100B12244E8
:108E6000B7370020B240AA8503C5D7F341016FA0F0
:108E7000AFB9B240224441018280411122C42A8408
:108E80000D4506C69770FB1FE780203B0DC1930779
:108E900000FD1CA1ED473CA100B12244B7370020E2
:108EA000B240AA8503C5D7F341016FA0EFB5B24028
:108EB0002244410182805A210111896606CE22CCCA
:108EC00026CA13866600AA876316C7009C47014519
:108ED0008C2301A8138686006319C7009C470545AB
:108EE0008C23EFF00FB805451DA81386960063117B
:108EF000C70237370020032747F101450DC39C47C0
:108F0000882369E585471CB30545EFA04047E1BFCD
:108F10001386A600631AC7009C478823293DF240A8
:108F20006244D2440561828013866603E300C7FA77
:108F300013867603E304C7FA13868603631BC70808
:108F40001C45373400201307E00F84238347C4F304
:108F50001304C4F3638BE7021307F00F6384E70283
:108F600011459770FB1FE780402DAA8501CD93071F
:108F700000FD1CA1894704B13CA1A3010500082004
:108F8000EFA08FA8F9571CA0B9BFB737002003A7DF
:108F900047F13E84014541D78DE885447D454485B0
:108FA000EFC0DFFF688613050002EFC03FFF832795
:108FB00044F1C8851307B10084B374001306A100FF
:108FC00085450545EFA0804539BF2685EFF0BFD127
:108FD00019BF13869603E301C7F41386E6036316ED
:108FE000C7001C4509458C23EDBD9386F603631B22
:108FF000D7021C45882335E96C001305D030EF40BB
:109000002270B247414793F7070FE38EE7EC9305D1
:10901000B10013056031EF40A26E88858545EFA051
:10902000A040D1B58966138606046312C7041C45A7
:109030008023B737002083C7C73022859DE70D45C1
:109040009770FB1FE780601FAA85E30E05E8930772
:1090500000FD1CA1D1473CA100B1B737002083A778
:1090600047F18823EFA04F9ABDBDD13BADBD13861C
:109070001605631AC7001C45882331E5854505455B
:10908000EFA0803C8DB5938626050145E319D7E80E
:109090009C478023B737002083C7E7F3228585E705
:1090A0000D459770FB1FE7804019AA85E30D05E287
:1090B000930700FD1CA1F1473CA1B737002000B188
:1090C00003C5D7F345B7553B39BDB737002083C734
:1090D000073B411106C6958B99CB37350020130508
:1090E00085FFEFC02FB04D45B24041018280014560
:1090F000EFC04FAF0145CDBF982193762500937700
:10910000D70F99C293672700131885011358884118
:1091100013F7F7076354080013E7070893768500F1
:109120009377770F99C2936787001377050293F6B9
:10913000F70D19C393E6070294A1634508009377DE
:10914000A50291C71C2293E7C7001CA282807DFD67
:109150001C22CD9BDDBF2D45631B071088210947CD
:109160006313E51001114EC6BE89DC4122CC26CA2C
:109170004AC806CE98339C23B68422075D8F4207E7
:109180008D664187938736A032842E89630BF70A58
:1091900063C0E702938716A06307F70863CAE70A6C
:1091A000938606A0630BD70423900400054559A0BD
:1091B000938766AA630EF708938786B86301F70A58
:1091C000938646A0E312D7FEDC45C1C321479AA08F
:1091D0009A2318A29A23218318B2BA2338A2BA2359
:1091E000218338B2DA2358A2DA23218358B2FA2332
:1091F00078A2FE23A1837CB22DA8C8459770FB1FDF
:10920000E780E01C420541814E86637335012A8662
:1092100092A0420641828325C90022859770FB1FD8
:10922000E780601139A0DC459E238AA01CA2A1839F
:109230001CB20145F2406244D2444249B249056140
:10924000828099479EA01946F9B723900400D5B7AC
:1092500085479EA08327C9009C231CA0D9BFE14756
:109260009EA061464DBF2390060005458280828006
:1092700083C805008947639BF816DC41797122D4C5
:1092800006D626D24AD04ECE52CC56CA03C81700B4
:109290009C232E8422083368F80042088D671358F7
:1092A0000841138327A0630F68102A8A3A89B6847D
:1092B000B285634C0301138707A0630BE802938711
:1092C00017A06301F80A854711A8138737A0630028
:1092D000E80C138767AA8D47E317E8FEB2502254C3
:1092E00092540259F249624AD24A3E8545618280CF
:1092F000484432C69770FB1FE780600D42054181EC
:109300009D47E36D25FDB73A0020938A7AF583C720
:109310000A00B3099900B24563D43701B5477DBF50
:1093200048442686C2094A959770FB1FE780A00033
:1093300003C60A00484493D909010506330636419D
:1093400081454E959770FB1FE7808005B737002059
:1093500083A7C7F599E3814751B79C438145E5DF72
:10936000528525A0AD47E31B09F6E39916FB1C3295
:1093700014225844A207D58F1EA3B737002083A715
:10938000C7F5F1DB9C43E1DB85458297E9B7B73749
:10939000002003C707F68D4731D3AD47E31009F42A
:1093A0009947E39DF6F6484419469770FB1FE780FE
:1093B00080F8B737002083A7C7F5D1DF9C43C1DF12
:1093C0008D4579BFB737002083C5C7ED8D47A1898B
:1093D00091D5AD4701F78547E392F6F4182293073C
:1093E0000008E3EDE6EE5C4498A3B5B785473E85FB
:1093F0008280B7370020411123AE07F4B737002031
:1094000022C4238D07F40944B7370020A38787ECD3
:10941000B7370020A38B07F4B7370020238687ECEB
:10942000B7370020239A07F4B7370020238E87EC44
:1094300037350020B73700202147238007F619462B
:10944000B73700208145130545F606C6A38EE7EC25
:109450009770FB1FE780C0F4B7370020238987ECA3
:109460003707A000B7370020938747ED130707059C
:1094700098C33707E803D8C3B7370020238787ECA2
:109480000547B7370020A386E7ECB7370020238FC6
:1094900087EC37350020B7370020238507F6614673
:1094A000B737002081451305C500238887EC9770E6
:1094B000FB1FE780E0EEB7370020A38887ECB737C3
:1094C0000020A38C07F437970400B7370020938758
:1094D00007E71307671598C3B24022443797040083
:1094E00013070727D8C323A40700410182809547AB
:1094F0006302F51A797122D426D206D64AD04ECE0E
:1095000052CCB2842E8463E4A7048947630DF5141A
:1095100063EFA7004DC50547630FE5120945B2503B
:10952000225492540259F249624A456182808D4721
:109530006304F5149147E313F5FEA1476395F5081D
:10954000373500202146A685130545ED3DAA930732
:1095500020046305F51663E1A7029D476306F51431
:10956000A147E31DF5FA8547639FF5041822B73735
:109570000020A38CE7F4F1A8930710086309F51401
:1095800093072008630DF51493070008E318F5F816
:109590008547639AF502B737002083C787F513879D
:1095A000F7FFB73500209385450212072E979207E3
:1095B00050478820A107BE95EFF01FB459A8930724
:1095C000800F63F4B700614599BF373A00208346A6
:1095D0008AF5B73700201387470292063697484727
:1095E00093894702130A8AF509C99770FB1FE78020
:1095F00060B2B7370020A38B07F4130614009165FF
:1096000093850571328503490A0032C69770FB1FA6
:10961000E78040A383470A0012094E999207232648
:10962000A900CE97C84745D1324681459770FB1FA8
:10963000E78000D783470A002286A6859207CE9747
:10964000C8479770FB1FE78000CFB7370020A38B78
:1096500087F40145E9B5E398F5F61A22B7370020FB
:10966000239AE7F4FDB78547E39FF5F41822B7374F
:1096700000202380E7F6F1BF9947E396F5F43735EC
:1096800000201946A685130545F69770FB1FE78055
:1096900080CAC1B78547639DF5061822B7370020F9
:1096A0000145A386E7EC8280E147E39EF5F037357C
:1096B00000206146A6851305C500C1BF8547E39418
:1096C000F5F01822B7370020238EE7EC59B785470D
:1096D000E39BF5EEB737002083C767F5C9B585472B
:1096E000E393F5EE082293772500E39E07ECB73766
:1096F000002083C717F6B7350020938545021387EE
:10970000F7FF120792072E97A1075047BE956DB538
:10971000614582804111AA8706C611472E8563865E
:10972000E70A6361F7020547638EE706A9C70947A1
:109730006381E7080D476384E7088947B2403E85A7
:10974000410182801D47638AE708636AF700154775
:10975000E395E7FEB737002083C7D7ECB9A82147C8
:109760006383E70813072004E399E7FCB737002079
:1097700083C7C7ED99A0B737002083C787F5139734
:109780004700B737002093874702BA97CC478947ED
:10979000D5D5B737002003C677F59770FB1FE78054
:1097A00080B931A0B737002083D747F59EA1814704
:1097B00071B7B737002083C707F61CA1CDBFB735F7
:1097C00000201946938545F6C9BFB73500202146CC
:1097D000938545EDEF40922DD9BFB7350020614606
:1097E0009385C5005DBFB737002083C797F5F1B7F4
:1097F000630F0538B73700209387A7F598236318C0
:10980000073885463738002094A309479307480254
:1098100098A337F70600130707A9D8C337F7060040
:109820001307C7A5D8C794A7239507007D57630DD5
:10983000E53413771500854539C3B7F606009386DE
:10984000C6A6D4CBB73600209386F6EC0947D4CF12
:10985000B736002098AB238CE6F42380E70237F775
:1098600006000546130747A790AF239D0700D8D3EE
:109870002384C7022395070223A607028D45137789
:1098800025002DC313974500B7F606003E97938633
:10989000C6A654C3B7360020894805469386C6EC51
:1098A00054C72300170110A72315070013871500BD
:1098B00042074183B7360020238BE6F41207B7F640
:1098C00006003E97938646A654C38905B736002006
:1098D000938646F5C2052300170110A7231507003C
:1098E00054C7C181137745002DC313974500B7F6C0
:1098F00006003E979386C6A654C3B7360020894813
:1099000005469386C6ED54C72300170110A72315FB
:1099100007001387150042074183B7360020A38054
:10992000E6F61207B7F606003E979386C6A854C31C
:109930008905B7360020938606F6C2052300170175
:1099400010A72315070054C7C1811377850021CFC5
:1099500013974500B7F606003E979386C6A654C3F4
:10996000854614A7B736002009469386D6ED54C71E
:1099700010A3231507001387150042074183120720
:10998000B7F606003E97938686A954C3A14614A74E
:109990008905B7360020938646F6C20510A3231525
:1099A000070054C7C1811377050129CF13974500DC
:1099B000B7F606003E979386C6A654C3B736002076
:1099C00089480546938626ED54C72300170110A742
:1099D0002315070013871500420741831207B7F6C6
:1099E00006003E97938686A854C38905B7360020A3
:1099F000938646EDC2052300170110A72315070023
:109A000054C7C1811377050229CF13974500B7F6D4
:109A100006003E979386C6A654C3B73600208948F1
:109A200005469386E6EC54C72300170110A72315BB
:109A3000070013871500420741831207B7F6060097
:109A40003E97938686A654C38905B7360020938631
:109A5000D6ECC2052300170110A72315070054C731
:109A6000C1811377050429CF13974500B7F6060087
:109A70003E979386C6A654C3B7360020894805464C
:109A80009386E6ED54C72300170110A7231507009E
:109A900013871500420741831207B7F606003E9769
:109AA000938646A954C38905B73600209386A6F647
:109AB000C2052300170110A72315070054C7C18151
:109AC0001377050821CF13974500B7F606003E9798
:109AD0009386C6A654C3D14614A7B73600200946BC
:109AE000938606ED54C710A32315070013871500AE
:109AF000420741831207B7F606003E97938686A772
:109B000054C3854614A78905B73600209386C6003E
:109B1000C20510A32315070054C7C1811375051092
:109B200039C913974500B7F606003E979386C6A637
:109B300054C3B736002009450546938616ED08A3A1
:109B400010A72315070054C7138715004207418348
:109B50001207BA9737F70600130787A7D8C38905F6
:109B600037370020130797F5C20588A390A72395E0
:109B70000700D8C7C181B7360020938606E7414663
:109B8000130548026F30E039130530037DB10145FC
:109B9000828001111388F5FF06CE22CC26CA4AC85E
:109BA0004EC652C41378F80FAD4563ED050BB7E50B
:109BB00006000A08938505382E983E8A83270800F8
:109BC000BA893689B28482878545EFB09F9F2A84FF
:109BD00019E1EFF08FCF2285F2406244D24442492E
:109BE000B249224A056182808945EFB09F9D2A844F
:109BF0007DF12685EFE06FB3F9BF9145EFB07F9C13
:109C00002A8471F95286CE854A85EFB0FF91EFF034
:109C1000CFCBEFF02F81EF60C07D75BFA145EFB0D6
:109C20005F9A2A844DF95286CE854A85EFB0DF8F40
:109C30002685EFE08FAFEFE0CFA5EF60807961BFC1
:109C4000B145EFB01F982A8459F55286CE854A85D2
:109C5000EFB09F8D2685EFE04FADEFE08FA3EF6073
:109C6000407775B7094485BF79714ECEAE896C00D7
:109C700022D426D24AD006D62A89B284EF0070694F
:109C80002A840DE1CE854A85EFA0BFEA2A8419E92E
:109C90003245B75604002687938666B22D46814525
:109CA000EF1040012285B250225492540259F249D9
:109CB0004561828079714ECEAE896C0022D426D265
:109CC0004AD006D62A89B284EF00B0642A840DE116
:109CD000CE854A85EFA07FF32A8419E93245B7562D
:109CE00004002687938606C04D468145EF00907C90
:109CF0002285B250225492540259F2494561828021
:109D0000397126DAAE844C0022DC4AD84ED652D4C1
:109D100006DEAA893289368AEF00B05F2A8421E9FB
:109D2000A685630D09009E202C007C84BE207C85C6
:109D3000930720307C86930780025C874E85EFA0D6
:109D40007FDC2A840DE55946A6851305A10023046E
:109D500021019760FB1FE780005E1245B7560400A3
:109D60005287938686AD25462C00EF00B07422857D
:109D7000F2506254D2544259B259225A216182801F
:109D8000797126D2AE846C0022D44AD04ECE06D64B
:109D9000AA893289EF00F0572A840DE1A6854E8505
:109DA000EFA0FFDA2A8419E93245B75604004A8742
:109DB000938626B43546A685EF00D06F2285B25033
:109DC000225492540259F24945618280BD47638C06
:109DD000F50663E9B702A5476387F50663EDB700AB
:109DE0009947638CF5049D47638FF5049547638C11
:109DF000F50401458280B5476387F50463E1B70444
:109E0000AD47F5B7DD47638EF50263EAB700C94792
:109E1000638BF502D9476386F502C547C9BFF5478D
:109E20006383F50263E4B700ED47D1B793072005DC
:109E3000638BF5009307200D5DBF48458280084184
:109E4000828008458280484182809307F00F630F2B
:109E5000F506011126CAAA841305000222CC4AC8BD
:109E60004EC652C456C206CE3A89B689B28A2E8AE6
:109E70009760FB1FE780603C2A844D450DC893071F
:109E800000FB1CA0A3005401231144012302340150
:109E900013058400614663050902CA859760FB1FAC
:109EA000E7806049A2852685EF900FB60145F24014
:109EB0006244D2444249B249224A924A05618280B0
:109EC00081459760FB1FE780A04DE9BF094582806F
:109ED000011122CC06CE2A844C86D0869770FB1FB7
:109EE000E78080BB05C15425B73700202147938701
:109EF000C73A639DE600E82378009306E007014631
:109F0000A285A137F2406244056182807800930601
:109F1000E0070146A285C833EDB793070064330616
:109F2000F6026F903F9515C51821854693072700C7
:109F300093F7F70F63FFF600411122C42A843A8594
:109F400006C6EF903FADFD571CA0B2402244410130
:109F5000828082801A219307000B6310F7025C2134
:109F60004947639AE700183985476398E7002A2133
:109F700085456F30101F6D47CDBF828001116C8405
:109F80006C0022CC26CA4AC806CE2A89B6847085BF
:109F9000EF0030382A840DE12C004A85EFA03FAD58
:109FA0002A8419E93245B756040026879386C6A24B
:109FB00015462C00EF0010502285F2406244D24436
:109FC0004249056182807971930720306C847085E5
:109FD0007C862C0093078002014606D65C87EFF052
:109FE0003FD2B25045618280C177797185073EC406
:109FF000894726D27C86AE84930780024C0022D407
:10A000004AD006D62A895C87EF00B0302A840DE159
:10A010002C004A85EFA0BFBC2A8419E91245B75627
:10A0200004002687938606BB45462C00EF00904827
:10A030002285B25022549254025945618280B286E0
:10A0400005466FF0FFCB797126D2AE846C0022D426
:10A050004AD04ECE06D6AA893289EF00902B2A84A8
:10A060000DE1A6854E85EFA05F982A8419E9324557
:10A07000B75604004A879386269D0D46A685EF00B5
:10A0800070432285B250225492540259F2494561DC
:10A0900082807971930720206C8470857C862C00E7
:10A0A00093078002014606D65C87EFF07FC5B25069
:10A0B00045618280011122CC06CE2A842EC632C48C
:10A0C00036C29770FB1FE780209D15C94825B7371A
:10A0D0000020A1469387C73A12472246B245631B28
:10A0E000D500E823B2862E86A2856244F24005613F
:10A0F0006FF0BFD5B286C8332E86A285FDB7F24079
:10A1000062440545056182806FF01FB66FF0DFB5D0
:10A110006FF01FC76FF0DFC679714ECEAE896C004D
:10A1200022D426D24AD006D62A89B284EF00701EE5
:10A130002A840DE1CE854A85EFA03FA32A8419E940
:10A140003245B756040026879386E6B53D468145DD
:10A15000EF0050362285B250225492540259F249EF
:10A1600045618280B28601466FF09FB9011122CC11
:10A170002E846C0026CA06CEAA84EF009019DD4713
:10A180006309F500930710101EA4A2852685EFA091
:10A19000DFA7F2406244D244056182802394050027
:10A1A0009E2599E36FF01FB109458280C5BFB7377F
:10A1B000002003C727FA854763F8E702011122CC84
:10A1C0002E846C0026CA06CEAA84EF00901401E902
:10A1D000930700101EA4A2852685EFA01FA3F240BE
:10A1E0006244D2440561828059458280B73700209D
:10A1F00023A6A7F68280B737002023A8A7F682807F
:10A20000011122CC26CA06CE2A84AE849770FB1F89
:10A21000E7808088A6852285EFA02FD105E92285D9
:10A2200064869770FB1FE78020870DC15425B737E0
:10A23000002021479387C73A639FE600E823780010
:10A240009306F0070146A285EFF03FC0F24062445A
:10A25000D24405618280C833DDB7011126CA06CE1B
:10A26000B68422CCDD4663E3B608D94663FFD50A3F
:10A27000A5466382D50A63EFB6049546638DD5087B
:10A2800099466388D50A054441687D186317060915
:10A290003AC6EFA04FCD3306854032474206418291
:10A2A000420441803305C4004205BA85418132C66B
:10A2B000EF302079AA8751C199C0324692A0B305E8
:10A2C00080406244F240D2443E8505611763FB1F23
:10A2D000670083F1C5466380D504C9460D44E39405
:10A2E000D5FAC167FD17E31DF6FA5DB7F546638041
:10A2F000D50463E4B600ED46D5B793062005638820
:10A30000D5029306200DE390D5F8C167FD170D44E3
:10A310006319F600B5BF094485BF9306200DE3918C
:10A32000D5F8310642064182A5BF15445DBF0D44F4
:10A330004DBFC167FD171D447DB7F2406244D24452
:10A3400005618280011122CC26CA06CED0212E843E
:10A350001307000281469945AA8401372AC621C500
:10A360001E205020930554007C803E207C8189472C
:10A370007C82930780025C839760FB1FE780A0FBD1
:10A380005C208A8526857C84EFA00FF12A8411C584
:10A3900032459760FB1FE780E0D72285F240624498
:10A3A000D244056182804D44CDBF5D7186C6A2C492
:10A3B000A6C2CAC04EDE89476306F600C1470944FB
:10A3C0006318F6040144A9C52E894C0832C6B68923
:10A3D000AA8481272A84324605EDC1778507CA857C
:10A3E0001305D1013ECC230EC1009760FB1FE7800F
:10A3F00080F42C082685B9372A8419E95245B756C6
:10A4000004004E879386E6A71D462C08EF00900AAD
:10A410002285B640264496440649F25961618280FD
:10A42000797122D436844AD04ECE52CCB2892E8A4B
:10A430003A898146130710022286D94526D206D6CC
:10A44000AA84EFF09FE12AC621C12286CA856084D2
:10A4500023124101231331019760FB1FE780A0ED18
:10A460004C002685EFA03F842A8411C532459760B1
:10A47000FB1FE78020CA2285B25022549254025911
:10A48000F249624A456182804D44F5B7011122CC00
:10A4900026CA06CE4AC8DD472A84AE846389F502FF
:10A4A00081470A206C005C86EFA0BF83054563806E
:10A4B000A4080824B165938505B8EF904F91E5474E
:10A4C0003CA0B7570400938787CD5CC085A058395E
:10A4D0003149B2863306270318499C42329710430C
:10A4E000E310F6FCDE225223E31CF6FA8C46084702
:10A4F0009760FB1FE78020F545D55C385828850715
:10A5000093F7F70F5CB863FAE702B387270318489D
:10A510000A20BA979847D623B2238E23113749F1E0
:10A520000824B165938505B8EF906F8A5945F240CC
:10A530006244D2444249056182807C289DB7011162
:10A5400022CC26CA06CEDD472A84AE846394F50663
:10A550000A21EFA04FA1522C36285A286D162A96B0
:10A5600042064182B307D640C20752ACC18363FAA8
:10A57000E7069305C5FF3308F7406359B802BA965A
:10A58000918EC206184C0E280A20C1823E97EFF029
:10A590003FE90DE10824B165938505B8EF902F835D
:10A5A0005945F2406244D244056182806D1593168C
:10A5B0000501C9BF81470A206C005C86EFA06FF2DD
:10A5C0000545E380A4FE0824B165938505B8EF90A6
:10A5D0000F80E5473CA0B7570400938787CD5CC048
:10A5E000C1B78547C9BF397126DAAE842C0022DC99
:10A5F0004AD84ED606DE2A89B289212B2A8439E52B
:10A600004A85EFA04F96D6206D1563C5A600931618
:10A610000501C1829844B2208E204A85EFF05FE0A8
:10A620002A840DE53146A6850808230601009760B7
:10A63000FB1FE78040D0BE202245B75604004E875E
:10A64000938606C75D466C00FC86AD252285F250D8
:10A650006254D2544259B2592161828069B761B7BC
:10A66000797126D206D622D44AD04ECE52CC56CAC2
:10A670005AC88944D9C951CA2E842A89BA8A368BC4
:10A68000328AEFA04F8E93054400814771159A21BD
:10A69000635EA708850793F7F70FB105E319FAFE84
:10A6A0008A854A85BD21AA842DE131453305AA0258
:10A6B000916593851570CD449760FB1FE780809866
:10A6C000AA8921C531463306CA02A2859760FB1FBD
:10A6D000E78060C61844562032200E204A85EFF0ED
:10A6E0003FD4AA8415ED0245B75604008547568726
:10A6F000938606C75D464C005C824EC4230641012A
:10A70000A3060100230761017523B2502254268558
:10A7100002599254F249624AD24A424B45618280C0
:10A720004E859760FB1FE780E09EC5B7ED44F1BF03
:10A7300079714ECE37F60600AE89C16526D2014743
:10A74000AA848946130606AAFD15054522D406D615
:10A750004AD0EF10407B054429C92A8913073002EB
:10A7600081461146F5452685EFF03FAF2AC6554490
:10A770000DCD8357A900CE8601467C8491477C8508
:10A7800085471CA1B2472C002685A38007003247CD
:10A79000FD573CA332473CB3EF10606C2A8411C5CF
:10A7A00032459760FB1FE780E0962285B250225425
:10A7B00092540259F24945618280411106C6EFF078
:10A7C000EFE019C5B24041011763FB1F6700839496
:10A7D000B24041018280011106CE2AC6EF909FDF70
:10A7E0003245B737002023A607F6B737002023A845
:10A7F00007F69145B7370020A386A73AEF30001F30
:10A80000F24005616F2050067971939705014AD097
:10A8100006D622D426D2C187014963DB070AB7379F
:10A82000002003C5D73A2E899760FB1FE78040A61A
:10A830002A8441CD18219307000A6315F70885473C
:10A840004C08DC85EF90BFE5AA8405ED83476101E4
:10A8500071476376F708138717FE1377F70F930690
:10A86000000263F5E608858BCDC7B737002083A7C4
:10A87000C7F6994499C72A201306B1004C0882975D
:10A88000AA849C8599C7084409C59760FB1FE78087
:10A89000608895E05247B7070001938707F07D8FE6
:10A8A000B707120093870710630EF7000347610193
:10A8B000ED476319F7002A208545EF30800ACD4720
:10A8C0006388F4002285EF805F8FA1673349F90028
:10A8D000B25022544A85925402594561828037070A
:10A8E000301405073357F700058B35DF3737002065
:10A8F000032707F759D70347510141F75C8699476A
:10A900002308F1002A206C0023170100EF901FFCA0
:10A910008DBFB737002083A707F78DC32A20130602
:10A92000B1004C08829731DDAA8483475101B1FB05
:10A9300083476101230891005C86E9B79944F5B724
:10A94000397122DC26DA06DE4AD84ED652D456D2E7
:10A950005AD0A5472A84B2846398F50E83474502EE
:10A960001A22835A260085072302F5029307F7FF70
:10A97000B387FA025442C207C183B69703C91700CE
:10A980009C23542522093369F90085476390F60218
:10A9900033075703231006008149014A130B350181
:10A9A000931A070193DA0A0163EA5905C167FD1793
:10A9B0006303F90A1E286370F90A05094209542441
:10A9C000135909012317240105470A209305E400C0
:10A9D000639CE6007C85930720307C869307800289
:10A9E000231421015C872C00EFA0CF910824B165CE
:10A9F000938505B8EF80BFBD5945B9A8B620DC40A6
:10AA00002C28ED1613865900C206C1823E965A853F
:10AA1000EF905FC105C5630B3A01C840B220B30592
:10AA2000350152959760FB1FE780E090BE203E9A6B
:10AA30009E20420A135A0A0185079EA0BE20BE9995
:10AA4000C20993D909018DB75822A9476310F702AB
:10AA50008347450281CF0145F2506254D254425996
:10AA6000B259225A925A025B21618280342813091A
:10AA7000340137F506004A868945130505A9EF908C
:10AA80007FBA19C10545C9BF342837F506004A8683
:10AA900089451305C5A9EF90FFB86DF5342837F542
:10AAA00006004A868945130545A8EF90BFB779F996
:10AAB000342837F506004A8689451305C5A6EF9068
:10AAC0007FB669F1D820BD47E3EEE7FAA567938723
:10AAD0004712B3D7E700858BD5D783474402850754
:10AAE0002302F40203D92400D1B5011106CE2EC6EB
:10AAF0009760FB1FE780A0EF11C93C25B245138783
:10AB000017006395E50093F707F83CA5F24005614F
:10AB10008280011106CE2EC69760FB1FE78020EDD4
:10AB20001DC1B24591C188C11C251307E00F5D45C9
:10AB30006388E7001307F00F01456383E700594579
:10AB4000F240056182800945E5BF411122C42A8493
:10AB5000210506C626C24AC0EFF0EFBC3C20A5176F
:10AB600093F7D70F89EB58248547631EF7041C48D9
:10AB700081443149A1E3FD57230104001CB42302A1
:10AB800004021305C4002244B240924402496146C3
:10AB9000814541011763FB1F67008380B38724034E
:10ABA0003E95084509C59750FB1FE780A0568504D0
:10ABB00093F4F40F5C280848E3E2F4FE9750FB1F7F
:10ABC000E78040554DBF084C75F975B7411122C457
:10ABD000416406C626C29307E4FF6301F502AA8416
:10ABE0009DE19760FB1FE78080E009E91305F4FF12
:10ABF0009760FB1FE780A0DF11C106A1B24022448D
:10AC000092444101828085476392F5049760FB1F5F
:10AC1000E780E0DD2A847DD1FD571EA11C241307A7
:10AC2000F00F6382E7021307E00F6389E700342027
:10AC3000083401475146A685EFF02FA12285EFF099
:10AC4000DFF0FD571CA4230504004DBF8947E3979F
:10AC5000F5FA8545EF40E04155F126859760FB1FE9
:10AC6000E780E0D82A845DF951BF21C518259307F4
:10AC7000F00F6300F704011122CC06CE2A843421A0
:10AC80000E21083501475D46EFF02F9C3820E14743
:10AC90006318F7000A206C0023060100EFA06F8400
:10ACA000F9571CA42285EFF05FEAF2406244056187
:10ACB000828082809307F00F6306F706011122CC91
:10ACC00026CA2A844EC6AE84B689AA859306850014
:10ACD00037B504004AC852C43A89328A1305A5C65A
:10ACE000794606CEEFF06FA3A304240123014401AB
:10ACF0002322340185C01305C4006244F240424956
:10AD0000B249224AA685D244614605611753FB1F0A
:10AD100067006362F2406244D2444249B249224A27
:10AD2000056182808280B7370020238CA7F682805D
:10AD300095476394F50683474502854685072302B8
:10AD4000F5021E2258423022FD17C207C18363124A
:10AD5000D6048A07BA9798339C232207D98F7A257D
:10AD600063F5E704411106C622C485075EA52A845F
:10AD70009305C5000A21EF909FCF0824B165938504
:10AD800005B8EF80DF84B2402244D9473E854101B7
:10AD90008280C946B387D70275BF542229478547A9
:10ADA0006396E6000347450211C381473E858280D2
:10ADB0009D47639BF504834745027625850723025B
:10ADC000F5021E225842FD178A073E971C331823AE
:10ADD000A207D98F014763F2D704411106C622C4E6
:10ADE00085072A845EA59305C5000A21EFF08FD55B
:10ADF0000824B165938505B8EF806FFDB240224409
:10AE000059473A85410182805422A94705476396F4
:10AE1000F60003474502133717003A858280411137
:10AE200022C406C626C2B5472A846395F504834723
:10AE30004502B28485072302F5020A21EF90BF92F2
:10AE40009E201307F5FF014563C1E7027A240A201B
:10AE50009305C400BA977EA4EF907FCF0824B16514
:10AE6000938505B8EF80AFF65945B240224492442D
:10AE70004101828058229D470545E318F7FE0345AE
:10AE8000440213351500D5B7C5476396F5061E2253
:10AE90003A22FD17B387E70203474502050723025D
:10AEA000E5025842C207C1833E973C333823A207CC
:10AEB000D98F41677D176395E70081473E85828082
:10AEC000138717005AA57A25E3F9E7FE411122C43A
:10AED0009305C5002A840A2106C6EF905FD0082496
:10AEE000B165938505B8EF808FEEB2402244D94713
:10AEF0003E8541018280542229478547E390E6FC44
:10AF0000034745025DFB5DBF011122CC26CA4AC83A
:10AF100052C406CE4EC6BC2115472A8AAE8432845E
:10AF20003689639AE7043686A2852685EFF05FE0CE
:10AF3000AA8955E585476314F40A03474900A947E0
:10AF40006300F70288344A8785460146D285EFE0E0
:10AF5000DFEF19E585454A85EFE05FE7133415001B
:10AF6000B420883401476946D285EFE01FEE26857C
:10AF7000EFF0BFBD49A01D476398E7003686A28564
:10AF80002685EFF0FFE26DB725476398E700368628
:10AF9000A2852685EFF0DF9A61BF35476398E70009
:10AFA0003686A2852685EFF09FE759B74547639817
:10AFB000E7003686A2852685EFF01FED95BF5D4739
:10AFC000639EE700D82585473686A2852685631DC2
:10AFD000F702EFF0AFCB8547631AF5048549A54723
:10AFE0006317F402835709009DE30544E38A09F6D9
:10AFF000D947E39EF9F62285F2406244D2444249A1
:10B00000B249224A05618280EFF06FD3E9B78834F4
:10B010004A87A2860146D285EFE03FE379F5A28513
:10B020004A85EFE0BFDA13341500C9B70544E1B72C
:10B03000397122DC06DE26DA4AD84ED652D456D2F0
:10B040009E211944B9E783C925002A89328A93874A
:10B0500059FE93F7D70FAE84DDE3B737002083C6E0
:10B0600087F71307F00F938A87F719446383E60283
:10B07000F5476395F9049760FB1FE7804097AA891D
:10B080001DCD30250DCE93178601E18763DD0700C6
:10B0900001442285F2506254D2544259B259225A84
:10B0A000925A21618280F5454A85EFE07FE283C7AD
:10B0B000A90093E707F82385F900D9BF8149D62075
:10B0C00090448C3088203800EF90BFC22A8471F100
:10B0D000B42003C50A0038000146CA85EFE0FFD658
:10B0E0002A8445F9B24799C323000A00BC2075475A
:10B0F000E390E7FAE38E09F82385F90059BF9760DA
:10B10000FB1FE780C08EAA8A41D58547639FF90857
:10B11000CE2088443000EF90EFE62A843DF903C743
:10B120002A00C54763FFE708DD47630DF70AB73715
:10B13000002003C59A0083C7D73A6398A70A014441
:10B1400003C72A008D47631EF7043C8403D7CA0057
:10B1500063F4E7002396FA0083D5CA004A85EFF02E
:10B160002F8AB737002083D7C71F6D47637BF7024D
:10B1700083D5CA005D476376B70213873500910512
:10B180006349F7001307B00FBE856374F70093059A
:10B19000B00F1166C20513060629C1814A85EF80EA
:10B1A000401B5685EFF07F9AEDB53C211144E392A8
:10B1B00037EF5C41E38F07ECCE2088443000829764
:10B1C000A9BFB72702009387072AB3D7E700858B6B
:10B1D000B9DFB0203400D6854A85EFF0FFD22300D6
:10B1E000AA0045BD83A70A01E5B7B420380001468F
:10B1F000CA85EFE09FC52A8421F5AC202800EFE046
:10B20000FFBC15DD23000A0025BF011122CC373415
:10B21000002006CE26CA4AC84EC652C49309C43A74
:10B2200003C589009307800291653305F502938574
:10B23000657037390020930449F79750FB1FE7806A
:10B2400060E003C689009307800281453306F60259
:10B2500088C09750FB1FE780A0149C404D459DCFB0
:10B260009304C43A130949F70144130A8002FD59B3
:10B270009C24636DF40237B5040013050503EFE069
:10B28000FFF637B504001305A5AEEF900FC037B534
:10B2900004001305C5BCEF30D0540145F2406244B0
:10B2A000D2444249B249224A05618280B30744032D
:10B2B000032509006146814505041374F40F3E958A
:10B2C0002310350123010500231435012305050052
:10B2D0002302050231059750FB1FE780600C49BF30
:10B2E00001458280B737002083C6573B814763E51D
:10B2F000D70001473A8582802E87910503D6C5FF86
:10B30000E30AA6FE8507E5B70DC93C210547890775
:10B3100093F7F70F6373F702411122C406C62A841C
:10B320000E2128310147F9465D46EFE01FB2F9577B
:10B330003EA0B2402244410182808280B737002083
:10B3400003C7573BFD56814763E3E700828016A1A0
:10B350002301050085071105C5BF014582803736E9
:10B3600000201306F6EE930700021CA237370020D8
:10B37000FD572307F7EE373700202300F7EE373766
:10B380000020A30FF7EC8545B73700202396B7EED2
:10B39000B7370020239D07F6B737002023A207F810
:10B3A000B737002023AA07F8B737002023A407F8EF
:10B3B000B7360020B7F70600938646EE938707A8B6
:10B3C000DCC2B7370020238E07F6B73700209387FB
:10B3D000C7E7094798A298A398AB2380E702238880
:10B3E000E70237F70600130707A7D4C7D8DBB7F67D
:10B3F00006000D47238CE7029386C6A63737002048
:10B40000D4CB032707F837F50600B7F60600130577
:10B4100005A9938606AAC8C38CA7239507008CAFFD
:10B42000239D0700D0CFD4D323840702239507029E
:10B4300023A60702239D0702D8DFB737002037B7BE
:10B4400004009387C7EB1307075023A00700D8C356
:10B4500023A407008280411106C6EFF0BFE809C5AA
:10B460002821B240410182800145E5BF411122C43B
:10B4700026C24AC006C6AA842E893284EFF09FE60F
:10B4800009E94165CA857D15EFF0DFE5C54701C5CE
:10B4900006A120A18147B2402244924402493E8540
:10B4A0004101828039E389483547639116050111CE
:10B4B00006CE22CC26CA1832102293C7F7FF2207E5
:10B4C000598EF18F32C68DE7C4452A84A685EFF0E8
:10B4D0009FF832460147630FA60022856244F2407E
:10B4E000A685D24405616FF07FF82D473A858280AA
:10B4F00013070008F2406244D2443A850561828015
:10B5000083C8050009486395080303A845008347DD
:10B51000180003480800A207B3E70701C2070D6837
:10B52000C187130828906395070189476FF09FF73B
:10B5300005458280011122CC37340020130404EE2B
:10B54000182006CE26CA4AC84EC69307F00F630FCE
:10B55000F702AA892945B2842E899750FB1FE780FC
:10B56000C0CD0DC59307100B1EA1230205002311AA
:10B5700035012313250106A5AA8508206244F2405F
:10B58000D2444249B24905616F701FC8F24062441B
:10B59000D2444249B249056182804111B737002047
:10B5A00026C2AE8483A507F822C406C62A84EFF01B
:10B5B0009FEA098909C922852244B240A68592449E
:10B5C00041016FF0EF96B24022449244054541019B
:10B5D0008280411122C426C24AC006C6AA8413042E
:10B5E00045001309850B1E209DC3084409C59750CB
:10B5F000FB1FE78020B22285314681459750FB1F13
:10B60000E78000DA3104231A04FEE31E24FDB24071
:10B610002244FD579EA00249924441018280B737DF
:10B62000002003C6573BB737002003A7C7F8814760
:10B630006315F600814636858280BA861307870B2C
:10B64000835587F4E389A5FE850793F7F70FCDB7F8
:10B65000B737002083A747F981CBDA236314A7000B
:10B66000884782809C43CDBF01458280411106C638
:10B67000EFF01FFE09C50845B24041018280014537
:10B68000E5BF011126CA9384450022CC4EC606CEE2
:10B690004AC852C456C25AC02687814901448146CD
:10B6A00081473D45122345CABDEE42233E23B28663
:10B6B000A297C207C18385093107E395A9FE35C466
:10B6C0002E8991659385457022859750FB1FE780F1
:10B6D00060972A8B39C9814A014A8C4495C1D2208E
:10B6E00033054B019750FB1FE780E0C4DE20884400
:10B6F0003E9A420A135A0A019750FB1FE78080A125
:10B7000063890A003146814526859750FB1FE780F3
:10B7100020C9850AB104E3E23AFD23266901231416
:10B720008900054521A0630DD6000145F240624421
:10B73000D2444249B249224A924A024B0561828070
:10B740003223E314F6FE52233294B2974204C20726
:10B750004180C1838DB70545E37A35FD8DB7B73795
:10B76000002083A787F899E30145828098473A270C
:10B770006315A7001385470082809C43EDB74111F4
:10B7800006C6EFF0DFFD09C50A21B2404101828003
:10B790000145E5BF411106C6EFF07FFC09C5282130
:10B7A000B240410182804145E5BF411122C42A8453
:10B7B0002E8506C6EFF01FFEAA8505462285EF30CE
:10B7C000406B95476305F500BD476313F5002145C0
:10B7D000B2402244410182804111B737002022C487
:10B7E00006C603A487F88146938787F821C01844CA
:10B7F000322718406317A60285CA98C22E8581C9D0
:10B800002146930544009750FB1FE780C0B2228574
:10B810009750FB1FE78000900145B2402244410150
:10B820008280A2863A84D9B798C3C9BF0545F5B7C7
:10B8300037370020832747F90146130747F9A9C77F
:10B8400003D847009443631CA802011106CE22CC02
:10B8500026CA0DCA14C2AA843E852E849750FB1FA7
:10B86000E780408B2C002685EFF01FF701E519C01B
:10B87000B2471CC0F2406244D244056182803E86D9
:10B88000B68775BF14C3C1BF05458280411122C46C
:10B890002A84090506C6EFE00FE9FD573CB0B24027
:10B8A000224441018280411122C4416406C626C25D
:10B8B0009307E4FF6301F502AA849DE19750FB1F03
:10B8C000E780001609E91305F4FF9750FB1FE78096
:10B8D000201511C106A1B240224492444101828048
:10B8E00085476392F5049750FB1FE78060132A8415
:10B8F0007DD1FD571EA13C201307F00F6382E702A4
:10B900001307E00F6389E70028300147F9465146E5
:10B91000A685EFE08FD32285EFF05FF7FD573CA0BF
:10B92000230204004DBF8947E397F5FA8545EF30C0
:10B93000407455F126859750FB1FE780600E2A84DE
:10B940005DF951BF1D71A6CACEC686CEA2CCCAC8AB
:10B95000D2C4D6C2DAC05EDEAE84AC21F947AA8971
:10B960006397F5049750FB1FE780800B2A8411ED45
:10B9700001442285F6406644D6444649B649264AE3
:10B98000964A064BF25B256182803C210547890778
:10B9900093F7F70FE37EF7FC28310147F94601469C
:10B9A000CE85EFE08FCA2285EFF05FEED1B703AB13
:10B9B0000400B7070001938707F037071200B37739
:10B9C000FB0013070710B28A0149638BE7022EC6FA
:10B9D0009750FB1FE780C0042A89B24515C150214A
:10B9E00005C293178601E187E3C407F84E85EFE0AF
:10B9F0002FCE8347490093E707F82302F9008DBF54
:10BA0000373A00200347EAEE9307F00F130AEAEEF5
:10BA10001944E300F7F6E147E3EDB7F493D71500D7
:10BA2000FD1713973700B7E706009387073BBA97D0
:10BA300003A80700E30F08F283AB4700E38B0BF288
:10BA4000420B135B0B0163050B00C947E393F5F24F
:10BA5000D62090448C308820380802982A8411F926
:10BA60002C084E85829B2A8431C19C30E39307F0D9
:10BA7000BC20230AA10039472308F1006396E7029E
:10BA800062471C331823A207D98F0C084E85FC810E
:10BA9000EF80DFE3E30E05EC14080546D9454E853B
:10BAA000EFE04FE12A84F1B5BC84C5B7B4209147DB
:10BAB000E380F6EC03450A0038080146CE85EFE046
:10BAC000CFB82A84E31705EAAC202808EFE00FB0CE
:10BAD00019C123800A009840B7070001938707F037
:10BAE0007D8FB707120093870710E303F7E8E301A0
:10BAF00009E8BC202302F900ADBD011106CE2EC617
:10BB00009750FB1FE780C0F111C95C21B245138734
:10BB100017006395E50093F707F85CA1F240056113
:10BB20008280397152D42E8A4ED69305E101AA89BA
:10BB3000528522DC4AD856D206DE26DA328936C64B
:10BB40003AC4BE8A9750FB1FE78040F0054435C1D8
:10BB5000AA84A8873944EFF0BFAF21CD0328450060
:10BB6000630908042247B246D6874A86A6854E85D1
:10BB700002982A841DED9307E00F638CFA02982047
:10BB800089476318F702D8401C331823A207D98FBE
:10BB9000C2070D67C18713072790639CE70083479F
:10BBA000190003460900D285A2075D8E4E85EFF08D
:10BBB0007F982285F2506254D2544259B259225A87
:10BBC000925A21618280797122D422214ECEAA8993
:10BBD000228556CA06D626D24AD052CC5AC85EC64C
:10BBE00062C4AE8AEFF0BFA301E92285EF90CFD9FE
:10BBF000594431E50144A1A003C789008547AA84BF
:10BC000001446317F702AA8513858900EFF07FA727
:10BC100029C9FA209624D044CE2003D52900E14733
:10BC2000EFF03FF0D9472A846318F50223A60400F9
:10BC30002685EFF01F9A41C0D947E30DF4FA22851B
:10BC4000B250225492540259F249624AD24A424BAB
:10BC5000B24B224C4561828061DDDE202390FA00E8
:10BC6000C1BF13894400014AB94B594C3D4B835520
:10BC70000900DDDDE14763067A010357C90011C3FE
:10BC8000D94703572900835649000326890003D565
:10BC90002900EFF01FE92A84631985012324090094
:10BCA000050A3109E3156AFD61B77DD9835709009B
:10BCB0002390FA00F5B703D529000DBF0111708755
:10BCC0009307E00F1306E1000147894606CEEFF027
:10BCD0005FE5F24005618280797122D42A840A25C9
:10BCE00026D2AE849305210106D64AD09750FB1F79
:10BCF000E780C0D579C51C252AC693F707029DC7E2
:10BD0000A881EFF0BF96AA87B24511E91E243945F4
:10BD10009EA0B250225492540259456182802A203A
:10BD20004946829701C51E249EA0E5B70359240009
:10BD30004A85EFF0DF8E01ED41657D15EFF03F8E16
:10BD400009E51E2425459EA0E9B723102501130708
:10BD500045008147BD46122339EE3147B387E702DC
:10BD6000130984003146CA8591073E959740FB1F11
:10BD7000E780605C3146CA8548089740FB1FE78032
:10BD8000805B52242A2041478146DD45EFE0EFCC1D
:10BD90002ACE09E51E2445459EA0A5BF0C48522485
:10BDA0009740FB1FE78020592A204C08EF908FB95D
:10BDB0002DD15945B9BF85073107E39ED7F82545F1
:10BDC0009DB705458DB7797122D42A840A2526D2DC
:10BDD000AE849305E1014AD006D632899750FB1F05
:10BDE000E780C0C62DC91C2593F7070295EF1838C8
:10BDF0009307200511E35C20362450440E242A20AA
:10BE00000147EFF01FD2AA8729E11C3891E72A20C9
:10BE1000EF904FAFD94711E18147B250225492546D
:10BE200002593E85456182802AC6A887EFF01F84AB
:10BE3000AA8705C5B2452A2049468297AA8745D9CF
:10BE40001A249AA0183869FBC9BF5947E31AE5FEBE
:10BE500023000900D1B78547E5B7B947D5B7397190
:10BE600022DC4AD84ED652D406DE26DAAA892E8A99
:10BE700032C636899750FB1FE78080BA09440DC54A
:10BE80003C211307E00FAA845D44638FE70013078A
:10BE9000F00F5944639AE700324605E2D2854E8599
:10BEA000EF90AFB22A841DCD2285F2506254D25455
:10BEB0004259B259225A2161828003550A009305E2
:10BEC000E101231F01009750FB1FE78020B8A887DE
:10BED000EFF05F8CAA8505464E85EF2090792A8485
:10BEE00055DDD9B79307F00FE300F9FC37B504002F
:10BEF000938624007946A68513058530EFE0EF810F
:10BF0000A381240155B73971B737002026DA83A4FD
:10BF100087F852D45AD05ECE62CC06DE22DC4AD8F4
:10BF20004ED656D266CA2A8BAE8B328C368A99E0B0
:10BF30008149A9A0804483DC44000149835AA400BC
:10BF4000631499018440E5B73E24A28963F8670130
:10BF500005094209135909014104DDB7E3EAFBFE73
:10BF6000630B0A000C204840D28662863AC6EF80F6
:10BF70006FEB324771DD19C323105701F250625441
:10BF80004E85D2544259B259225A925A025BF24B10
:10BF9000624CD24C216182809A21B621854763E5AB
:10BFA000E60439C34111D42126C237F50600938433
:10BFB000550022C426862E84130505A9894506C688
:10BFC000EF804FE6C14719C954202E200A200147AF
:10BFD0002686EFF05FF3814711E1A947B240224482
:10BFE00092443E85410182803E8582802E860A22CF
:10BFF000AE21854763E1A50219CD542241110147C5
:10C00000150606C6EFF03FF0814711E1A947B2409F
:10C010003E85410182803E8582802E860A22AE21A5
:10C02000854763E1A50219CD542241110147150648
:10C0300006C6EFF05FED814711E1A947B2403E85AA
:10C04000410182803E85828039714ED6BE2183D9DE
:10C05000050006DE22DC26DA4AD852D456D25AD05F
:10C060005ECE62CC66CA6AC863EA371585476388C4
:10C070000912416BAE8A2A8A2314010002C60144C8
:10C0800001497D1B894B054CC94C054D83D52A00C0
:10C090000147814601464E8523130100EFF0BFE6BC
:10C0A000AA84630B050E09EC1307200293066100B6
:10C0B0005A8695455285EFE04F9A2A84630205100F
:10C0C00038849C2041CB18856305A70741476385C9
:10C0D000E7022C005285EF80FFD309CD34001546CE
:10C0E000D9455285EFD01FFD11C532459740FB1F42
:10C0F000E7804002814765A0BE2441461305240025
:10C100001CA0BE24A1831CB0CC409740FB1FE7803D
:10C11000802249043C848507C207C1837C8463FD77
:10C120002707BE24638A67078509C20993D90901D5
:10C13000B1BFE39077FBBE240946130524001CA081
:10C14000BE24A1831CB0CC409740FB1FE780A01EFB
:10C150001104C9B722C603596100B824130524008D
:10C16000638F7701335999032305710118A0BE2409
:10C170004146A1831CB0CC401379F90F79B7230550
:10C18000810118A0BE24135929001379F90FA18346
:10C190001CB00946CC404DBF3C8485FFA947F250F6
:10C1A0006254D2544259B259225A925A025BF24B0B
:10C1B000624CD24C424D3E85216182808547C5B795
:10C1C000C547F1BFB737002003C727FA854763F497
:10C1D000E706011122CC26CA4AC806CE2A84328933
:10C1E000AE849750FB1FE780A08319C538219307C1
:10C1F000E00F5D456308F700631C0900A6852285F2
:10C20000EF805FF9F2406244D24442490561828086
:10C210008A209305E100231701009750FB1FE78058
:10C22000E0822887EFF00FD7AA8505462285EF2008
:10C23000504469D5C1BF5945828013F7050201C733
:10C24000B2856FF08FD6411126C24AC006C622C4FD
:10C2500013F98500AA846317090013978501618784
:10C26000635B070232853684EFF0CFD2AA8505469C
:10C270006313090001462685EF20B03F01E901451F
:10C28000B240224492440249410182801C34EDDBD9
:10C290001C24F5F7F5B793F72500F5F30D45CDB759
:10C2A0007971AE8622D42A848A229305E10106D6CA
:10C2B00036C69740FB1FE780607919C90C25B24646
:10C2C000B0872285EFF07FF7B2502254456182801B
:10C2D0000545DDBF13F7050201C7B2856FF0EFCC4E
:10C2E000411122C426C206C693F485002A8491E433
:10C2F000139785016187635007023285EFF08FC97C
:10C30000AA85054691E0014622852244B240924426
:10C3100041016F20103693F72500014591E30D454B
:10C32000B24022449244410182807971AE8622D487
:10C330002A848A229305E10136C606D69740FB1F60
:10C34000E780C070B24611C90C25B0872285EFF096
:10C350007FF8B2502254456182800545DDBF797176
:10C3600026D2AA842A25C16722D44AD04ECE06D628
:10C3700023170100FD173284B6890149630CF500CB
:10C3800005059420D04042051307E1004181EFF0FC
:10C390009FB72A899420D04037F5060089451305B8
:10C3A00005A9EF802FA815C5A2242285EFF02FBD87
:10C3B00009C57D142A9442044180638409002390B6
:10C3C0008900B25022544A8592540259F24945617B
:10C3D00082809420D04037F5060089451305C5A911
:10C3E000EF804FA471F19420D04037F506008945C5
:10C3F0001305C5A6EF800FA311C9E30809FA3C870E
:10C40000E39587FA0354A9007D1475B7A22475B784
:10C41000397122DC26DA4AD84ED652D456D25AD0B6
:10C4200062CC06DE5ECEBE899C252A8AAE84C18B94
:10C43000328C36843A89C28A468B9DE783CB0400CE
:10C440008947638BFB046285EFF08FA01DC18328B1
:10C450000500638008025A88D6874E87CA862286DE
:10C46000A6855285829839A03285EFF02FA0AA8741
:10C4700011ED3945F2506254D2544259B259225A00
:10C48000925A025BF24B624C216182802946A6855A
:10C490005285829745D5F9BFD8401C331823A2078F
:10C4A000D98FC2070D67C187930607906383D71E94
:10C4B00063CCF60693062780638ED70A63C0F60224
:10C4C00013070780E3C1E7F82D45E39509FADC443B
:10C4D0009023CC432310C9002285B9A213073780CB
:10C4E000E393E7F62D45E39709F885472310F90014
:10C4F000DC4481459C231CA0AA24050542054181FA
:10C500009740FB1FE7808054835709006310051094
:10C5100091072310F9001146814513051400974037
:10C52000FB1FE780E0E7F1A8930627906386D71406
:10C5300063C1D71093063790638DD71413074790C4
:10C54000E393E7F02D45E39709F2DC441D47231000
:10C55000E900982318A0983318B0BA2338A0BA235A
:10C56000218338B0D82358A0FA2358B0FE23A183E2
:10C570007CA041A82D45E39F09EEDC446C0083C9F3
:10C5800017009823A209B3E9E90011472310E90035
:10C590009C234E851CA0DC449C331CB09740FB1FA1
:10C5A000E780C04AAA8425C13086C1659306E100B0
:10C5B000FD158329C500EFF09FDA09ED9420D040E6
:10C5C00037F5060089451305C5A9EF80AF8519E148
:10C5D000FD577C8703C7090089476310F70283A5CD
:10C5E00049000946130544009740FB1FE780A0D48B
:10C5F0008357090089072310F9003C873CA0A183D9
:10C600003CB0014585BD23173101C5BF18218907FD
:10C61000BA972310F9003E251CB03E25A1833CA00B
:10C6200010214C41130534009740FB1FE780A0D038
:10C63000C9BFC8449740FB1FE78060D99317050125
:10C64000C1832A871D45E3E737E36399F900231087
:10C650000900CC4403560900CE95BDBD4207B38600
:10C660003A01418363C7E600B38737412310F900DD
:10C67000CDB723105901F1BF2D45E39D09DECC4410
:10C680005285EFE05FDD2310790108A0218108B019
:10C690008DBF2D45E39009DEDC44231079019C23F6
:10C6A0001CA0DC449C331CB0A9BF1D71CAC82A89D8
:10C6B0002A21A2CCCEC6D2C4D6C2DAC05EDE62DCEB
:10C6C00066DA6ED686CEA6CA6AD8AE8AEF80AF8901
:10C6D000130CF5FF93170C01B73B0020C1832A8A86
:10C6E000814913844B153EC6373B0020B73C0020E0
:10C6F000C16D8357C90063F5F9001E2063CC870123
:10C700000355290093854B15EF80BF942A8D15CDD5
:10C71000594D25A883278900139719009305E10136
:10C72000BA9784339C23A204DD8C26859740FB1F97
:10C73000E780C031AA8515E923909A004840054D4D
:10C7400009C59740FB1FE780E09CF64066446A8578
:10C75000D6444649B649264A964A064BF25B625C85
:10C76000D25C425DB25D25618280324883484900D7
:10C7700083A64CF8B0870355290081471307ABF710
:10C78000EFF01FC92A8D13884CF809C523909A0031
:10C7900048407DB75C4085E70355290051478146F5
:10C7A0001386FDFFBD45EFD05FABB737002048C013
:10C7B000138847F809E523909A00454D79B71E2064
:10C7C0000357ABF79304ABF73E976346470113C794
:10C7D000F7FF52979AA048409220832508003E9583
:10C7E00085099740FB1FE78000B51E209A20C209EB
:10C7F00093D90901BA971EA0EDBD397122DC2A84B4
:10C800002A2106DE26DA4AD84ED652D45AD05ECE37
:10C8100062CC66CA2E8B56D26AC8EF70DFF42A8AC1
:10C8200054242E240A2478001306D400130CBAFFD3
:10C83000651AEFF04FED420A37390020AA8981448A
:10C84000135A0A01B73B0020B73C002013094915D1
:10C850006382090463D08405938A4CF883484400BA
:10C8600083A60A0030862A20528881471387ABF7B7
:10C87000CE85138DABF7EFF0BFB91DC1814A30866D
:10C880002E244E859306E100EFF07FADAA896399CF
:10C890000A065DFDF1E41E2429452310FB0035A89E
:10C8A00083570D001228E31BF6FC83A50A004848B5
:10C8B0009740FB1FE78020B971D18327490095EF8E
:10C8C0002A204166454781467D169D45EFD0FF9859
:10C8D0001DE11E2445452310FB00F2506254D25442
:10C8E0004259B259225A925A025BF24B624CD24CD4
:10C8F000424D216182802322A90083DAA90041B739
:10C9000083274900A6972380570193871400139724
:10C91000070183274900418393DA8A00BA9723806D
:10C920005701138724008326490093873400420768
:10C9300091044183C207C204C183C180369711C9E3
:10C94000348714A303274900BA973887218398A313
:10C9500001B7FD5614A303274900BA9794A31DBF3E
:10C960002A20B73500208980239A95149385451590
:10C97000EF80CFD53DD159458DB7411122C406C6B0
:10C9800093F705012A84328585C3EFE0BFE0AA85CD
:10C9900005462285EF20E04D95476305F500BD472C
:10C9A000631DF502214515A893F7450099CBEFE0EB
:10C9B0007FDE0546AA8522852244B24041016F20D0
:10C9C000404B93F7050489C7EFE0DFDC0146DDB794
:10C9D00013F51500133515000605B2402244410138
:10C9E000828079714AD04ECE52CC06D622D426D23D
:10C9F0002A8AAE89014983D749006364F900014559
:10CA000081A083A70900131419009304140033872D
:10CA100097001823A297882322079305E100598DD8
:10CA20009740FB1FE780800205E583A709000545C5
:10CA30003E94182098A383A70900BE94982098B329
:10CA4000B250225492540259F249624A456182809E
:10CA50000C2530875285EFF05FF201CD83A70900E6
:10CA60003E94182098A383A70900BE94982098B3F9
:10CA7000C1BF0509420913590901B5BF011122CCF3
:10CA80002A848A219305E10006CE9740FB1FE780A8
:10CA9000E0FB11C90C2530872285EFF01FEEF24034
:10CAA0006244056182800545DDBF1D71CAC82A89BF
:10CAB0002A2186CEA2CCA6CAD2C4D6C2DAC05EDEF5
:10CAC00062DC66DA2E8ACEC66AD86ED6EF70BFC92F
:10CAD0002AC68346C9008355A900035589007808F2
:10CAE0001306D900EFF02FC2B247B7340020416BD4
:10CAF000938AA7FFC20AAA8B014493DA0A01373C42
:10CB00000020B73C0020938444157D1B63820B18E2
:10CB1000B08683C58B0003552900EFF01FE6AA8D70
:10CB2000631305168348490083A64CF8B086035565
:10CB30002900568881471307ACF7DE85EFF05F8D3B
:10CB4000AA8D9309ACF7138D4CF8631E051215CC12
:10CB500003D70900BE2011076397E7003247A29769
:10CB60006D1763C7E706B735002093874515BA23CD
:10CB700003552900938545153354E40282A3EF80C1
:10CB80000FD1AA8D15C1D94D05A0035529004947DC
:10CB900081465A86C545EFD04FECC8C015E583D70E
:10CBA000AB00C54D2310FA00F64066446E85D644AE
:10CBB0004649B649264A964A064BF25B625CD25C0D
:10CBC000425DB25D2561828083D709009107BEA0D6
:10CBD000DC4003D7AB009306E101A29798A393072B
:10CBE000140013970701DC4041835E85BA9703D791
:10CBF000AB00218398A3B0868355A900EFF02FF6F0
:10CC000013072400D44093073400420711044183E2
:10CC1000C2074204AA8BC1834180369715EDFD56A9
:10CC200014A3D84083250D00BA9794A3C84003D617
:10CC3000090022959730FB1FE780E06F83D709003A
:10CC40003E944204418005F0835789002310FA0086
:10CC5000E39C0DF4A94D89BFB48783250D0014A36F
:10CC6000D840BA97B887218398A3C84003D6090053
:10CC700022959730FB1FE780006C83D709003E9414
:10CC80004204418061B583D7AB002310FA0065BF31
:10CC9000814D55BF5D71A6C2CAC0AA8403598500E3
:10CCA0002A21A2C44EDE52DC5AD85ED662D466D2A5
:10CCB00086C656DA6AD06ECE2E8BEF70DFAA930B43
:10CCC000D5FF7115131A0501B73900200144135A15
:10CCD0000A01373C0020B73C002093894915635B6B
:10CCE0007413D424AE241307E1001386D4004A85BC
:10CCF000EFF06FA12A8D630F05100359A5000C25D5
:10CD00003087AA20EFF07FC7631B051083C844005B
:10CD100083A64CF83087AA20528881471307ACF7C6
:10CD2000EA85EFF0EFEE930DACF713884CF865E968
:10CD300005C883D70D0003D7290089076308F706C4
:10CD4000B7350020138745153E23AA209385451546
:10CD50003354F40202A3EF802FA00DC559451DA046
:10CD6000AA2041664D4781467D16A545EFD0EFCEFE
:10CD7000B737002023A2A900138847F81DE123102C
:10CD80002B014545B640264496440649F259625A5D
:10CD9000D25A425BB25B225C925C025DF24D6161F1
:10CDA000828083D70D0089072391F90083D70D0076
:10CDB000A29763D1770783A749000357AD00930A71
:10CDC0002400A29798A305049317040103A4490023
:10CDD000C183C20A3E948357AD008325080093DACD
:10CDE0000A01A1831CA003A5490003D60D00569596
:10CDF0009730FB1FE780205403D40D00C167FD1757
:10CE0000569442044180E30CF9EC05094209135998
:10CE10000901F1B529450DF423102B01A5B76DDCEF
:10CE200005B71E2181E789473E858280411126C2D0
:10CE3000444122C406C64AC09420D0402A8437F513
:10CE400006008945130505A9EF70CFFD11C93C20E7
:10CE50002547E51793F7F70F6376F702E14721A817
:10CE60009420D04037F5060089451305C5A9EF7019
:10CE70006FFB71FD8947B2402244924402493E85CE
:10CE800041018280373900208356C9EE8547130956
:10CE9000C9EEF5D21A203697C166E3CEE6FC91655D
:10CEA0009385257031459730FB1FE780A019AA8430
:10CEB000CD4771D1314681459730FB1FE780404E09
:10CEC0001E208355090001460147B386E500C206CE
:10CED000C182636BF702AE97C207C18319C22310E8
:10CEE000F90023A004002146A28513854400973051
:10CEF000FB1FE7804044B7370020938787F89843AB
:10CF000009EF84C3814785BF5040131547000507CB
:10CF10002A9636A6054655BF3E871C43F5FF04C337
:10CF200099BF011106CE22CC26CA4AC809E9894414
:10CF3000F240624426854249D244056182802AC675
:10CF40002A84280036896C845085EFF09FEDAA84EE
:10CF500065F1E30F09FC3E24F9DB9165938555707B
:10CF600031459730FB1FE780E00D05C53E242320A7
:10CF70000500232425015EA1B7370020938747F9D8
:10CF8000984301E788C36DB73E871C43F5FF08C38C
:10CF900045B7CD4471BFB73700209387C7F79823B3
:10CFA0000DE3054798A3058909CDB736002037352D
:10CFB00000209386C6EB414691451305C5E76FF007
:10CFC0005FF601458280B73700202380A7EE82807C
:10CFD000C167FD176315F5002E856FE02FB641116F
:10CFE00006C6EFE02FB009C5FD571EA123010500BD
:10CFF000B2404101828001114AC806CE22CC26CA25
:10D0000085472A896392F5044A85EFE04FE131E9CB
:10D01000C16437F606009385F4FF1307E1008946E3
:10D02000130606A70545EFE01FEE2A84FD1405C48C
:10D030004C444A85EFF0DFF9308722858146A6858A
:10D04000EFF0EFB12A84E5B789476396F50085458F
:10D05000EF20200255D9F2406244D2444249056192
:10D060008280EFE00FD76DB7011126CAB7340020D8
:10D070009384C43A22CC8834373400201304C4F893
:10D08000B73700203737002006CE4AC84EC62320C7
:10D09000040023A807F8232007F859C1138907F9CA
:10D0A0009307200C3305F50291659385157093095C
:10D0B00007F81905420541819730FB1FE78080F88A
:10D0C00090349307200C81453306F60208C01906F8
:10D0D0009730FB1FE780C02C1C4098348145938615
:10D0E000870B7D5563E8E5069306800BB306D702F0
:10D0F0000146FD550507B6972320F900BE868EA28E
:10D10000ACB2ACA22382060005069906E369E6FEEE
:10D11000F95696A399463307D702BA9723A0F90088
:10D1200037C5040013054594EFD0EF8C37C50400D4
:10D130001305A5AFEF700FD637C504001305658A38
:10D14000EF10306AF2406244D2444249B24901458C
:10D15000056182802394A6F41386C6F4231006008A
:10D16000232406003106E31BD6FE85059386860B35
:10D1700095BF411106C622C42A84EFC08FA7EFE0F5
:10D180000F9EB7370020A38F87ECB737002003A589
:10D1900007F8EFE0AF9AB7370020238787EE2244E5
:10D1A000B24037D50400130565FF41016F1070636D
:10D1B00093970501C18763D10730B737002003C5B6
:10D1C000F7ED797122D45AC806D626D24AD04ECE6F
:10D1D00052CC56CA2E8B9730FB1FE780600B2A84F7
:10D1E00029C518219307000B631EF702B7340020EE
:10D1F0008547938444F8DC849C4023150100B9E3FF
:10D20000EF0080759165938535709730FB1FE7803F
:10D2100060E388C005E99C8491C74C201305840015
:10D22000EFD0AFD92285EF505FF9B250225421657B
:10D230003345AB0092540259F249624AD24A424BFA
:10D2400045618280373A00206146814513054A15C1
:10D250009730FB1FE780C0140349440089479304BB
:10D260004A15D289930A4A15631AF904F5258AA04A
:10D270002A2093054A15EF705FB63A209E201624A7
:10D2800001ED63E3F6001EA40E243A85EFC05FF7BC
:10D290002285EFC03FCC41B763E3F6001EA41E24F5
:10D2A000D945938649150D463A852390FA00EFC07B
:10D2B0007FE08D4571DD1385491565A89947631990
:10D2C000F9029305A1002285EFF02FD3AA8469D13A
:10D2D000D947639EF40C05092A201379F90FD94523
:10D2E000938649154A86EFC0FFDCCA8555D1E1B760
:10D2F000A1476318F9009305A1002285EFF09F99DB
:10D30000F1B7A947631AF9060A246C009730FB1F8E
:10D31000E780C0732A89630905122A2041669306B3
:10D32000E10055477D16AD45EFC03FF3C8C0AA8662
:10D3300025CD834844000358E10030862A208147E8
:10D3400013074A15CA85EFF0AF8CAA84631F050C3A
:10D350002A2093054A15EF70DFC51DD92A209306B0
:10D360004A152D46D945EFC0FFD41DD1AD45130553
:10D370004A15EFD08FC429BFB147631BF90C0A24AB
:10D380006C009730FB1FE780606CAA8455CD2A2083
:10D3900041669306E10059477D16B545EFC0FFEBA6
:10D3A00023A2AA00AA8631E11E24C5447C85183038
:10D3B000D147E30FF7EC5C202A20938549152380A1
:10D3C000FA003C8523829A002391FA00EF700FD077
:10D3D000E30005EC2A20938649150546D945EFC0A0
:10D3E0007FCDE30705EA8545F9B583484400035836
:10D3F000E1003E2430862A20A68513074A15EFF067
:10D400002F81AA841DE12A2093054A15EF70BFBF22
:10D41000E30005E82A20D94593064A153546EFC0B2
:10D420007FC9B545E30605E679B5D9476393F400AE
:10D43000814403A54A009730FB1FE780A0CDE38914
:10D4400004E41E247C85A5B71E2485447C8585B70D
:10D45000B9476318F9009305A1002285EFF0EFA406
:10D46000B5B5C1476318F9009305A1002285EFF017
:10D47000CFE3A9BDC947631AF900130691009305CC
:10D48000A1002285EFE03F9491B5D947631DF900D3
:10D490009305A1002285EFE03F84AA84E31A05E208
:10D4A000A3040100F5B3E147E314F9DE9305A100FD
:10D4B0002285EFE04FF119BD01458280F9CE0111BF
:10D4C00052C42E8A854522CC4EC656C206CE26CAE6
:10D4D0004AC8AA8AB6893284EF10B039D1471DC52F
:10D4E000B73700203737002083C707FA834617FA7B
:10D4F000814419E0B684BE8637370020032787F9B8
:10D5000093974400BA9763EDD400D547F240624444
:10D51000D2444249B249224A924A3E8505618280FC
:10D520003E89C10703D727FF09C7850493F4F40F89
:10D53000D9BF31CC9565938525C01305000297307E
:10D54000FB1FE78020B02326A90061D1130600024B
:10D550008145938404049730FB1FE78060E4231126
:10D56000990023000900231359010DC43737002007
:10D570001C34032607312304F900118C8327C900CA
:10D5800011841180C0AF23A02901814741B7232610
:10D590000900C1BF23044901FDB785473E8582804C
:10D5A000B737002083C507FAB737002003A787F9EC
:10D5B00081476395F5008146368582803223BA869D
:10D5C00019C2E30BA6FE850793F7F70F4107D5B7FE
:10D5D000B737002003C607FAB737002003A787F93B
:10D5E00081476315F6008146368582802E23BA86F0
:10D5F00081C54C23E38AA5FE850793F7F70F410702
:10D60000CDB7B737002083C537FAB737002003A757
:10D61000073181476395F500814636858280122364
:10D62000BA8619C2E30BA6FE850793F7F70F4107E9
:10D63000D5B7B737002003C817FAB737002083A73C
:10D6400087F901476315E800814636858280B22359
:10D65000BE8609CAF2236317A600D04701C632224C
:10D66000E305B6FE05071377F70FC107E1BF4111C8
:10D6700022C4404526C206C6AA8415C0484409C52E
:10D680009730FB1FE78000A9484809C59730FB1F6A
:10D69000E78040A822859730FB1FE780A0A726855A
:10D6A000414681459730FB1FE78080CFB24022443E
:10D6B000FD579CB4924441018280011122CC2A84FE
:10D6C0002A2106CE2EC6EF102068324622858145DB
:10D6D000EF00F05622856244F24005616FF03FF999
:10D6E00005C53A21411122C406C62A8411CBDD4565
:10D6F000EF00F05722852244B24041016FF03FF71E
:10D70000B2402244410182808280411126C2B1464A
:10D710009304C5FFB386D402B737002013870732BE
:10D7200006C622C4369736276397B602484305C516
:10D73000138407329307F00F6305F6001C21639CE6
:10D74000C7009730FB1FE780E09CB147B387F40226
:10D75000A29723A20700B240224492444101828052
:10D76000411122C42E8426C24946AA8481452285BD
:10D7700006C69730FB1FE780A0C295CCDC2C139720
:10D780004700B737002083A70731BA979A231AA01A
:10D79000BA23FE233AA0373700200357E7F95AA0EF
:10D7A0009A207AA0BA201AA4DA203AA4FA205AA41D
:10D7B0009A241EA87AA4B240224492444101828055
:10D7C000B737002083C507FAB737002003A8073111
:10D7D000B737002003A687F9014781476394E50026
:10D7E0003E858280142299CA544689CAD42E920654
:10D7F000C2966315D500850793F7F70F05071377D2
:10D80000F70F4106E1BF130600643386C502930695
:10D810009500AA8537D504001305056E6F608F85C6
:10D82000411122C406C62A840835EF60AF9EFD5719
:10D830001CB4B240224441018280011122CC4AC86A
:10D840004EC652C456C25AC006CE26CA2A89AE89CE
:10D850000144373A0020B73A00201D4B83471AFA9B
:10D860006365F40463990902B7390020373A002050
:10D87000930AF00F83C709FA6364F4061144A144C4
:10D880002285050442041306F00FCA854180EFF09B
:10D89000DFE7E31794FEF2406244D2444249B249C2
:10D8A000224A924A024B0561828083A78AF9931427
:10D8B0004400BE949C208DC3FE20639F2701639586
:10D8C0006901AA20EF10404826854E868145EF0069
:10D8D00010372685EFF0BFD905041374F40FBDBFD0
:10D8E00083278AF993144400BE949C208DC39C34F2
:10D8F000638F5701FE20639C27012685EFF05FF2BE
:10D900002685D145EF00B0362685EFF05FD60504B9
:10D910001374F40F85B741677917630BE502411162
:10D9200022C406C685472A846399F50022852244CD
:10D93000B240814541016FF05FF089476396F50081
:10D940008545EF1000737DD1B240224441018280B1
:10D9500082809D456FF07FEEB737002003D5E7F951
:10D960008280B737002003C7C7F9011106CE688748
:10D970006C8685476318F70070009305E100054544
:10D98000EF50F01DF24005618280A947631DF60249
:10D990009C319821A207D98F1EA1BC31B821A207C2
:10D9A000D98F3EA1DC31D821A207D98F5EA1FC31ED
:10D9B000F821A207D98F7EA19C359825A207D98F7F
:10D9C0001EA501458280054582809147631EF600B1
:10D9D0009C319821A207D98F1EA1BC31B821A20782
:10D9E000D98F3EA101458280054582809387C5FF7E
:10D9F00093960701C1820D47636ED7003147B38705
:10DA0000E7023737002013070732BA97A8A38EA37F
:10DA100001458280094582809306402037370020E7
:10DA2000AA8763F4A60093074020F117231FF7F895
:10DA3000B73700202381B7FAB73700202382B7FA1F
:10DA400082801905956542054111938535C0418154
:10DA500006C69720FB1FE780E05E01C9B240E9558A
:10DA600041011723FB1F67002378B24041018280E8
:10DA7000B7370020238107FAB737002079710547AF
:10DA8000238E07F8B7370020238EE7304ECEB73706
:10DA90000020B739002022D426D24AD037340020C3
:10DAA000B7340020A38207FA37390020B7370020A7
:10DAB000938939FA06D652CC2AC6230004FAA380E9
:10DAC00004FA239F07F8232C09F823800900EF109C
:10DAD00040303245B737002013060003238AA730B1
:10DAE000373500201305053281459730FB1FE7804D
:10DAF000208B373A002003450A35130404FA938437
:10DB000014FA130989F905CD9565938545C0120569
:10DB10009720FB1FE7800053373700202328A730CA
:10DB200019CD03460A3593070A359C332380C90073
:10DB3000814512069CA09730FB1FE7806086B737AF
:10DB4000002003C5473B9C209565938555C03E95B5
:10DB50001375F50F08A012059720FB1FE780804E74
:10DB60002320A90051C11020814512069730FB1FC8
:10DB7000E7800083032709001420814725077D568D
:10DB8000639EF604EF104045B1473305F5029565F5
:10DB9000938565C0420541819720FB1FE780804A3D
:10DBA000B737002023ACA7302A8401CDEF10C04244
:10DBB00031463306C502814522859720FB1FE78049
:10DBC000207E2254B25092540259F249624A37E5FB
:10DBD00004001305659145616F10A040850710A3EF
:10DBE00093F7F70F410769BF230004002380040067
:10DBF00051BF41119397050126C206C622C44AC0EF
:10DC0000C187AE8463DE07083739002003454931F8
:10DC10009720FB1FE780C0672A8429C91821930732
:10DC200000096312F7041831CD476319F706B736B8
:10DC300000200348250003C5B61F3737002083475F
:10DC400027FA1306640081458146130727FAAA883C
:10DC50006316D80291C11CA31C2391C70345493107
:10DC60008545EF509F8E2285EF502FD52165258D5C
:10DC7000B240224492440249410182800C22AE9774
:10DC800093F5F70F93F7F80F63F4A50093F7F50FEB
:10DC9000850693F6F60F090685455DBF092BE1B7AA
:10DCA00093F715000145E9D7EF00305209CDB7379A
:10DCB000002083C727FA81CBB737002003C547313F
:10DCC0008545EF509F8813C514005DB785462A87A8
:10DCD00063FFC6029C319021A207D18F1EA16399D8
:10DCE000D700BC31B421A207D58F3EA10145828067
:10DCF00089460145639ED700BC31B421A207D58F68
:10DD00003EA3DC31D421A207D58F5EA382800545D6
:10DD100082809147631EF6009C319821A207D98F1B
:10DD20001EA1BC31B821A207D98F3EA10145828036
:10DD3000054582809147631EF6009C319821A20719
:10DD4000D98F1EA1BC31B821A207D98F3EA10145B0
:10DD5000828005458280A1476318F6029C31982194
:10DD6000A207D98F1EA1BC31B821A207D98F3EA12D
:10DD7000DC31D821A207D98F5EA1FC31F821A2079E
:10DD8000D98F7EA10145828005458280894763192C
:10DD9000F6009C319821A207D98F1EA101458280EF
:10DDA000054582803E2279714ECE06D622D426D2F7
:10DDB0004AD01307F007AE896371F70209473AC4E6
:10DDC0007C86300093F5F50FEF00F076B2502254C8
:10DDD00092540259F249456182805A22D9462A89D1
:10DDE000328463F7E6007E2263F4F6006379F7007D
:10DDF00023140100300093F5F90F4A85F1B70A2288
:10DE000002C4EFF01F80AA8435C5EFF07F9B9C24ED
:10DE10006369F5001146A246CE854A85EF00706819
:10DE200075B7340026869305F00F4A85EFF00FE9A9
:10DE300075F1A2471A24DC479AA33A20BAA35A20C4
:10DE4000DAA37A20FAA3DA209AA7DC4495C793F4E0
:10DE5000F90F2286A6854A858297C167FD172A8613
:10DE6000E31BF5FA22459947F9451CA144A1EFF0BF
:10DE70009F99A9BF094645B7014671BFA947631DD0
:10DE8000F6029C319821A207D98F1EA1BC31B8217E
:10DE9000A207D98F3EA1DC31D821A207D98F5EA17C
:10DEA000FC31F821A207D98F7EA19C359825A207C5
:10DEB000D98F1EA501458280054582809C211CA129
:10DEC0009C311CB1BC31B821A207D98F3EA1828000
:10DED00023220500D82189476304F7000545828085
:10DEE000F6210D47E37CD7FE9C45011106CE22CCDE
:10DEF00026CA4AC84EC684339023A204D18C138606
:10DF000044006311D604A033BC23AE8922045D8C87
:10DF10009307C4FFC207C1832A896361F70203A57F
:10DF200089002311990023108900F1559720FB1FC8
:10DF3000E780802B2322A900014531A02285EFF044
:10DF40002FE671FD0545F2406244D2444249B24990
:10DF500005618280397122DC2E841C204AD806DEBD
:10DF600026DA4ED619472A89B2856392E706302011
:10DF70002800EFF01FDAAA8405E92884EFF04FE2C9
:10DF8000AA890C3015C937F704002E861307A7C8D5
:10DF900034009D454A85EF00702F4E850946814526
:10DFA00079294E85EFF0AFECF25062542685425944
:10DFB000D254B2592161828089477C803C840A8690
:10DFC0007C813C857C824A85EF00F056F1BF494751
:10DFD0006398E70232202800EFF0FFD7AA8469F5A2
:10DFE00037350020130505325E2599E381446DBF66
:10DFF0001830142068253C000146CA85CD2C6DB729
:10E000005147639EE70032202800EFF01F98AA8452
:10E0100041FD0C3030004A85EFF0DFD871B7594729
:10E02000639BE70432202800EFF03F9AAA842DFD7D
:10E030002C844A85EFF0EFDF05C9584534851E234F
:10E04000B697C207C1831EA3D5D35C47C5D3B737E4
:10E05000002083C727FAD9DBB737002003C5473133
:10E060008545EF508FCE89B789473EC03C840A86EC
:10E070000C307C8289BF0C300A8623100100EF002F
:10E08000904BADB75D71A6C256DA86C6A2C4CAC0AF
:10E090004EDE52DCAA8A8831AE8432C6EFF04FD30E
:10E0A000B24501ED8144B640264426850649964492
:10E0B000F259625AD25A616182802302050023110B
:10E0C000050083C9040085472A846399F900B020BC
:10E0D0002808EFF0BFBFAA8405491DA09D476391A2
:10E0E000F90418218D47E31FF7FAB02028080549E5
:10E0F000EFF05FC4AA8409E50546814522858126A3
:10E100002285EFF0EFF108243C080147CE862686F1
:10E11000D685F12AE30909F82285EFF04FD561B7DA
:10E12000CD47639BF90018219147E31DF7F6B02016
:10E130002808EFF0BFC545B7D547E395F9F6034A80
:10E1400005008947E310FAF6B02028080549EFF0EA
:10E15000FFD2AA8455F583570102A1EBB8841306B8
:10E16000F0035C44930607FCC206C182636AD600D2
:10E17000B085D94663F6C600B486D94563EDD500AF
:10E180002A20BAA30549EF00303C03560102D2858C
:10E190002285A92CB5B7AC87BAA3D2A38EA3F6A3C8
:10E1A00085471CA0014A0149CDB7014AF9BF7971E1
:10E1B000AA8522D426D22221AA84280806D6EFF0E6
:10E1C0003FD1F24599E53DE185452285EFF06FF9B4
:10E1D00075A0BC8415476395E706B8858D4763F73E
:10E1E000E7046800EFF09FCD3887DD4763FBE70069
:10E1F0008C86B70717008507100822853EC8EF00F8
:10E2000090333C87B88591076305F7002285EFF0CE
:10E210004FF41C8672466C00858B1106228591CFC7
:10E22000EFF05FE601C52285EFF0AFF2884449DDEB
:10E230009720FB1FE78000EE41BFEFF0BFD1DDB7B5
:10E2400011476389E7001387A7FF4207418385468B
:10E2500063EBE6023147F117B387E7023737002057
:10E2600013070732BA979A2371D3A8233008A285DF
:10E2700005204DFDB8849147E318F7F4B2502254BD
:10E280009254456182802C082285FD2445F1FDB71A
:10E2900001114AC82A89314526CA06CE22CC2EC68B
:10E2A000B2849720FB1FE78040F921C1B245930754
:10E2B000000A1EA12EA12A84214611058DC0A68523
:10E2C0009720FB1FE7802007A2854A85EF40DFF3F8
:10E2D0000145F2406244D244424905618280814551
:10E2E0009720FB1FE780C00BC5B70545DDB77971E7
:10E2F00026D2AA841305000206D622D42ECE32CC12
:10E3000036CA3AC83EC69720FB1FE78000F329C5EE
:10E310006246F2454247D246B2472A84130520FAA4
:10E3200008A010B02EA058A054B013058400614678
:10E3300091CFBE859720FB1FE780E0FFA285225486
:10E34000B2502685925445616F401FEC814597205D
:10E35000FB1FE780E004DDB7B250225492544561C0
:10E3600082805845797122D406D62A84AE862DC77C
:10E370003E23FC85930720066397F504B7370020FA
:10E3800003D6E7F97E236373F600B28713F6F70F1F
:10E390002E2B1C2B8D8F93F7F70F81E5890793F7B1
:10E3A000F70FB297FD17B3C7C702FC863E206E2059
:10E3B0000824FC8401473C080146EFF05FF3B250AB
:10E3C000225445618280582FB737002083A7073138
:10E3D0001207BA97FE23D1BF2EC6194681452808D9
:10E3E0009720FB1FE780C0FBB246C9B7797122D4E2
:10E3F00006D626D22A8499CD814701479306000686
:10E400002E866E200824EFF09FEEB25022549254D4
:10E4100045618280B284280059469720FB1FE7801F
:10E4200020F8648499E43E2048446C007C85EFF039
:10E430002FB33C000147930600060146D9B7797116
:10E4400006D6814791E93E21584570867C843C0080
:10E4500001C73E237C853C002E866E21082501479E
:10E4600093060006EFF0BFE8B2504561828041118B
:10E4700022C406C61C2111472A846392E7022E8615
:10E480006E21082581470147CD46EFF05FE64946FA
:10E490006E202244B240154541016FF00FA713F7DB
:10E4A000B70F89466317D7000146EFF03FF4514696
:10E4B000C5B70D476398E7002244B24001464101C9
:10E4C0006FF0FFF7B2402244410182809A21B146A9
:10E4D000B737002071173307D70293870732BA97EF
:10E4E000D84301EBD841AAA70145D8C3BA219AA7BE
:10E4F000828059458280797122D4404526D24AD003
:10E5000006D6AA842E8931C4484419C59720FB1F1A
:10E51000E78040C0232604001E20EE2088247C854E
:10E520003E200147930640067C861E244A867C874F
:10E530001C483EC8BE207C843C00EFF05FDBA30E8D
:10E54000240123280400B2502254925402594561F8
:10E5500082802800314681459720FB1FE78040E4F8
:10E56000BE20EE2088247C8401473C0093064006B0
:10E570004A86EFF0DFD7C1BF797152CC2A8A8A214F
:10E5800026D206D622D44AD04ECE56CAAE84EFF05A
:10E590002F8119E1854795A84045AA8965DC7E2130
:10E5A000E39A47FF1E2463890710542CB73A0020D2
:10E5B00003A70A319206FD173697C2077A23C18353
:10E5C0001EA46316F70093053006EFF09FD95C4850
:10E5D000A5EFC840034915001C2122093369F90041
:10E5E000BE2013072900631CF702F9559720FB1F73
:10E5F000E78080BFC8C02391240103C58900268617
:10E60000D285EFF0FFC8814721E1B25022549254E5
:10E610000259F249624AD24A3E8545618280956537
:10E62000938515C04A859720FB1FE780A0A148C8A5
:10E63000C840231C2401F9559720FB1FE780C0BA6E
:10E64000BE20C8C0F917BEA0484825CDB220362C40
:10E650001E2C3308D60063C80707582C83A70A313D
:10E6600095451207BA97BE2363C90705CC40369576
:10E670009720FB1FE78020CC3A2CBE20BA97C20718
:10E680001A2CC1833EACE397E7F003D7290003C5FA
:10E690008900300078845848D2857C853AC6EFF0EE
:10E6A0003FBF11C548489720FB1FE780A0A6232A3B
:10E6B0000400232C0400F9BD99454E85EFE0FFFFCF
:10E6C000D1BDA545DDBF9145CDBFBA2171CBB737CF
:10E6D000002083D6E7F9ED4763E5E60C011122CC73
:10E6E0002E8426CAAA844840914506CE9720FB1F57
:10E6F000E78080AF3E20AA861CA13E20A1831CB1EA
:10E700001E203CA11E20A1833CB13220C167F91715
:10E710001106420641826394F4042AC4314532C68C
:10E720009720FB1FE78060B1AA85CD471DC19307E5
:10E7300000F91CA13246F957A2463EA189475CA1C7
:10E74000B737002072A114C503C54731EF40DFABD6
:10E750008147F2406244D2443E8505618280814512
:10E760002685EF405054AA8711E9B736002003C729
:10E7700026FA65D37D172381E6FAE1BF09476304D2
:10E78000E5021D476303E50249476302E5027D4751
:10E79000E311E5FCB736002003C726FA8147D1BF55
:10E7A000ED473E858280D1476DB791475DB7894778
:10E7B0004DB701114AC831471309C5FF3307E902B4
:10E7C000B737002026CA9384073206CE22CCBA94EB
:10E7D000D84029C713840732B737002083C627FAE9
:10E7E000854795C668849E24AA242C003AC67C8559
:10E7F000EFF0BFED11C5C8409720FB1FE780809167
:10E80000B147B307F902A29723A207008547F24058
:10E810006244D24442493E85056182808147C5BF3A
:10E82000797126D24445373700204AD0FE2003595B
:10E83000E7F952CC06D622D44ECE56CA2A8A63F3C2
:10E8400027013E89BA284209135909019E2835CF6C
:10E85000998F4A8463D52701139407014180894524
:10E860002285EFF00F9EAA89CD4A31C5BE202AC667
:10E8700060857C84BE2899EB9E28930925001CA105
:10E880009E28A1831CB1637424058228BE28CC4431
:10E8900022864E85BE959720FB1FE780C0A90355B1
:10E8A0006A002C00EFF07FE2AA8A15C54E859720FA
:10E8B000FB1FE7802086B25022545685925402599D
:10E8C000F249624AD24A45618280890759B7791470
:10E8D0004204418065BFBA289E203A94FD17C207C2
:10E8E00042049A28C18341809EA0A2A86376E400D6
:10E8F000F9F3FD57DCBCC1B781455285EFF0BFBFCE
:10E900005DBF79714AD03739002052CC034A59FA99
:10E9100022D456CA5AC85EC662C406D626D24ECE85
:10E920005284B73A0020054B930BF00F373C002080
:10E9300083A78AF993144400BE9483C90400639B9F
:10E940006907DC44A5CBD84735C79A2329CBB7370D
:10E95000002083C727FA99CF2685EFF07FECAA85A0
:10E9600015E9B737002083C717FA05046351F4028D
:10E97000A30289FAB25022544E8592540259F249A8
:10E98000624AD24A424BB24B224C45618280A3027A
:10E9900009FACDB72685EFF01FB68149E1BFDC3F0C
:10E9A000639A7701930520062685EFF09F9BDC4450
:10E9B000A38E070083471CFA05041374F40F6363E6
:10E9C000F4000144E31644F7C9BF4111154506C6DA
:10E9D000EFF03FDE09C50545B2404101828019458F
:10E9E000EFF03FDD6DF91145EFF0BFDC6DF51D4532
:10E9F000EFF03FDC6DF1B737002083C717FAE9DF8E
:10EA0000B24041016FF0FFEF9E210D47F117C207A1
:10EA1000C1836363F706DC41A5C3411122C42E8480
:10EA2000854526C206C6AA84A92529C92685B92BEB
:10EA3000C167F917638FF40009ED3E2099CB1620CA
:10EA400019476393E604373700200357E7F963FD5E
:10EA5000E702B737002083C727FAA285268599C722
:10EA60002244B240924441016FF03FC62244B2407A
:10EA7000924441016FF09FA5094582805145B24003
:10EA800022449244410182806D45D5BF397126DA16
:10EA90004ED6AA84AE895D4589454AD806DE22DC79
:10EAA000328936C63AC4EFE0DFF935C122472A84FD
:10EAB000014511C7B24613054400B6850297935726
:10EAC000850023003401A30024013CB09547FC8459
:10EAD000B737002083C727FA28A01105E88522CE82
:10EAE0002C08268595C3EFF05FBEAA8411C5228548
:10EAF0009710FB1FE7800062F2506254268542594E
:10EB0000D254B25921618280EFF05F9CF9BFCD44AD
:10EB1000E5B7797126D24AD052CC56CA06D6BA8AFF
:10EB200022D44ECE19472E89B284368A6395E506E3
:10EB30002A220944EFE0DFA62AC635C55C45835981
:10EB40006500BE239EA0B247B7360020154723803C
:10EB5000570103C6C631BAA3130716001377F70F80
:10EB6000238EE630D0A301E70547238EE6305147D8
:10EB70006317E9001547BAA0DC479A249AA7528781
:10EB8000A686CA854E85EFF07FF02A84324515C4EB
:10EB9000EFE0FFAD09A842867400BE85AA89EFE0C8
:10EBA000FF912A844DD12285B250225492540259A9
:10EBB000F249624AD24A45618280F945EFE0BFC41A
:10EBC000DDB79E211CA19E21A1831CB1BE213CA1C9
:10EBD000BE21A1833CB1114582809E211CA19E21B2
:10EBE000A1831CB1BE213CA1BE21A1833CB1DE2189
:10EBF0005CA1DE21A1835CB1FE217CA1FE21A18369
:10EC00007CB1214582809E211CA19E21A1831CB143
:10EC1000094582809E211CA19E21A1831CB1BE2199
:10EC20003CA1BE21A1833CB1DE215CA1DE21A183F8
:10EC30005CB1FE217CA1FE21A1837CB19E251CA597
:10EC40009E25A1831CB5294582809A218546AA87E5
:10EC500018A19A21218318B19A216319D700BA21EA
:10EC600038A1BA21218338B1114582800945631D3D
:10EC7000A700BA211945B8A3BA212183B8B3DA2174
:10EC8000D8A3DA212183D8B382809E211CA19E21A2
:10EC9000A1831CB1BE213CA1BE21A1833CB1114581
:10ECA0008280797126D24AD04ECEB2842A89AE892A
:10ECB00029468145480022D406D636849710FB1F8A
:10ECC000E780006E64868DE43E207C82B7370020AA
:10ECD00083D7E7F97C845C4481CFD42F3737002079
:10ECE0000327073192069E2736973A237C8578833F
:10ECF00037F704004A85130747C1540013F6F90F8C
:10ED0000D545EFF0BFD82A8911C195E085471CA0F1
:10ED100023020400014681452285EFF02FEDB25019
:10ED200022544A8592540259F249456182802285D3
:10ED3000EFE0FF93EDB737F70400B2861307A7C4DF
:10ED40002E8685456FF09FD401116887B7F60400C1
:10ED50004165700001489307F00F0D47938626BC6C
:10ED600099457D1506CEEFF0DFDAF240056182802D
:10ED7000B7F60400B28701482E8611479386A6BDD8
:10ED8000C9456FF01FD937F70400B286130767C073
:10ED90002E86CD456FF09FCF011122CC3734002055
:10EDA0001304843526CA4AC84EC606CE2A89AE89BF
:10EDB000930404031C4081C7CE854A8582971104C1
:10EDC000E31A94FEF2406244D2444249B2490561DA
:10EDD0008280B737002003C51720411122C4373481
:10EDE0000020937735001304C43A09811CB4AA9714
:10EDF00006C626C21CA4ADCB1305C0033385A702EB
:10EE0000A5658505B73400209710FB1FE780802398
:10EE100010249307C00381453306F60223AAA434C5
:10EE20009710FB1FE780C05783A744351424014780
:10EE300089077D566341D7022244B2409244373558
:10EE40000020130600038145130585354101171382
:10EE5000FB1F6700E35492A32381070023A5070249
:10EE600005079387C703F9B7B24022449244410192
:10EE70008280011122CC2EC632C406CE2A8497206D
:10EE8000FB1FE78060C12246B24511E9C167F9174F
:10EE90006303F4005145F240624405618280545599
:10EEA0005C218DC213F7270141456314A700154566
:10EEB0007DF2C18B3D45E5D3BC2E0145E3FDB7FC9A
:10EEC0003145D1BFC18B0145F9F71545E9B77971D6
:10EED00026D24AD0B7340020416922D44ECE52CC3B
:10EEE00056CA5AC806D6AA8901449384C43A373A06
:10EEF0000020930AC0037D19054B9C246364F40031
:10EF0000014525A8B307540303274A35BA97BA2306
:10EF10006316270105041374F40FC5B7C833300016
:10EF200093856700EFC091711946CE852800971030
:10EF3000FB1FE7804051E31F65FDB25022549254FD
:10EF40000259F249624AD24A424B45618280B73740
:10EF5000002083C5473BC166B737002003A747356C
:10EF6000FD1681476395F50001463285828003587E
:10EF700027003A866306D80003480700E307A8FE87
:10EF8000850793F7F70F1307C703E9BF411106C6BB
:10EF90009720FB1FE78040B009C54A29B2404101D4
:10EFA00082800145E5BFB737002083C6473BB737AE
:10EFB000002003A747350145814711076393F600F9
:10EFC0008280102301C605051375F50F850793F799
:10EFD000F70F1307C703DDB7B737002003C5473B5B
:10EFE000828037370020930687358147130787359E
:10EFF00031468C4291E58A07BA9788C301458280E1
:10F0000085079106E397C7FE4D458280411106C6EC
:10F0100022C49720FB1FE78020A80DCD2A842A2137
:10F020008545EFF07FD7485409C59710FB1FE7804F
:10F03000600E22851306C00381459710FB1FE780F1
:10F040002036FD573EA0230204000145B240224471
:10F05000410182800945DDBF411106C69720FB1F93
:10F06000E78080A309C54825B2404101828001455F
:10F07000E5BFC167F9176305F502411122C406C651
:10F080002E849720FB1FE78020A1AA87014589C70E
:10F09000C823698C33358000B2402244410182800C
:10F0A00005458280011106CE2EC69720FB1FE78002
:10F0B000A09E854701C95A29B24585476304B70018
:10F0C0004EA98147F2403E850561828029CD01111C
:10F0D0004AC84EC637390020C16922CC26CA52C45C
:10F0E00056C206CE0144AA841309C93A373A002011
:10F0F000930AC003FD1983478900634BF400F24073
:10F100006244D2444249B249224A924A056182800D
:10F110003305540383274A353E953E2163833701E7
:10F1200082940504C9BF8280B737002003C6473BDD
:10F13000B737002083A74735C166014589070147D6
:10F14000FD1691456313E600828003D8070063092A
:10F15000D80003C8A7006315B80005051375F50F9F
:10F1600005071377F70F9387C703E9BFB737002069
:10F1700003C6473BB737002083A647350147814781
:10F1800091066310E602858393C7F7FFC207C18328
:10F1900005456362E50285473395A7004205418135
:10F1A00082808C2299C1CE36CD8F05071377F70F59
:10F1B0009386C603F9B793F61700F1FE050585831C
:10F1C0001375F50FF9B7797156CAAA8A2E8526D21A
:10F1D0004AD04ECE52CC5AC85EC662C406D622D49D
:10F1E000AE84328B368CBA8B3E8AC2894689972090
:10F1F000FB1FE780608A3DED41657D159720FB1F71
:10F20000E78080892A84554531C81946DE85130573
:10F210006400A30284019710FB1FE780C01183578D
:10F22000010326A0230264013EA883574103230063
:10F230005401232604025EA8230644012317340147
:10F2400023182401EFF09FF20AB8232A040226852E
:10F25000232C04028145EFF03FB40145B250225403
:10F2600092540259F249624AD24A424BB24B224C62
:10F27000456182804545DDB7B737002083C6473BEF
:10F28000B737002003A7473581476395F6004165EE
:10F290007D1582803A861307C703835547FF639421
:10F2A000A5002A228280850793F7F70FF9BFB737A9
:10F2B000002003C8473BB737002083A64735416687
:10F2C00001477D16954811436314E800014582808B
:10F2D000BE223685638EC702CC5A9DC9BC31AC2193
:10F2E00089CD938597FD93F5F50FE372B3FE938770
:10F2F000D7FA93F7D70F89EF82809385F7FD93F5BF
:10F30000F50FE3F6B8FC9387D7FA93F7D70FE1D35D
:10F3100005071377F70F9386C6037DB7B73700202D
:10F3200083C5473B4166B737002003A747357D16A5
:10F33000814725486394F5000145828036233A854C
:10F34000638BC600545B81CAB4329386E6FD93F6A4
:10F35000F60FE374D8FE850793F7F70F1307C7037B
:10F36000D1BF011122CC2A84494506CEEF601FC3CC
:10F370001DC12AC622859710FB1FE780E07101CDD1
:10F380006244B737002032460E39F24003C5F73ADF
:10F3900005616F406FB9F240624405618280397146
:10F3A0004ED652D4AE892A8A93053005414526DAD5
:10F3B0004AD856D206DE22DC32C63689BA8A97107F
:10F3C000FB1FE78020C8CD4429C92A848944638172
:10F3D000090432468145F08241469710FB1FE780C1
:10F3E00020FC5686CE8522859710FB1FE780A0F46F
:10F3F0002146630E0902CA8528089710FB1FE78083
:10F4000080F3A28650082C085285EF301079AA8428
:10F4100022859710FB1FE780E0CFF25062542685CB
:10F420004259D254B259225A925A2161828081455E
:10F4300028089710FB1FE780A0F6E1B7411122C40E
:10F44000405926C206C6AA8429CC085409C597107B
:10F45000FB1FE78020CC285809C59710FB1FE780C9
:10F4600060CB685809C59710FB1FE780A0CA285CCD
:10F4700009C59710FB1FE780E0C9685C09C59710B4
:10F48000FB1FE78020C90325040809C59710FB1F4F
:10F49000E78040C822859710FB1FE780A0C723AAFA
:10F4A00004022244B73700208E38B240924403C58C
:10F4B000F73A41016F404FCF411126C206C622C420
:10F4C000AE849710FB1FE780205D29C14C592A8428
:10F4D00095CD83A8C50703A88507FC59B859F42121
:10F4E0009221AC212685EF607FB32285EFF01FF5D6
:10F4F000EFF0DFE201CD2244B7370020B240924462
:10F5000003C5F73A854541016F402F84B24022443C
:10F51000924441018280011122CC06CE2A842EC65B
:10F520009710FB1FE78040575C5989CF9E23B24557
:10F53000639A870085476397F5006244F24005614E
:10F540006FF0DFEFF240624405618280411106C630
:10F5500022C426C2EFF0BFD529C14059AA8415CCD8
:10F560003C209DC7B737002083A7C73889C7DC4335
:10F5700099C32285829738309307F002631FF70002
:10F580002244AA20B2409244814541016FF0DFF24B
:10F59000B737002083A78738D1BFB24022449244B6
:10F5A00041018280411126C24AC006C622C4AA84F3
:10F5B0002E899710FB1FE780204E05CD405955C47A
:10F5C0001E206394970A3C30130710026395E708E6
:10F5D0003C20ADCF7C5403270408DE2B15E313F742
:10F5E000170019CF18545A23058B19CB9307200203
:10F5F0003CB0B24022449244024905454101828018
:10F6000013F7270001CB18545A23098B01C793071E
:10F610004002F9BF918B81CB1C54DE23918B81C7B3
:10F6200093076002F1B7B737002083A7C738F1D33B
:10F63000DC43E1D32285829738309307F00281457D
:10F64000E319F7FA2685EFF03FE765B7B7370020F3
:10F6500083A78738E9BF1307A0026398E700630414
:10F66000090013092003CA85F1BF631C0900268520
:10F670009710FB1FE780404209C55C2193E7070113
:10F680005CA1A6854A85EF604FABA5B7797126D2FC
:10F690009947EC85AA842E858D4522D406D632C69C
:10F6A00036C4FC84EFE0EFB92ACE4D441DC132468A
:10F6B000A246AA85328582962A8419E52C082685D9
:10F6C000EFF08FB42A8411C572459710FB1FE780B5
:10F6D00060A42685EFF0FFC82285B25022549254D0
:10F6E000456182804111B716050022C42E862E8402
:10F6F0009386A6F3894506C626C24AC02A89EFF03A
:10F70000FFF80C20AA844A85EFF01FDBB2402244A8
:10F7100026850249924441018280B737002083A7A1
:10F72000873885CB9C4395C71D71A2CC86CE984166
:10F7300010082A843AC8D84185453ACA829711C52B
:10F7400048862A206C00EFF0FFF9F64066442561F8
:10F7500082808280AE8711CD785501CF142394A189
:10F76000143394B1342BB4A1142F584BB4B1D8C175
:10F770008280414681453E851713FB1F670043C2C7
:10F78000B737002083A7C73891C703A38700630357
:10F7900003000283094582803737002003278759F9
:10F7A0001DC75843AA8705450DC703A50708411182
:10F7B00006C6930605021306050C930505061305F8
:10F7C00005040297B2401375F50F4101828005458B
:10F7D000828082804DC9357122CD2A840A2126CBB0
:10F7E0004AC94EC756C306CF52C55AC1DEDEB68AD5
:10F7F000B2892E899710FB1FE780002AAA8431C5A1
:10F800000C182285EFF01FF53C20138A6400A9CB69
:10F81000EF501FED2A8B014583CB5400EF505FEA78
:10F82000AA840C100818EF10E05408542C10EF10A4
:10F830000055D288268A56C05E88D2875A8714100F
:10F840003010CE854A85EF20207CFA406A44DA44A5
:10F850004A49BA492A4A9A4A0A4BF65B0D618280A4
:10F86000EF501FE8AA8B014503CB5400EF505FE532
:10F870002ACE08540C10EF10E04F2C100818EF108F
:10F880000050F2484DBF8280C14719C91455C14785
:10F8900081CA785511C7BC32BD4663F3F6001C2FF0
:10F8A0003E858280894779C9F1C9411106C622C4C3
:10F8B00026C21C312E849CA13C219CB13C31BCA1B0
:10F8C0005C21BCB15C31858B93968700DE2193F778
:10F8D000F7EFD58FDEA1543193F7F7DFA20693F649
:10F8E0000620DD8ED6A1583193F6F6BF2207137796
:10F8F0000740558FDAA15C31FD769386F67F8D87C0
:10F90000858B758FAE07D98FDEA17421F99B858A0F
:10F91000DD8ED6A178219377270013F7D6FF5D8F70
:10F92000DAA17C2193F647009377B7FFD58FDEA14C
:10F930007821DD9B4D45218BD98FDEA1EF600FE64D
:10F94000AA845145EF608FE5383093F4F40FC9472E
:10F95000636097021375F50F636CE500142011477F
:10F96000E1476367D700143005476363D7008147D9
:10F97000B240224492443E85410182803E8582808D
:10F9800015C1AA8709458DC141112E854146938530
:10F99000170006C69710FB1FE780E099B2400145AB
:10F9A0004101828009458280828089470DC585C5D5
:10F9B000411106C61831AE87194698A19305250056
:10F9C000138517009710FB1FE780E096B240814730
:10F9D0003E85410182803E85828015C1AA87094506
:10F9E0008DC141112E8541469385170006C697109B
:10F9F000FB1FE7804094B2400145410182800945E8
:10FA000082808280894705C99DC5411106C638217B
:10FA10001431AE872207558F9AA1214693053500F0
:10FA2000138527009710FB1FE780E090B2408147C5
:10FA30003E85410182803E85828015C1AA870945A5
:10FA40008DC141112E8541469385170006C697103A
:10FA5000FB1FE780408EB24001454101828009458D
:10FA600082808280894709C981C91831BD46E14732
:10FA700063E4E60098A181473E85828015C1AA878C
:10FA800009458DC141112E8541469385170006C653
:10FA90009710FB1FE780208AB24001454101828018
:10FAA00009458280828015C1AA8709458DC141110F
:10FAB0002E8541469385170006C69710FB1FE780E9
:10FAC0008087B24001454101828009458280828061
:10FAD0001DC1AA87094595C141112E851306000451
:10FAE0009385170006C69710FB1FE780C084B240BD
:10FAF00001454101828009458280828015C1AA8723
:10FB000009458DC141112E8541469385170006C6D2
:10FB10009710FB1FE7802082B2400145410182809F
:10FB20000945828082801D71A2CC2A84084586CE38
:10FB3000A6CA23060100042135479387F4FF93F7F3
:10FB4000F70F6364F70C37E706008A0713070741CE
:10FB5000BA979C4382870C08EFF0DFD4C947631043
:10FB6000F50299475C862A206C00EFF0BFB7F6409B
:10FB70006644D644256182800C08EFF01FEC31C545
:10FB80001C86F5F32A20EFF0CFFDD5B70C08EFF077
:10FB9000FFEEF5B70C08EFF0FFECD5B70C08EFF06F
:10FBA0003FDEF1BF0C08EFF0FFE5D1BF0C08EFF02E
:10FBB000DFE2F1B70C08EFF05FDFD1B70C08EFF030
:10FBC0009FEE75BF1C312308F1002A209710FB1F00
:10FBD000E78080ECA14705C15825631AF702B737C3
:10FBE000002003A7C7389D4719C7184309C7100845
:10FBF000A6850297AA875C8661B70C08EFF05FEDD7
:10FC0000BDBF0C08EFF09FEF9DBF9D47A1BFB73769
:10FC1000002003A78738C1BF011122CC06CE26CA17
:10FC20004AC84EC61821930720092A846313F71285
:10FC30001C3139476393E70A5621096761078147F9
:10FC40006391E610B739002003A5C939CE84630A51
:10FC5000050E0C4403C90500631E09001C2185051F
:10FC60002146A9CF29059700FB1FE780C06C83A719
:10FC7000C439B5C349459700FB1FE780005C2A845F
:10FC80000DC5930710FC1CA1A300250183A5C43951
:10FC90000905414689059700FB1FE780C06983A7D6
:10FCA000C439A2858833EF302FD603A5C439970015
:10FCB000FB1FE780204623AE043831A809059700D2
:10FCC000FB1FE7804067EF30006D05494DF183A7CA
:10FCD000C939238027018547ADA01307E003639846
:10FCE000E70838219547631CF7024A21EFF0CFB6A9
:10FCF0009147E312F5FEB737002083A78738E1DF8D
:10FD000003A38700E30903FC72244A2093056400DF
:10FD10006244F240D2444249B24905610283A1479C
:10FD2000631CF7006C204A206244F240D2444249EE
:10FD3000B24905616FF01F87930600038147E30313
:10FD4000D7FEF2406244D2444249B2493E85056141
:10FD500082809306000A8147E315D7FEEFF0BFDCEF
:10FD6000084435D99700FB1FE780C03AADB78147FB
:10FD7000C9BF011126CA06CE22CC89440DCD85CD3E
:10FD8000AA842E8468008D45EF500FE71C872685D6
:10FD9000228693F7F70393E707046C005C87EF2054
:10FDA000A01DAA8409E90D466C00130534009700D4
:10FDB000FB1FE7804058F24062442685D24405612B
:10FDC00082805D714EDE86C6A2C4A6C2CAC052DC65
:10FDD00056DA5AD85ED6894945CD5DCA138B45009F
:10FDE000420B135B0B01AE8A2A8A930530055A85B4
:10FDF000B2849700FB1FE780E0242A84CD4949C9DB
:10FE0000EF50FF8F2A895686D285935A8900135A5C
:10FE10000901937BF90F1305440093FAFA0F137A43
:10FE2000FA0F135989019700FB1FE7804066A30171
:10FE3000740123015401A300440123002401EF5065
:10FE40007F8BAA85414608089700FB1FE780206446
:10FE5000214734005A86A2850808EF206038AA8915
:10FE60001DE121462C0023807401A38054012381CD
:10FE70004401A3812401138544009700FB1FE78000
:10FE80000061EF509F8822859700FB1FE780802844
:10FE9000B64026444E8596440649F259625AD25AD3
:10FEA000425BB25B6161828001114AC82A892E855A
:10FEB00006CE22CC26CA2EC69710FB1FE780C0BDF7
:10FEC00055CD405955CC5C300947B24593F6B70F34
:10FED0006386E60011474945639DE7061E200945F4
:10FEE0006399B706930484004146CA852685970026
:10FEF000FB1FE78040444146CA85130584019700F3
:10FF0000FB1FE7804043383085469307F7FE93F7A1
:10FF1000F70F63E6F6041306C4033285C14532C603
:10FF2000EF508FCD32469306C402A6852285EFF0AE
:10FF30007F8A3C2089CB22856244F240D2444249E8
:10FF400005616F10C0073830C947E306F7FE3CB0C3
:10FF50000145F2406244D2444249056182809307E0
:10FF600010050145E317F7FE3C20E5D722856244E2
:10FF7000F240D244424905616F10A00A0945D1BF41
:10FF80004945C1BF397152D42A8A328526DA4ED604
:10FF900006DE22DC4AD8AE8932C69710FB1FE78006
:10FFA000A0AFC94451C14059C9443DCC1E2032467E
:10FFB000639CC7065C30A18BB1CB37390020832707
:10FFC00089599304E00FADC39C47B9CF93048401D2
:10FFD00026854146D2859700FB1FE780C0358327E1
:10FFE00089598325040826869C47938505041808AB
:10FFF00081462E858297AA844146CE8508089700BF
:020000025000AC
:10000000FB1FE780404493F4F40F11E1894438303A
:100010009307B005631AF7002285EF00707D3C203E
:1000200089CF9307C0053CB0F250625426854259EF
:10003000D254B259225A216182809307E005E5B774
:1000400039C9011126CA06CE22CCAA8409459DCD04
:100050000D4628002E848D059700FB1FE780A02DFC
:100060001C8570002C0093F7F70393E7070426859F
:100070005C85EF10707019E90D46A2856800970045
:10008000FB1FE780403C7D153335A000F240624401
:10009000D2440561828009458280011152C42A8AB6
:1000A00032854EC656C25AC006CE22CC26CA4AC88F
:1000B0002E8BB28AB6899710FB1FE780E09D09ED71
:1000C0008944F240624426854249D244B249224AD8
:1000D000924A024B056182805C592A89C544F5F336
:1000E0004D45EF50BFEB1374F50F5145EF501FEB2B
:1000F000E38809FC83C78901E3E487FC1375F50FE6
:10010000E360F5FC93053005130540089700FB1FDD
:10011000E78040F3232AA9022A84CD445DD1130647
:10012000400881459700FB1FE7808027A30104005A
:1001300023014401230264012310540123263407C0
:1001400023240402A30204008144E30C0AF622855E
:10015000EF003061AA8435D54A85EFF02FAE95B710
:10016000397122DC06DE26DA4AD84ED652D456D26F
:100170005AD05ECE62CC66CA0944630D0610630B8A
:100180000710AA8B3A89368BB28A2E8C9710FB1FE8
:10019000E78080902A8A5144630E050E930530054E
:1001A00041459700FB1FE780E0E9AA894D447DC1E6
:1001B0008344190083472900A204C207BE948347E1
:1001C0000900BE9483473900E207BE9483278A0260
:1001D00063E697007D5709446399E70A63070C00BB
:1001E00083474A000544898BCDC3930C4B002146BD
:1001F00081450A85C20C9700FB1FE780601A93DCDB
:100200000C019305300566859700FB1FE78080E3AE
:100210002A8C4D443DC95A86D68511059700FB1F8F
:10022000E780E0261146CA8562859700FB1FE780BC
:100230000026414693058A014E859700FB1FE78003
:10024000002521478A866686E2854E85EF10507923
:100250002A841DE521468A8528009700FB1FE78038
:10026000002321469305490028009700FB1FE780E3
:10027000801D8547631EF502A6855E85EF60CF88E9
:1002800062859700FB1FE780E0E84E859700FB1F23
:10029000E78040E82285F2506254D2544259B25964
:1002A000225A925A025BF24B624CD24C21618280FC
:1002B0000544F9B779719397050122D406D626D261
:1002C0004AD04ECEC1872E8463D50704B7340020B0
:1002D0009384C43AA8309700FB1FE78060FB2AC6CE
:1002E00009CDEFF07F93B24511E5A8209307F00FF9
:1002F000631EF5002E85EF205FEC2165218DB25045
:10030000225492540259F24945618280EF20DFEF76
:10031000EDB793F7150091C7EFF04FA31345140005
:10032000F9BFA1E10145E1BF850493F4F40FEFE0CB
:10033000BFCAE3F9A4FE33959900131905011359B7
:100340000901B3772401EDD34A85EFE0FFF2C167DD
:10035000FD176305F500DD45EFF00F9633452401E9
:1003600079BF85448549E1B7B737002023AE073808
:10037000B737002023A6073837170500B737002006
:100380001307A79123A40738B737002023A0E73A23
:10039000370705009387073A13078766D8C337F7EF
:1003A00004001307E73998C737170500B73700204F
:1003B0001307077A23A8E73837170500938707390B
:1003C0001307E734D8C3371705001307E75E98C74C
:1003D0008280B737002083C7073BA18B89C7B73717
:1003E00000209387073A373700202326F738014546
:1003F0008280B737002083C7073B918B89C7B73707
:10040000002093870739373700202324F738014528
:100410008280011106CE2AC6EFF01FF53245B737AC
:1004200000209945A387A73AEFD04FDCF24037F57B
:1004300004001305655105616FE0BFBA1C5581C703
:10044000A1473E858280011122CC26CA2A84AE842F
:10045000130500049305300506CE9700FB1FE780C7
:1004600060BE08D475C113060004A6859700FB1F63
:10047000E78060EC78543C2B93F68700F5CA14545F
:10048000B422A18AF5C683270408DDEF9305300561
:10049000130500109700FB1FE780C0BA2320A408B3
:1004A0008D4745C5A302040078549C30143391EB6A
:1004B00091EABC20918BC5E33C2B918BC9EF85471A
:1004C00001A881C6214758B089C75C3093E707016E
:1004D0005CB06C54BC29858B99CB1C540547BC235C
:1004E0008D8B6396E7007C2093E717007CA0832721
:1004F000040889C77C2093E787007CA05C3005470F
:10050000639AE70A93048400414681452685970053
:10051000FB1FE780E0E84146814513058401970011
:10052000FB1FE780E0E71306C4033285C14532C6EE
:10053000EF409FEC832704083246B9CF2285EF00B5
:10054000502E9307000525C5A147F2406244D244CE
:100550003E85056182809C2014231547B387E702FE
:1005600037E7060013074746BA97B6979C238DB71F
:10057000943089C6143399C2E14799BFB420D58F0E
:10058000918B95DF9C2014231547B387E70237E74B
:10059000060013078744C9BF9306C402A6852285B7
:1005A000EFF04FA32285EF009021C14751FD3CB0F1
:1005B000814761BF13F787012DCFC18B930484005E
:1005C0004146A9C7890526859700FB1FE780A0D66D
:1005D00041468145130584019700FB1FE78040DCFD
:1005E0007C201306C403328593E747007CA0C145F5
:1005F00032C6EF407FE083270408324699CF228538
:10060000EF003022930720055DD13DBF814526854F
:100610009700FB1FE780C0D865BF9306C402A6857C
:100620002285EFF02F9B2285EF007019CD4741D135
:1006300021BF09478545638AE700114789456386DD
:10064000E70019476396E7008D450A20EF50FFB594
:100650007C2093E747007CA08327040881C7930789
:100660001005B1B7C547A1B73C21638B072279714B
:1006700022D406D626D24AD03C31130750052A840C
:10068000639DE706034975001306C503C1459357EB
:100690003900AA973285842732C6EF40FFD5B73795
:1006A000002083A78759A1C79C47B1C3032504082D
:1006B00093767900B3D6D4403246858A93050504F3
:1006C000180893E606081305050882971375F50FB9
:1006D00019ED41460C081305C4029700FB1FE78083
:1006E00080C52285EF00B00D930760053CB0B25085
:1006F000225492540259456182801307100263927A
:10070000E7021C5503270508DE2361E313F70710F2
:100710004DCF78555A2B1377071045CB93077002AE
:100720003CB03C30130770026397E70C3C5885E3FC
:100730009305300571459700FB1FE780A09028D8EE
:1007400019C5714681459700FB1FE78060C5245895
:10075000B1C4BC2C89E72285EFF00F93A8AC2858D0
:10076000814541469700FB1FE78080C328583D47DD
:100770002C2D9387F5FF93F7F70F6364F700EF4095
:10078000BFC7EF207FC23C58A1458AAB1385270124
:10079000EF409FC62C580A20EF00B031930780022B
:1007A0000A203CB09700FB1FE780002F414609C597
:1007B0007E2513D617003E96B737002003C5F73ABB
:1007C00006068545EF205FF61DB713F7072009CB16
:1007D00078545A2B1377072001C79307900289B7E3
:1007E00093F707409DDF7C54DE2B93F7074095DBA2
:1007F0009307B00235B7130780026397E7023C58AE
:1008000099C78E2B0A2013862701EF00F02F1C5466
:10081000DE2313F7072029CF78545A2B13770720AC
:1008200021CB93079002ADBF13079002639BE700B3
:10083000EF40BFEBAA850A20EF00102C9307A0021F
:1008400085B71307A0026390E704EF407FE9AA850C
:10085000854701456384F500814505452EC6EF4077
:100860003FE62A86B2450A20EF00B0251C54DE235D
:1008700093F707409DC37C54DE2B93F7074091CF3D
:100880009307B00231BF1307B0026398E700EF404F
:100890007FE6AA850A20EF00902A9307F002B9B5F7
:1008A0008280411122C4405926C206C67C54AA84C3
:1008B000DE2B13F7071011C718545A2313770710AC
:1008C0000DE313F7072011C718545A231377072095
:1008D00009EB93F707408DCB1C54DE2393F70740B9
:1008E00085C7930710023CB02285EFF0FFD7383060
:1008F0009307F002631EF7002244AA20B2409244FC
:10090000814541016FE05FBB9307F0023CB0EDB75A
:10091000B2402244924441018280397122DC405924
:1009200026DA4AD84ED606DEAA89AE843289630218
:10093000043A2A211E206384A700A14421A03C2060
:1009400091EB9D44F250625426854259D254B259DB
:10095000216182809387E5FF93F7F70F2D47E362CC
:10096000F7FE37E706008A0713070748BA979C4344
:100970008287B2852285EFF07FACAA84E1B7414639
:10098000CA851305C4049700FB1FE780C09A22851F
:100990008525AA8411C1A1443C3013074005639604
:1009A000E700930790053CB071BF1307600563959E
:1009B000E7009307A005C5BFD147F5B79309C40564
:1009C0004E854146CA859700FB1FE780C0960325E8
:1009D000040845C53C30130790056398E70022855D
:1009E0004D259307E0053CB079A01307A00563905F
:1009F000E7087C3013D73700229714279D8BB3D696
:100A0000F640B737002083A78759858A93E606F812
:100A100093F6F60F9DD39C478DD3930505081808D0
:100A20004E861305050482979374F50FE39704F03F
:100A300041460C081305C4049700FB1FE780A0A0E3
:100A40007C304D47850793F7F70F7CB06377F7004D
:100A50002285052D9307E005B9B7B737002003C5F8
:100A6000F73A8545EF207FAE930750052DBF13075A
:100A7000C005E386E7F68144F1B5130984004E868C
:100A8000CA8522851408EFE0FFD441469305C404CB
:100A900008089700FB1FE780009BE30505EA8A86AC
:100AA0001306C403CE854A85EF10206A05E122852E
:100AB000EFE09FDDB73700202A8783A7873A0A2017
:100AC000814601468A858297AA8411C1A144930771
:100AD0002002D1BD0C22EFE03F9E71BF383093075A
:100AE0002002E310F7E67C5889EB93053005714549
:100AF00097F0FA1FE780005568D86858E30305E4CB
:100B00004146CA859700FB1FE780E0826458228532
:100B1000EFE09FD7A8AC93073002F1B538309307C8
:100B20003002E310F7E21E2268582146930529009F
:100B30001EA9490597F0FA1FE780E07F7C54DE2B61
:100B400013F727002DC718545A23098B2DC3930779
:100B5000400251BD383093074002E314F7DE3C5C9D
:100B600081EB85455D4597F0FA1FE780A04D28DCB5
:100B7000285CE30205F0834709004146CA857CA949
:100B800097F0FA1FE780207B93075002A9BD383009
:100B900093075002E317F7DA285C1946930519000A
:100BA000410597F0FA1FE78000797C54DE2B918B8A
:100BB00095CF1C54DE23918B95CB9307600225B50E
:100BC0007C5C89EB93053005514597F0FA1FE7806F
:100BD000604768DC685CE30205D64146CA8597F049
:100BE000FA1FE78040757C5C7D5798CB4E85EFF00F
:100BF0005FCB51B50325040813060004CA8513050D
:100C0000050497F0FA1FE78000732285EFE0DFB854
:100C10003C30130700056395E70093074005E1B3F7
:100C200013071005639CE700B737002003C5F73AA8
:100C30008545EF209F919307500575B31307200555
:100C4000E39BE7E2B737002083A78759E38707CE06
:100C50009C47E38407CE8325040893048400180886
:100C600093850508814626862E8582970A201008DE
:100C7000A685EF506FDC9307B005B5B33830930706
:100C8000E005E310F7CC8325040841464A8597F038
:100C9000FA1FE780407BAD44E30605CA032504083C
:100CA0004146CA8597F0FA1FE780E0682285EFE0A9
:100CB000BFBDB73700202A8783A7873A2C580A2060
:100CC000814601468297AA8411C1A144930710026C
:100CD000D9B9AD47E391F5DA14222E211306650048
:100CE0000821EF407FD641BB894759C2D1C108A234
:100CF0009C211CB29C313CA2BC213CB2BC31A30261
:100D000006005CA2DE21A183858B5CB2DA21137719
:100D1000072001C793E727005CB2DE2193F7074065
:100D200089C75C3293E747005CB2DE211397470125
:100D3000635607005C3293E787005CB2230306002A
:100D4000DC21858B7CA2DA21098B01C793E7270080
:100D50007CA2DE21918B89C77C2293E747007CA28D
:100D6000DA218147218B09C778221367870078A28F
:100D70003E8582802E86AA8505456FF0FFF62E8679
:100D8000AA8509456FF05FF6894785C51DC14111E8
:100D900006C6AE870D47AA8598A31385170041465E
:100DA00097F0FA1FE7802059B24081473E85410104
:100DB00082803E858280894785C51DC1411106C656
:100DC000AE871147AA8598A313851700414697F06F
:100DD000FA1FE7804056B24081473E85410182803C
:100DE0003E858280894785C51DC1411106C6AE87F3
:100DF0001947AA8598A313851700414697F0FA1F53
:100E0000E7806053B24081473E85410182803E8544
:100E10008280894795C90DC9411106C61D4798A111
:100E20001A21AE87214698B11A212183B8A19305D2
:100E300025001385370097F0FA1FE780C04FB240B6
:100E400081473E85410182803E858280894785C5F4
:100E50001DC1411106C6AE872147AA8598A31385F7
:100E60001700414697F0FA1FE780E04CB2408147F7
:100E70003E85410182803E85828089479DC515C59A
:100E8000411106C6254798A11821AE87194698B189
:100E9000930515001385270097F0FA1FE780A049F6
:100EA000B24081473E85410182803E8582808947EC
:100EB00085C51DC1411106C6AE872947AA8598A3DD
:100EC00013851700414697F0FA1FE780C046B240ED
:100ED00081473E85410182803E85828089478DC55C
:100EE00005C5411106C6AE873147AA8598A313856B
:100EF00017001306000497F0FA1FE780C043B240C2
:100F000081473E85410182803E858280894785C533
:100F10001DC1411106C6AE873547AA8598A3138522
:100F20001700414697F0FA1FE780E040B240814742
:100F30003E85410182803E858280894799C511C5E1
:100F400095479CA11C219CB181473E8582808947A1
:100F500099C511C5AD479CA11C219CB181473E8517
:100F600082800DC55D718A8586C6A2C42A84EFE0A1
:100F70006FFE0A20B71605000A86938646D79D4560
:100F8000EFE0CFF0B6402644616182800545828063
:100F90000DC55D718A8586C6A2C42A84EFE08FFBE9
:100FA0000A20B71605000A869386E6D79D45EFE02E
:100FB000EFEDB640264461618280054582805D7117
:100FC000A2C49305C5022A8441460A8586C697F0C5
:100FD000FA1FE78040360A20B71605000A86938676
:100FE00086D8C545EFE08FEAB6402644616182802D
:100FF0005D71A2C49305C5032A8441460A8586C64D
:1010000097F0FA1FE78020330A20B71605000A86FA
:10101000938666DBC545EFE06FE7B6402644616125
:101020008280B737002083A78759A9CB9C435D7185
:10103000A2C486C62A841305E00F8DCF03250408B9
:101040009305050C130505088297832504081306EC
:1010500000040A859385050897F0FA1FE780A02D04
:101060000A20B71605009386C6ED0A86930510047C
:10107000EFE0CFE1B6402644616182801305E00FC6
:101080008280317122DD2A840A2126DB06DF4AD9DB
:101090004ED752D556D35AD15ECF62CD9700FB1FA3
:1010A000E780809F3C58AA8489EB93053005714501
:1010B00097F0FA1FE78000F928D82858CD4705C9CE
:1010C0007146814597F0FA1FE780802D03290407B8
:1010D0002285EFE06FFB230DA9003C20373900206B
:1010E000638107128327895985E39307E00FFA503C
:1010F0006A54DA544A59BA592A5A9A5A0A5BFA4B2C
:101100006A4C3E852961828083AB0701E38F0BFC2B
:10111000032B0408EF40CFDC2A8C0145EF404FDA67
:10112000DC303858130B0B029309C403130AC405AF
:10113000938A64003AC0B337F0002A879308010409
:101140005688B33680015286CE855A85829B1C54C0
:10115000B8232307E1029833A306E1029C23230668
:10116000F10283278959D1D303AB4701E30F0BF673
:10117000DC30B337F0003ECEEF408FD6AA8B01456E
:10118000EF400FD403270408F2472AC03AC2B3380D
:10119000700156887810930684004E86D2858800A8
:1011A000029B7C54B82B2305E1029833A304E1028F
:1011B0009C232304F1028327895903A94701EF40A7
:1011C0002FD22A8B0145EF40AFCF83C854009C0833
:1011D0002A883EC2B3381001B33760013810930635
:1011E00084015286CE8556C0880002990A20B7161F
:1011F00005009386C6F09008C545EFE02FC9AA8781
:10120000FDB5D43083278959032B0408B336D000A9
:1012100083AB070136CEEF40AFCC2A8C0145EF40BF
:101220002FCA3C58F246130B0B02130AC40593094C
:10123000C403938A64002A88930801044E86D285E9
:101240003EC05687B33780015A85829B1C54130BCE
:101250000103B8232307E1029833A306E1029C238C
:101260002306F1028327895983AB4701DC30B3376A
:10127000F0003ECEEF40CFC62A8C0145EF404FC470
:10128000F2472AC0B338800156887810930684004C
:101290004E86D2855AC28800829B83250408414627
:1012A0005A8597F0FA1FE780001AAD47E31B05EE59
:1012B0003DBDB71605002E86938646DEC5456FE018
:1012C000EFBC5D71B287A2C44C802A84BE85130531
:1012D0001100194686C697F0FA1FE780C005B716B9
:1012E00005000A8622859386A6E7A145EFE00FBA9E
:1012F000B640264461618280B71605002E8693862B
:10130000C6E4C5456FE08FB85D71B287A2C46C803A
:101310002A84BE8513052100214686C697F0FA1F50
:10132000E7806001B71605000A862285938626E1CC
:10133000AD45EFE0AFB5B640264461618280B71697
:1013400005002E869386E6EAC5456FE02FB47971D5
:1013500022D406D626D23C31130730052A84638175
:10136000E708130750056392E7089307A0053CB10F
:101370007C31C14513D737002A9714279D8B13055D
:10138000C503B3D6F640858A93E606F893F6F60FC2
:1013900036C6EF406F86B246B737002083A787591D
:1013A0009DCB9C478DCB0325040818081306C40366
:1013B000930505041305050882971375F50F01EDD4
:1013C0001305C40241460C0897F0FA1FE780A0F607
:1013D0002285EFF0DFBEB2502254925445618280E4
:1013E000930790053CB1814645BF130710026391F6
:1013F000E7027C5503270508DE2B61EF13F7170082
:1014000069CB18555A23058B69C7930720023CB056
:101410003C30130720026394E70E3C5889EB930598
:101420003005714597F0FA1FE780C0C128D82458CD
:10143000ADCC2285EFE04FC5A8AC28588145414688
:1014400097F0FA1FE780C0F528583D472C2D938769
:10145000F5FF93F7F70F636DF702B737002083C7E7
:10146000375AD9CB41468145080897F0FA1FE780E3
:1014700020F3B7350020194693850526080897F014
:10148000FA1FE78040EB30580C082E85EF204140D2
:10149000EF109FF13C58A1458AAB13852701EF302F
:1014A000BFF52C580A20EFF0DFE0930730020A2046
:1014B0003CB097F0FA1FE780205E414611C17225CB
:1014C000B737002003C5F73A06068545EF20CFA5BC
:1014D00019B713F7270001CB18545A23098B01C7FA
:1014E000930740022DB7918B85D71C54DE23918B37
:1014F00085D39307600221BFEF301FF051BF130760
:1015000030026396E7023C5899C78E2B0A20138657
:101510002701EFF07FDF7C54DE2B13F7270021CB70
:1015200018545A23098B21C79307400249B7130760
:101530004002639BE700EF404F9BAA850A20EFF033
:10154000BFDB93075002A5B713075002639DE70264
:10155000EF400F9915E5814505452EC6EF404F96A2
:101560002A86B2450A20EFF0DFD57C54DE2B918B22
:101570008DC71C54DE23918B8DC39307600205BF7A
:1015800085450145D9BF130760026398E700EF4026
:101590006F96AA850A20EFF09FDA7C54032704088F
:1015A000DE2B09EF13F7071011CB18545A231377CA
:1015B000071009C7930770023CB031BD13F707202D
:1015C00009CB18545A231377072001C793079002B9
:1015D000E5B793F7074089CB1C54DE2393F7074008
:1015E00081C79307B002C9BF9307F002F1B7397101
:1015F00022DC26DA4ED652D406DE4AD8AE89328AAA
:10160000AA8497F0FA1FE780204940594146814556
:101610000A8597F0FA1FE780A0D835C40359040063
:1016200063139906383093071002631FF70283276C
:10163000040899CF2C58A1C94A85EF10D05605450A
:10164000F2506254D2544259B259225A21618280D6
:101650008A861306C4059305C40313058400EF00AE
:10166000D02E15E18A85C9BF2C5891CD9E29639C47
:1016700047012146C9054E8597F0FA1FE780A0DC97
:1016800019C12C5855BF268597F0FA1FE780C04036
:101690002A84054555D44C54B1C59E296394470509
:1016A0002146C9054E8597F0FA1FE780C0D98547C6
:1016B000631AF502B737002083C777EF89C74C5408
:1016C000BC3D639AA70CBD452685EF105048B7373F
:1016D000002083A707220145A5D71D45894582978C
:1016E0000145B9BFB737002003C7475AB7390020B3
:1016F0009389C91E058B3E8929C3B737002058300E
:1017000083C7C759631BF702B73500201946938575
:10171000D5591305640097F0FA1FE780C0D28547BA
:10172000631DF50083A7490381C791451D45829735
:10173000BD452685EF10B04119B737370020034764
:10174000375A83A7490331CB0347495A098B09CB41
:1017500081C795451D4582972685EF101045C5B573
:1017600081C78D451D45829741468145080897F000
:10177000FA1FE780E0C2B735002019469385052699
:10178000080897F0FA1FE78000BB0C082E850A8630
:10179000EF2001108A8526854DB58545C5FF6DBFB3
:1017A000797122D440594AD04ECE52CC06D626D298
:1017B000AA892E8A3289630604622A211E20638C3C
:1017C000A700A144B2502254268502599254F249EE
:1017D000624A45618280242099C09D44E5B7938781
:1017E000F5FF93F7F70F3147E369F7FE37E7060098
:1017F0008A071307074BBA979C4382871C54F1F35F
:10180000930530051305000497F0FA1FE7808083E5
:1018100008D445D903470900914763F4E7008D4494
:1018200055B7034719008547E3EBE7FE13060004AD
:10183000CA8597F0FA1FE78000B00C547054A302D9
:101840000400D4415C4A858AFD8E5E2AF99BD58FBF
:101850005EAAD841544AF59B0583058B8582F98E93
:101860008606DD8E56AADC41584AED9A8983858B1F
:1018700009837D8F0A07558F5AAAD4415C4A5D9B24
:101880008D82858A8D83F58F8E07D98F5EAAD84188
:10189000544A93F7F7EF2183058BA182F98EA206B4
:1018A000DD8E56AADC41584AA583858B25837D8F22
:1018B0009317970013F7F6DF5D8F5AAAD4415C4A5D
:1018C000A982858AA983F58F9396A7009377F7BF9E
:1018D000D58F5EAAD441584AAD82858A2D83758FF3
:1018E000FD769386F67F2E07F58FD98F5EAA3C2A68
:1018F00003250408A18BF1CFBC21A18BF9CBE31206
:1019000005EC930530051305001097E0FA1FE780FA
:1019100060732320A40801D57C54A302040003476C
:101920001900943399E63DCF5C3093E707015CB032
:1019300021A0A1475CB06DFB2285EFF06FE56C54F0
:10194000BC29858B89CB1C54BC238D8B89C77C20FB
:1019500093E717007CA08327040889C77C2093E7BE
:1019600087007CA05C3005476398E70A41468145C3
:101970001305840097F0FA1FE78080A24146814555
:101980001305840197F0FA1FE78080A1C145130574
:10199000C403EF307FA683270408ADCF930700056B
:1019A0003CB00DB5B82B118B19E703472900118BFB
:1019B00019E38547ADBF9C23154783460900B387CC
:1019C000E70237E7060013074746BA97B6979C2306
:1019D000B9BF19C597E0FA1FE780C0732320040838
:1019E0007C54983311C70347190019C3E14781B7E5
:1019F000B82B118B09E703472900118B5DDB9C2372
:101A0000154783460900B387E70237E70600130747
:101A1000874465BFC14769B713F7870131CBC18BD5
:101A20001305840041468DCF890597F0FA1FE780A2
:101A30008090414681451305840197F0FA1FE780A5
:101A400020967C20C1451305C40393E747007CA082
:101A5000EF309F9A8327040891CB9307200589B71D
:101A6000814597F0FA1FE780A093E1B7CD470DBFFE
:101A700009478945638AE700114785456386E70082
:101A800019476396E7008D450A20EF400FF27C204E
:101A900093E747007CA08327040881C793071005BC
:101AA00001B7C547F5BD4146CA851305C40497F083
:101AB000FA1FE78040883C3013076005639CE7000D
:101AC000B737002003C5F73A8545EF101FA89307E5
:101AD0005005F9B545476383E7029306C402130630
:101AE000C403930584002285EFD0DFCE2285EFF07A
:101AF0000FCDAA8411C1A144D1475DB5C9474DB5E9
:101B00009309C4054E854146CA8597F0FA1FE780C0
:101B100080820325040869C53C301307900563984B
:101B2000E7002285EFF0CFCC9307E00595BD1307C2
:101B3000A0056399E706B737002083A78759E38E8E
:101B400007C803A88700E30A08C87C309305050886
:101B50004E8613D73700229714279D8B0A87B3D65A
:101B6000F640858A93E60608130505040298414667
:101B70008A851305C40497F0FA1FE780C08C11E131
:101B8000D2842285EFF0CFC67C30CD461307E00526
:101B9000850793F7F70F7CB063E4F6001307600541
:101BA00038B00DB11307C005E39EE7C0B73700207A
:101BB00083A78759E38307C29C47E38007C2930545
:101BC0000508130984000A8781464A862E85829774
:101BD0000A200A86CA85EF402FE69307B005C9B3ED
:101BE0008A864E86930584002285EFD0BFBE41468B
:101BF0009305C4040A8597F0FA1FE780C0848547DF
